:100000000C94572E0C94882E0C94882E0C94882EC9
:100010000C94882E0C94882E0C94882E0C94882E88
:100020000C94882E0C94882E0C94882E0C94882E78
:100030000C94882E0C94882E0C94882E0C94882E68
:100040000C94882E0D94DD090C94882E0C94882E27
:100050000C94882E0C94882E0C9425F50C94B8E101
:100060000C94882E0C94D5DA0C94CBDA0C94882E50
:100070000C94882E0C94882E0C94882E0C94882E28
:100080000C94689C0C94882E0C94882E0C94882ECA
:100090000C94882E0C94882E0C94882E0C94882E08
:1000A0000C94882E0C94882E0C943A9C0C94882ED8
:1000B0000C94882E0C94882E0C94882E0C94882EE8
:1000C0000C94882E0C94882E0C94882E0C941D9DD4
:1000D0000C94E79C0C94882E0C94882E0C94882EFB
:1000E0000C94882E084AD73B3BCE016E84BCBFFDE2
:1000F000C12F3D6C74319ABD56833DDA3D00C77FF8
:1001000011BED9E4BB4C3E916BAAAABE0000008090
:100110003F05A84CCDB2D44EB93836A9020C50B91F
:10012000918688083CA6AAAA2ABE000000803F0744
:10013000634236B79BD8A71A39685618AEBAAB5582
:100140008C1D3CB7CC5763BD6DEDFD753EF6177247
:1001500031BF000000803F08000000BE9224491219
:100160003EABAAAA2ABECDCCCC4C3E00000080BE3D
:10017000ABAAAAAA3E00000000BF000000803F001A
:1001800000000000084178D3BB4387D1133D190E0E
:100190003CC3BD4282AD2B3E68EC8276BED98FE176
:1001A000A93E4C80EFFFBE01C4FF7F3F000000006E
:1001B00000000C94E19D0C94125F0D9499370C94FF
:1001C000DA5E0C94525C0D94FB360D9471460C94DF
:1001D00077DB0C9413DB0D94DA370D948B4B0D9475
:1001E00059470C94A89D0C948EDF0D94F1360D9414
:1001F0004E4C0D94D0370D94A3370D946D440D944F
:10020000573A0D94434A0D945F4A0D94C03E0D94A5
:10021000A1440C94C39D0C9495E10D9403460C9459
:100220007FDB0D943D450D94C6370C940EE00C9485
:10023000B4DC0D94BC370C943B970D94D8360D94D8
:10024000E4360D94C1360D94AD370C943ED70C9422
:1002500042DB0D94EE370D946E4A0D94464A0D9490
:10026000D1460C9491DB0C948CE00C9499DB0D94AA
:10027000784A0C948A9D0D946B370D94783B0D94BD
:10028000CD450C94B39D0C94A55C0D94E4370D946E
:100290008F370D942E4F0D9413370C94F9DE0D9477
:1002A000DC360D947F370D94AE460D94D8420C94F5
:1002B000C79D0D94D6590C9467DB0D941E440D9484
:1002C00075370D9461370C9402D60C9443D70D9476
:1002D00046470D94E5460C94CBE00D945C370C94A6
:1002E000B5DC0C9416DF0C94B0D50C9460DB0D9447
:1002F000164A0C94995E0D94873C0C94F3DF0D9490
:1003000051440C9486DB0D9405370D949A460C9459
:1003100073DB0D940D370D94994A0D9409370C94A5
:1003200042840C94CE9D0C94AF9D0D94F4590C9482
:1003300007D60C949EE00D945D3C0C9451DB0C941C
:100340006FDB0D9417370D94ED360C946BDB0D9429
:1003500009480D9487370D947A4B0C946D5E0C947C
:10036000A15C0C94AFDF0D948C4A0C944AD70C948A
:100370007BDB0D94C6360D94E7360D94EF3D0C945F
:10038000999D0D943E400D9454370C94BF9D0D944F
:100390003D4A0C94B79D0D9404470D94F7360D9487
:1003A000E0360D94FF360C94B7D50C94BB9D0C949D
:1003B000D99D0C945B9D0C9432DC4E414E494E49C4
:1003C0005459494E46CDCCCC3D0AD7233C17B7D122
:1003D0003877CC2B329595E6241FB14F0A000020C8
:1003E000410000C84200401C4620BCBE4CCA1B0E47
:1003F0005AAEC59D7400407A10F35A00A0724E1890
:10040000090010A5D4E80000E87648170000E40BC6
:1004100054020000CA9A3B000000E1F5050000808C
:10042000969800000040420F000000A086010000E6
:1004300000102700000000E8030000000064000036
:100440000000000A00000000000100000000002C75
:1004500076D888DC674F0823DFC1DFAE59E1B1B73A
:1004600096E5E3E453C63AE651997696E8E6C28407
:1004700026EB898C9B62ED407C6FFCEFBC9C9F401F
:10048000F2BAA56FA5F490055A2AF75C936B6CF944
:10049000676DC11BFCE0E40D47FEF520E6B500D01A
:1004A000ED902E0300943577050080841E0800002F
:1004B000204E0A000000C80C333333330F986E12FD
:1004C000831141EF8D2114893BE65516CFFEE6DB03
:1004D00018D1844B381BF77C1D901DA4BBE424204D
:1004E0003284725E228100C9F124ECA1E53D2743EC
:1004F0004F4D4D554E49434154494F4E004452597A
:1005000052554E004552524F525300494E464F00ED
:100510004543484F0020496E76616C6964206578D8
:10052000747275646572200047322F473320626110
:100530006420706172616D65746572730A00536C3A
:100540006565702E2E2E005A2050726F6265205005
:10055000617374204265640A005A2050726F6265AC
:1005600020506173742042656400205A3A200020B4
:10057000593A200042656420583A20004D6573685E
:1005800020706F696E74206F7574206F66207261C1
:100590006E67650A004D302053746F70004D312036
:1005A00053746F7000436F6E74696E756500436CB1
:1005B00069636B20746F20526573756D652E2E2EE6
:1005C000004E6F204D6F76652E00456E6420666983
:1005D0006C65206C6973740A00426567696E2066F9
:1005E000696C65206C6973740A004E6F206D6564D8
:1005F00069610A00526573756D696E672053440026
:10060000286E6F2066696C65290043757272656E8D
:10061000742066696C653A20005072696E742074AB
:10062000696D653A20000A53746174733A20466913
:100630006C616D656E7420757365643A20002C20C2
:100640004C6F6E67657374206A6F623A2000546F56
:1006500074616C2074696D653A2000537461747321
:100660003A20002C204661696C65643A20002C20F9
:1006700046696E69736865643A20005072696E74E9
:10068000733A200053746174733A2000436F6F6CA7
:10069000696E672E2E2E0048656174696E672E2E76
:1006A0002E0045202553006F6B006F666600100515
:1006B0000B050405FD04EF0444454255473A004D3F
:1006C00031313320530042656420436F6F6C696E93
:1006D000672E2E2E004265642048656174696E673E
:1006E0002E2E2E00544D334420453520506C75730A
:1006F000204F46462E002F2F002052004163636595
:100700006C65726174696F6E3A2050004D323036FC
:1007100020580046523A0020466C6F773A20003A43
:10072000200020536572766F2000206F7574206F53
:10073000662072616E67650A00536572766F2000ED
:1007400020643A0020693A0020703A00496E7661D0
:100750006C69642065787472756465720A0020643F
:100760003A0020693A0020703A0064697300656EAF
:100770000043290A0061626C656420286D696E205F
:1007800074656D702000436F6C64206578747275B9
:10079000646573206172652000504944204175747E
:1007A0006F74756E6500504944204175746F74759F
:1007B0006E65206661696C65642120426164206811
:1007C00065617465722069640A0046696C616D65D3
:1007D0006E742072756E6F75742064697374616EC7
:1007E000636520286D6D293A200046696C616D654E
:1007F0006E742072756E6F757420004F6666736537
:100800007473204170706C696564004572723A209F
:10081000546F6F206661722100546F6F20666172A1
:100820002066726F6D207265666572656E63652005
:10083000706F696E740A00454550524F4D204F4B02
:100840000A002E0A002028302D3130290020766140
:100850006C7565206F7574206F662072616E6765B8
:1008600000416476616E6365204B3D00506F776593
:10087000722D6C6F7373207265636F766572792069
:10088000004D383400446F6E65207072696E746973
:100890006E672066696C650A004D3737004D33314D
:1008A000004361703A004D4541545041434B004371
:1008B0004F4F4C45525F54454D504552415455524F
:1008C00045004348414D4245525F54454D504552C5
:1008D00041545552450042414259535445505049A4
:1008E0004E470041524353004D4F54494F4E5F4DC8
:1008F0004F44455300544845524D414C5F50524F70
:1009000054454354494F4E004C4F4E475F46494C67
:10091000454E414D45004155544F5245504F52545C
:100920005F53445F5354415455530053445F5752EF
:1009300049544500524550454154005344434152A7
:10094000440050524F4D50545F535550504F5254E5
:1009500000454D455247454E43595F50415253451E
:100960005200434153455F4C494748545F42524906
:100970004748544E45535300544F47474C455F4CEE
:10098000494748545300534F4654574152455F50CE
:100990004F574552004255494C445F5045524345DC
:1009A0004E54004C4556454C494E475F44415441D6
:1009B000005A5F50524F42450052554E4F55540019
:1009C0004155544F4C4556454C005052494E545F8A
:1009D0004A4F420050524F475245535300415554DD
:1009E0004F5245504F52545F54454D5000564F4C56
:1009F000554D455452494300454550524F4D0042D4
:100A0000494E4152595F46494C455F5452414E53FD
:100A10004645520053455249414C5F584F4E5F582E
:100A20004F4646004649524D574152455F4E414D53
:100A3000453A4D61726C696E20322E302E375F441C
:100A400057372E3320544D334420453550534D44B1
:100A50004255202841707220323420323032312009
:100A600031393A34373A32302920534F55524345C1
:100A70005F434F44455F55524C3A68747470733A03
:100A80002F2F6769746875622E636F6D2F496E73BF
:100A9000616E6974794175746F6D6174696F6E2FE1
:100AA0004D61726C696E2F747265652F437265615A
:100AB0006C6974794477696E5F322E302050524FE2
:100AC000544F434F4C5F56455253494F4E3A312E87
:100AD00030204D414348494E455F545950453A54A2
:100AE0004D334420453520506C7573204558545281
:100AF000554445525F434F554E543A312055554960
:100B0000443A63656465326132662D343161322D59
:100B1000343734382D396231322D6335356336320E
:100B20006633363766660A0050726F6265204F661C
:100B300066736574205A0050726F6265204F666656
:100B4000736574205A00290A0020746F20003F5AF0
:100B5000206F7574206F662072616E6765202800B3
:100B6000290A0020746F20003F59206F7574206F90
:100B7000662072616E676520282D00290A002074A6
:100B80006F20003F58206F7574206F662072616E71
:100B9000676520282D0050726F6265204F6666736E
:100BA000657420580043616E6E6F74206F70656EBF
:100BB0002073756264697220002569730025696D70
:100BC00020256973002569682025696D20256973D2
:100BD00000256964202569682025696D20256973D1
:100BE0000025697920256964202569682025696DBB
:100BF00020256973003D3D4477696E20496E697414
:100C000020436F6D706C6574653D3D002A2A2A4E45
:100C10006F7A7A6C6554656D705374617475735B2B
:100C2000325D203D003D3D48656174696E6720443A
:100C30006F6E65204368616E67652046696C616D03
:100C4000656E743D3D002020737461727470726F24
:100C5000677265737320003D3D77616974776179D0
:100C600020353D3D003D3D776169747761792034E1
:100C70003D3D003D3D7761697477617920333D3DAD
:100C8000003D3D7761697477617920313D3D003DDC
:100C90003D6F6E5072696E7454696D657253746FF6
:100CA000707065643D3D003D3D6F6E466163746FDD
:100CB000727952657365743D3D00270A0A0000276A
:100CC0002027002027002D006E6F7469666963611C
:100CD00074696F6E200063616E63656C00507269A9
:100CE0006E742041626F72746564004469736D694B
:100CF00073730055492041626F72746564007265B8
:100D000073756D65004D3234002A2A2A43506C6198
:100D10007920546F6E652A2A2A003D3D6F6E50720D
:100D2000696E7454696D65725061757365643D3D9B
:100D300000486F6D696E67204661696C6564006F7D
:100D400070656E00545249474745524544003A2069
:100D50000066696C616D656E74007A5F6D696E0026
:100D6000795F6D617800785F6D6178005265706FB2
:100D70007274696E6720656E6473746F702073742B
:100D8000617475730A0020746F6F206C6F6E67203A
:100D9000657874727573696F6E2070726576656EB2
:100DA0007465640A0020636F6C64206578747275E2
:100DB00073696F6E2070726576656E7465640A0083
:100DC000486F6D65202573257325732046697273FE
:100DD00074005761726E696E673A20486F6D696E74
:100DE000672042756D702044697669736F72203C8C
:100DF00020310A000202040000B4430000B44300A2
:100E00000000000000B4430000B4430000C84300E9
:100E100000004100000041000000400101FF00000F
:100E20000001000000010000800055555500000041
:100E3000400033333300AAAA2A004992240000005C
:100E40002000C7711C0099991900D145170055550C
:100E500015003BB1130024491200111111000000CC
:100E600010000F0F0F00E3380E0043790D00CCCCBB
:100E70000C00C3300C00E8A20B0064210B00AAAAEE
:100E80000A00703D0A009DD80900427B09009224A7
:100E90000900DCD308008888080010420800000020
:100EA0000800F0C107008787070075500700711C14
:100EB00007003EEB0600A1BC0600699006006666CE
:100EC0000600703E06006118060017F4050074D194
:100ED00005005BB00500B290050062720500555533
:100EE000050078390500B81E0500050505004EEC23
:100EF000040087D40400A1BD040090A70400499217
:100F00000400C17D0400EE690400C7560400444497
:100F100004005C32040008210400411004000000B9
:100F200004003FF00300F8E0030026D20300C3C32F
:100F30000300CCB503003AA803000A9B0300388ED7
:100F40000300C08103009F750300D0690300505E59
:100F500003001D53030034480300913D0300333365
:100F6000030016290300381F030097150300300CF7
:100F70000300030303000BFA020049F10200BAE880
:100F800002005CE002002DD802002DD0020059C8FA
:100F90000200B0C0020031B90200DAB10200AAAA10
:100FA0000200A0A30200BC9C0200FA9502005C8F24
:100FB0000200DF88020082820200457C0200277660
:100FC000020027700200436A02007C640200D05EC7
:100FD00002003F590200C8530200FFFDFCFAF8F678
:100FE000F4F2F0EEECEAE9E7E5E3E1E0DEDCDAD9A1
:100FF000D7D5D4D2D0CFCDCBCAC8C7C5C3C2C0BF46
:10100000BDBCBAB9B7B6B4B3B2B0AFADACAAA9A8BB
:10101000A6A5A4A2A1A09E9D9C9A99989795949309
:1010200092908F8E8D8B8A89888786848382818037
:101030007F7E7D7B7A797877767574737271706F45
:101040006E6D6C6B6A696867666564636261605F38
:101050005E5D5C5B5A59585857565554535251501F
:10106000504F4E4D4C4B4A4A4948474646454443EB
:10107000424241403F3E3E3D3C3B3B3A39383837A7
:10108000363535343332323130302F2E2E2D2C2B55
:101090002B2A2929282727262525242323222121F5
:1010A00020201F1E1E1D1C1C1B1B1A191918181787
:1010B0001616151514131312121111100F0F0E0E10
:1010C0000D0D0C0C0B0A0A0909080807070606058E
:1010D000050404030302020100003D3D6F6E5072DF
:1010E000696E7454696D6572537461727465643DA0
:1010F0003D000000B4430000B4430000C8430000BA
:10110000000000000000000000003D3D6F6E5374C1
:101110006F726553657474696E67733D3D003D3D44
:101120006F6E436F6E66696775726174696F6E5337
:10113000746F72655772697474656E3D3D005365D6
:101140007474696E67732053746F72656400363708
:1011500026033C3D380E2E303E121A1C180AFF435F
:1011600009070844000124F404D9201BC40C5C0EB8
:101170009804C4095F0265077101F405F900FB04D6
:10118000B30048048700C1036900580355000303F6
:101190004500BE023A008402310053022A002902AF
:1011A000250004022000E4011C00C8011900AF0161
:1011B00017009801140084011300710110006101EF
:1011C000100051010E0043010D0036010B002B01F0
:1011D0000B0020010B00150109000C01090003019F
:1011E0000800FB000800F3000800EB000700E40023
:1011F0000600DE000600D8000600D2000600CC0083
:101200000500C7000500C2000500BD000400B900CC
:101210000400B5000400B1000400AD000400A90002
:101220000400A5000300A20003009F0004009B002F
:101230000300980003009500020093000300900053
:1012400003008D0002008B0003008800020086006E
:10125000020084000300810002007F0002007D0084
:1012600002007B0002007900020077000100760096
:1012700002007400020072000100710002006F00A1
:1012800002006D0001006C0002006A0001006900AC
:1012900002006700010066000100650001006400B3
:1012A00002006200010061000100600001005F00B7
:1012B00002005D0001005C0001005B0001005A00BB
:1012C00001005900010058000100570001005600BC
:1012D00001005500010054000100530000005300BC
:1012E00001005200010051000100500001004F00B8
:1012F00001004E0000004E0001004D0001004C00B6
:1013000001004B0000004B0001004A0001004900B1
:1013100001004800000048000100470001004600AD
:1013200000004600010045000000450001004400A7
:1013300001004300000043000100420000004200A1
:1013400001004100000041000100400001003F0099
:1013500000003F0001003E0000003E0001003D0093
:1013600000003D0001003C0000003C0000003C008B
:1013700001003B0000003B0001003A0000003A0081
:101380000100390000003900010038000000380079
:10139000000038000100370000003700010036006F
:1013A0000000360000003600010035000000350066
:1013B000000035000100340000003400000034005B
:1013C0000100330000003300000033000100320050
:1013D0000000320000003200010031000000310046
:1013E000000031000100300000003000000030003B
:1013F00001002F0000002F0000002F0000002F0030
:1014000001002E0000002E0000002E0001002D0023
:1014100000002D0000002D0000002D0001002C0018
:1014200000002C0000002C0000002C0001002B000C
:1014300000002B0000002B0000002B0001002A0000
:1014400000002A0000002A0000002A0001002900F4
:1014500000002900000029000000290000002900E8
:1014600001002800000028000000280000002800DB
:1014700000002800010027000000270000002700CE
:1014800000002700000027000100260000002600C1
:1014900000002600000026000000260001002500B4
:1014A00000002500000025000000250000002500A8
:1014B000000025000100240000002400000024009A
:1014C000000024000000240001002300000023008D
:1014D0000000230000002300000023000000230080
:1014E0000000230001002200000022000000220072
:1014F0000000220000002200000022000100210064
:101500000000210000002100000021000000210057
:101510000000210000002100010020000000200048
:10152000000020000000200000002000000020003B
:10153000000020000000200001001F0000001F002C
:1015400000001F0000001F0000001F0000001F001F
:1015500000001F0001001E0000001E0000001E0011
:1015600000001E00000024F4D43050C38E20C2A21C
:101570004017828B7011127A910D816CD90AA86183
:10158000E108C7586607615143061E4B5D05C1451A
:10159000A7041A411104093D9803713931034036FB
:1015A000DB0265339102D4305402802E1D02632C7D
:1015B000EE01752AC501B028A001102781018F25F1
:1015C00064012B244B01E0223401AC211F018D204A
:1015D0000D01801FFC00841EED00971DDF00B81C6C
:1015E000D200E61BC600201BBC00641AB200B21970
:1015F000A8000A19A0006A189900D1179100401795
:101600008B00B516840031167E00B31579003A15AB
:101610007300C7146F0058146A00EE136600881335
:10162000630025135E00C7125B006C125700151291
:101630005400C111510070114F0021114B00D61000
:1016400049008D1047004610440002104200C00FB0
:101650004000800F3E00420F3C00060F3B00CB0EC7
:101660003800930E37005C0E3500270E3400F30D62
:101670003200C10D3100900D3000600D2E00320D92
:101680002D00050D2C00D90C2B00AE0C2900850C6B
:1016900029005C0C2700350C27000E0C2600E80BF7
:1016A0002400C40B2400A00B23007D0B23005A0B45
:1016B0002100390B2100180B2000F80A1F00D90A5D
:1016C0001E00BB0A1E009D0A1D00800A1D00630A41
:1016D0001C00470A1B002C0A1B00110A1A00F709FC
:1016E0001A00DD091900C4091900AB091900920993
:1016F00017007B091800630917004C09160036090A
:101700001600200916000A091500F5081500E00862
:101710001400CC081400B8081400A40814009008A1
:1017200013007D0812006B081300580812004608C9
:1017300012003408110023081100120811000108DA
:101740001100F0071000E0071000D0071000C007DC
:101750001000B0070F00A107100091070E008307CB
:101760000F0074070F0065070E0057070E004907AA
:101770000E003B070D002E070E0020070D0013077B
:101780000D0006070D00F9060C00ED060D00E00641
:101790000C00D4060C00C8060C00BC060C00B006F9
:1017A0000C00A4060B0099060C008D060B008206A7
:1017B0000B0077060B006C060B0061060A0057064B
:1017C0000B004C060A0042060A0038060A002E06E4
:1017D0000A0024060A001A060A0010060900070675
:1017E0000A00FD050900F4050900EB050900E20502
:1017F0000900D9050900D0050900C7050900BE0583
:101800000900B5050800AD050800A50509009C05FF
:101810000800940508008C050800840508007C0574
:101820000800740508006C050700650508005D05E3
:101830000700560508004E0507004705070040054C
:10184000080038050700310507002A0507002305B1
:1018500007001C050600160507000F050700080510
:10186000060002050700FB040600F5040700EE046D
:101870000600E8040600E2040700DB040600D504C5
:101880000600CF040600C9040600C3040600BD0418
:101890000600B7040600B1040500AC040600A60467
:1018A0000600A00405009B040600950405009004B2
:1018B00006008A04050085040500800406007A04F9
:1018C000050075040500700405006B04050066043E
:1018D0000500610405005C0405005704050052047E
:1018E00005004D04050048040500430405003E04BE
:1018F00004003A04050035040500300404002C04FB
:10190000050027040400230405001E0404001A0433
:10191000040016040500110404000D040400090469
:1019200005000404040000040400FC030400F803A0
:101930000400F4030400F0030400EC030400E803D3
:101940000400E4030400E0030400DC030400D80303
:101950000400D4030400D0030400CC030400C80333
:101960000300C5030300726F746174696F6E206DAC
:1019700061747269783A0A0024F404D9201BC40CFB
:101980005C0E9804C4095F0265077101F405F90053
:10199000FB04B30048048700C103690058035500E5
:1019A00003034500BE023A008402310053022A00BC
:1019B0002902250004022000E4011C00C8011900CE
:1019C000AF01170098011400840113007101100089
:1019D0006101100051010E0043010D0036010B00A2
:1019E0002B010B0020010B00150109000C0109005F
:1019F00003010800FB000800F3000800EB000700EB
:101A0000E4000600DE000600D8000600D200060052
:101A1000CC000500C7000500C2000500BD000400A1
:101A2000B9000400B5000400B1000400AD000400DA
:101A3000A9000400A5000300A20003009F00040009
:101A40009B00030098000300950002009300030030
:101A5000900003008D0002008B000300880002004C
:101A60008600020084000300810002007F00020063
:101A70007D0002007B000200790002007700010077
:101A80007600020074000200720001007100020082
:101A90006F0002006D0001006C0002006A0001008E
:101AA0006900020067000100660001006500010096
:101AB000640002006200010061000100600001009A
:101AC0005F0002005D0001005C0001005B0001009E
:101AD0005A000100590001005800010057000100A0
:101AE00056000100550001005400010053000000A1
:101AF000530001005200010051000100500001009C
:101B00004F0001004E0000004E0001004D0001009A
:101B10004C0001004B0000004B0001004A00010096
:101B20004900010048000000480001004700010092
:101B3000460000004600010045000000450001008D
:101B40004400010043000000430001004200000087
:101B5000420001004100000041000100400001007E
:101B60003F0000003F0001003E0000003E00010079
:101B70003D0000003D0001003C0000003C00000072
:101B80003C0001003B0000003B0001003A00000067
:101B90003A0001003900000039000100380000005F
:101BA0003800000038000100370000003700010055
:101BB000360000003600000036000100350000004D
:101BC0003500000035000100340000003400000042
:101BD0003400010033000000330000003300010036
:101BE000320000003200000032000100310000002D
:101BF0003100000031000100300000003000000022
:101C0000300001002F0000002F0000002F00000016
:101C10002F0001002E0000002E0000002E00010009
:101C20002D0000002D0000002D0000002D000100FF
:101C30002C0000002C0000002C0000002C000100F3
:101C40002B0000002B0000002B0000002B000100E7
:101C50002A0000002A0000002A0000002A000100DB
:101C600029000000290000002900000029000000D0
:101C700029000100280000002800000028000000C2
:101C800028000000280001002700000027000000B5
:101C900027000000270000002700010026000000A8
:101CA000260000002600000026000000260001009B
:101CB0002500000025000000250000002500000090
:101CC0002500000025000100240000002400000081
:101CD0002400000024000000240001002300000074
:101CE0002300000023000000230000002300000068
:101CF0002300000023000100220000002200000059
:101D0000220000002200000022000000220001004A
:101D1000210000002100000021000000210000003F
:101D2000210000002100000021000100200000002F
:101D30002000000020000000200000002000000023
:101D40002000000020000000200001001F00000013
:101D50001F0000001F0000001F0000001F00000007
:101D60001F0000001F0001001E0000001E000000F8
:101D70001E0000001E00000024F4D43050C38E204A
:101D8000C2A24017828B7011127A910D816CD90A10
:101D9000A861E108C7586607615143061E4B5D05FF
:101DA000C145A7041A411104093D98037139310353
:101DB0004036DB0265339102D4305402802E1D027E
:101DC000632CEE01752AC501B028A00110278101FE
:101DD0008F2564012B244B01E0223401AC211F012B
:101DE0008D200D01801FFC00841EED00971DDF007B
:101DF000B81CD200E61BC600201BBC00641AB2004F
:101E0000B219A8000A19A0006A189900D117910008
:101E100040178B00B516840031167E00B31579008B
:101E20003A157300C7146F0058146A00EE13660069
:101E30008813630025135E00C7125B006C12570005
:101E400015125400C111510070114F0021114B00A7
:101E5000D61049008D104700461044000210420081
:101E6000C00F4000800F3E00420F3C00060F3B00B9
:101E7000CB0E3800930E37005C0E3500270E340071
:101E8000F30D3200C10D3100900D3000600D2E00B9
:101E9000320D2D00050D2C00D90C2B00AE0C2900A5
:101EA000850C29005C0C2700350C27000E0C260041
:101EB000E80B2400C40B2400A00B23007D0B23009F
:101EC0005A0B2100390B2100180B2000F80A1F00C3
:101ED000D90A1E00BB0A1E009D0A1D00800A1D00B3
:101EE000630A1C00470A1B002C0A1B00110A1A0077
:101EF000F7091A00DD091900C4091900AB09190016
:101F0000920917007B091800630917004C09160095
:101F100036091600200916000A091500F5081500F3
:101F2000E0081400CC081400B8081400A408140039
:101F3000900813007D0812006B0813005808120067
:101F4000460812003408110023081100120811007D
:101F500001081100F0071000E0071000D007100082
:101F6000C0071000B0070F00A107100091070E0076
:101F700083070F0074070F0065070E0057070E0058
:101F800049070E003B070D002E070E0020070D002D
:101F900013070D0006070D00F9060C00ED060D00F5
:101FA000E0060C00D4060C00C8060C00BC060C00B1
:101FB000B0060C00A4060B0099060C008D060B0061
:101FC00082060B0077060B006C060B0061060A0008
:101FD00057060B004C060A0042060A0038060A00A3
:101FE0002E060A0024060A001A060A001006090036
:101FF00007060A00FD050900F4050900EB050900C4
:10200000E2050900D9050900D0050900C705090046
:10201000BE050900B5050800AD050800A5050900C5
:102020009C050800940508008C050800840508003C
:102030007C050800740508006C05070065050800AC
:102040005D050700560508004E0507004705070017
:102050004005080038050700310507002A0507007C
:10206000230507001C050600160507000F050700DD
:102070000805060002050700FB040600F50407003A
:10208000EE040600E8040600E2040700DB04060094
:10209000D5040600CF040600C9040600C3040600E8
:1020A000BD040600B7040600B1040500AC04060038
:1020B000A6040600A00405009B0406009504050084
:1020C000900406008A0405008504050080040600CB
:1020D0007A04050075040500700405006B04050012
:1020E00066040500610405005C0405005704050052
:1020F000520405004D040500480405004304050092
:102100003E0404003A0405003504050030040400D0
:102110002C04050027040400230405001E04040009
:102120001A04040016040500110404000D04040040
:10213000090405000404040000040400FC03040076
:10214000F8030400F4030400F0030400EC030400AB
:10215000E8030400E4030400E0030400DC030400DB
:10216000D8030400D4030400D0030400CC0304000B
:10217000C8030300C503030024F404D9201BC40CC6
:102180005C0E9804C4095F0265077101F405F9004B
:10219000FB04B30048048700C103690058035500DD
:1021A00003034500BE023A008402310053022A00B4
:1021B0002902250004022000E4011C00C8011900C6
:1021C000AF01170098011400840113007101100081
:1021D0006101100051010E0043010D0036010B009A
:1021E0002B010B0020010B00150109000C01090057
:1021F00003010800FB000800F3000800EB000700E3
:10220000E4000600DE000600D8000600D20006004A
:10221000CC000500C7000500C2000500BD00040099
:10222000B9000400B5000400B1000400AD000400D2
:10223000A9000400A5000300A20003009F00040001
:102240009B00030098000300950002009300030028
:10225000900003008D0002008B0003008800020044
:102260008600020084000300810002007F0002005B
:102270007D0002007B00020079000200770001006F
:10228000760002007400020072000100710002007A
:102290006F0002006D0001006C0002006A00010086
:1022A000690002006700010066000100650001008E
:1022B0006400020062000100610001006000010092
:1022C0005F0002005D0001005C0001005B00010096
:1022D0005A00010059000100580001005700010098
:1022E0005600010055000100540001005300000099
:1022F0005300010052000100510001005000010094
:102300004F0001004E0000004E0001004D00010092
:102310004C0001004B0000004B0001004A0001008E
:10232000490001004800000048000100470001008A
:102330004600000046000100450000004500010085
:10234000440001004300000043000100420000007F
:102350004200010041000000410001004000010076
:102360003F0000003F0001003E0000003E00010071
:102370003D0000003D0001003C0000003C0000006A
:102380003C0001003B0000003B0001003A0000005F
:102390003A00010039000000390001003800000057
:1023A000380000003800010037000000370001004D
:1023B0003600000036000000360001003500000045
:1023C000350000003500010034000000340000003A
:1023D000340001003300000033000000330001002E
:1023E0003200000032000000320001003100000025
:1023F000310000003100010030000000300000001A
:10240000300001002F0000002F0000002F0000000E
:102410002F0001002E0000002E0000002E00010001
:102420002D0000002D0000002D0000002D000100F7
:102430002C0000002C0000002C0000002C000100EB
:102440002B0000002B0000002B0000002B000100DF
:102450002A0000002A0000002A0000002A000100D3
:1024600029000000290000002900000029000000C8
:1024700029000100280000002800000028000000BA
:1024800028000000280001002700000027000000AD
:1024900027000000270000002700010026000000A0
:1024A0002600000026000000260000002600010093
:1024B0002500000025000000250000002500000088
:1024C0002500000025000100240000002400000079
:1024D000240000002400000024000100230000006C
:1024E0002300000023000000230000002300000060
:1024F0002300000023000100220000002200000051
:102500002200000022000000220000002200010042
:102510002100000021000000210000002100000037
:102520002100000021000000210001002000000027
:10253000200000002000000020000000200000001B
:102540002000000020000000200001001F0000000B
:102550001F0000001F0000001F0000001F000000FF
:102560001F0000001F0001001E0000001E000000F0
:102570001E0000001E00000024F4D43050C38E2042
:10258000C2A24017828B7011127A910D816CD90A08
:10259000A861E108C7586607615143061E4B5D05F7
:1025A000C145A7041A411104093D9803713931034B
:1025B0004036DB0265339102D4305402802E1D0276
:1025C000632CEE01752AC501B028A00110278101F6
:1025D0008F2564012B244B01E0223401AC211F0123
:1025E0008D200D01801FFC00841EED00971DDF0073
:1025F000B81CD200E61BC600201BBC00641AB20047
:10260000B219A8000A19A0006A189900D117910000
:1026100040178B00B516840031167E00B315790083
:102620003A157300C7146F0058146A00EE13660061
:102630008813630025135E00C7125B006C125700FD
:1026400015125400C111510070114F0021114B009F
:10265000D61049008D104700461044000210420079
:10266000C00F4000800F3E00420F3C00060F3B00B1
:10267000CB0E3800930E37005C0E3500270E340069
:10268000F30D3200C10D3100900D3000600D2E00B1
:10269000320D2D00050D2C00D90C2B00AE0C29009D
:1026A000850C29005C0C2700350C27000E0C260039
:1026B000E80B2400C40B2400A00B23007D0B230097
:1026C0005A0B2100390B2100180B2000F80A1F00BB
:1026D000D90A1E00BB0A1E009D0A1D00800A1D00AB
:1026E000630A1C00470A1B002C0A1B00110A1A006F
:1026F000F7091A00DD091900C4091900AB0919000E
:10270000920917007B091800630917004C0916008D
:1027100036091600200916000A091500F5081500EB
:10272000E0081400CC081400B8081400A408140031
:10273000900813007D0812006B081300580812005F
:102740004608120034081100230811001208110075
:1027500001081100F0071000E0071000D00710007A
:10276000C0071000B0070F00A107100091070E006E
:1027700083070F0074070F0065070E0057070E0050
:1027800049070E003B070D002E070E0020070D0025
:1027900013070D0006070D00F9060C00ED060D00ED
:1027A000E0060C00D4060C00C8060C00BC060C00A9
:1027B000B0060C00A4060B0099060C008D060B0059
:1027C00082060B0077060B006C060B0061060A0000
:1027D00057060B004C060A0042060A0038060A009B
:1027E0002E060A0024060A001A060A00100609002E
:1027F00007060A00FD050900F4050900EB050900BC
:10280000E2050900D9050900D0050900C70509003E
:10281000BE050900B5050800AD050800A5050900BD
:102820009C050800940508008C0508008405080034
:102830007C050800740508006C05070065050800A4
:102840005D050700560508004E050700470507000F
:102850004005080038050700310507002A05070074
:10286000230507001C050600160507000F050700D5
:102870000805060002050700FB040600F504070032
:10288000EE040600E8040600E2040700DB0406008C
:10289000D5040600CF040600C9040600C3040600E0
:1028A000BD040600B7040600B1040500AC04060030
:1028B000A6040600A00405009B040600950405007C
:1028C000900406008A0405008504050080040600C3
:1028D0007A04050075040500700405006B0405000A
:1028E00066040500610405005C040500570405004A
:1028F000520405004D04050048040500430405008A
:102900003E0404003A0405003504050030040400C8
:102910002C04050027040400230405001E04040001
:102920001A04040016040500110404000D04040038
:10293000090405000404040000040400FC0304006E
:10294000F8030400F4030400F0030400EC030400A3
:10295000E8030400E4030400E0030400DC030400D3
:10296000D8030400D4030400D0030400CC03040003
:10297000C8030300C503030070012C019001270167
:10298000B0012201C0011D01F00118011002130164
:1029900030020E016002090190020401C002FF0032
:1029A0000003FA004003F5008003F000D003EB00C1
:1029B0002004E6007004E100E004DC004005D700DC
:1029C000C005D2004006CD00D006C8008007C30075
:1029D0003008BE00F008B900C009B400B00AAF006A
:1029E000B00BAA00D00CA500000EA000500F9B0059
:1029F000C01096005012910000148C00C015870082
:102A0000B0178200B0197D00D01B7800001E730043
:102A100040206E0090226900F024640040275F008F
:102A200090295A00E02B5500102E500020304B000A
:102A300010324600E033410090353C00103737003B
:102A400070383200A0392D00B03A2800A03B230096
:102A5000603C1E00103D1900903D1400103E0F0018
:102A6000703E0A00C03E0500003F0000403FFBFFF3
:102A7000803FF6FFC03FF1FF1000C90210012C019A
:102A80004001220170011801B0010E01F0010401A2
:102A90005002FA00B002F0003003E600D003DC0080
:102AA0009004D2007005C800A006BE000008B40063
:102AB000B009AA00D00BA000600E960060118C0037
:102AC0000015820020197800C01D6E00A02264004D
:102AD000B0275A00902C500000314600E0343C00F2
:102AE00010383200903A2800603C1E00A03D1400CF
:102AF000803E0A00203F00005A5F6D6F76655F637D
:102B00006F6D700A0024F404D9201BC40C5C0E986D
:102B100004C4095F0265077101F405F900FB04B301
:102B20000048048700C103690058035500030345AA
:102B300000BE023A008402310053022A0029022515
:102B40000004022000E4011C00C8011900AF0117B5
:102B5000009801140084011300710110006101103C
:102B60000051010E0043010D0036010B002B010B3B
:102B70000020010B00150109000C010900030108E8
:102B800000FB000800F3000800EB000700E400066B
:102B900000DE000600D8000600D2000600CC0005CA
:102BA00000C7000500C2000500BD000400B9000414
:102BB00000B5000400B1000400AD000400A9000449
:102BC00000A5000300A20003009F0004009B000377
:102BD000009800030095000200930003009000039A
:102BE000008D0002008B00030088000200860002B6
:102BF0000084000300810002007F0002007D0002CB
:102C0000007B0002007900020077000100760002DC
:102C1000007400020072000100710002006F0002E7
:102C2000006D0001006C0002006A000100690002F2
:102C300000670001006600010065000100640002F9
:102C4000006200010061000100600001005F0002FD
:102C5000005D0001005C0001005B0001005A000102
:102C60000059000100580001005700010056000102
:102C70000055000100540001005300000053000102
:102C8000005200010051000100500001004F0001FE
:102C9000004E0000004E0001004D0001004C0001FC
:102CA000004B0000004B0001004A000100490001F8
:102CB00000480000004800010047000100460000F5
:102CC00000460001004500000045000100440001ED
:102CD00000430000004300010042000000420001E8
:102CE000004100000041000100400001003F0000E1
:102CF000003F0001003E0000003E0001003D0000DA
:102D0000003D0001003C0000003C0000003C0001D0
:102D1000003B0000003B0001003A0000003A0001C7
:102D200000390000003900010038000000380000C0
:102D300000380001003700000037000100360000B5
:102D400000360000003600010035000000350000AC
:102D500000350001003400000034000000340001A0
:102D60000033000000330000003300010032000097
:102D7000003200000032000100310000003100008C
:102D80000031000100300000003000000030000180
:102D9000002F0000002F0000002F0000002F000176
:102DA000002E0000002E0000002E0001002D00006B
:102DB000002D0000002D0000002D0001002C00005F
:102DC000002C0000002C0000002C0001002B000053
:102DD000002B0000002B0000002B0001002A000047
:102DE000002A0000002A0000002A0001002900003B
:102DF000002900000029000000290000002900012E
:102E00000028000000280000002800000028000022
:102E10000028000100270000002700000027000014
:102E20000027000000270001002600000026000007
:102E300000260000002600000026000100250000FA
:102E400000250000002500000025000000250000EE
:102E500000250001002400000024000000240000E0
:102E600000240000002400010023000000230000D3
:102E700000230000002300000023000000230000C6
:102E800000230001002200000022000000220000B8
:102E900000220000002200000022000100210000AA
:102EA000002100000021000000210000002100009E
:102EB000002100000021000100200000002000008F
:102EC0000020000000200000002000000020000082
:102ED0000020000000200001001F0000001F000073
:102EE000001F0000001F0000001F0000001F000066
:102EF000001F0001001E0000001E0000001E000058
:102F0000001E00000024F4D43050C38E20C2A24022
:102F100017828B7011127A910D816CD90AA861E128
:102F200008C7586607615143061E4B5D05C145A79A
:102F3000041A411104093D9803713931034036DB0D
:102F40000265339102D4305402802E1D02632CEEB0
:102F500001752AC501B028A001102781018F2564C1
:102F6000012B244B01E0223401AC211F018D200DE7
:102F700001801FFC00841EED00971DDF00B81CD2ED
:102F800000E61BC600201BBC00641AB200B219A8E0
:102F9000000A19A0006A189900D117910040178BF8
:102FA00000B516840031167E00B31579003A15730A
:102FB00000C7146F0058146A00EE1366008813638C
:102FC0000025135E00C7125B006C125700151254E7
:102FD00000C111510070114F0021114B00D6104952
:102FE000008D1047004610440002104200C00F4000
:102FF00000800F3E00420F3C00060F3B00CB0E3816
:1030000000930E37005C0E3500270E3400F30D32AE
:1030100000C10D3100900D3000600D2E00320D2DDD
:1030200000050D2C00D90C2B00AE0C2900850C29B5
:10303000005C0C2700350C27000E0C2600E80B2442
:1030400000C40B2400A00B23007D0B23005A0B218E
:1030500000390B2100180B2000F80A1F00D90A1EA6
:1030600000BB0A1E009D0A1D00800A1D00630A1C89
:1030700000470A1B002C0A1B00110A1A00F7091A44
:1030800000DD091900C4091900AB091900920917DC
:10309000007B091800630917004C09160036091651
:1030A00000200916000A091500F5081500E00814AB
:1030B00000CC081400B8081400A4081400900813E9
:1030C000007D0812006B0813005808120046081211
:1030D0000034081100230811001208110001081122
:1030E00000F0071000E0071000D0071000C0071024
:1030F00000B0070F00A107100091070E0083070F13
:103100000074070F0065070E0057070E0049070EF1
:10311000003B070D002E070E0020070D0013070DC2
:103120000006070D00F9060C00ED060D00E0060C88
:1031300000D4060C00C8060C00BC060C00B0060C3F
:1031400000A4060B0099060C008D060B0082060BEE
:103150000077060B006C060B0061060A0057060B91
:10316000004C060A0042060A0038060A002E060A2B
:103170000024060A001A060A001006090007060ABB
:1031800000FD050900F4050900EB050900E2050949
:1031900000D9050900D0050900C7050900BE0509C9
:1031A00000B5050800AD050800A50509009C050847
:1031B00000940508008C050800840508007C0508BB
:1031C00000740508006C050700650508005D05072B
:1031D00000560508004E0507004705070040050892
:1031E0000038050700310507002A050700230507F9
:1031F000001C050600160507000F05070008050658
:103200000002050700FB040600F5040700EE0406B3
:1032100000E8040600E2040700DB040600D504060B
:1032200000CF040600C9040600C3040600BD04065E
:1032300000B7040600B1040500AC040600A60406AD
:1032400000A00405009B04060095040500900406F8
:10325000008A04050085040500800406007A040540
:103260000075040500700405006B04050066040584
:1032700000610405005C04050057040500520405C4
:10328000004D04050048040500430405003E040405
:10329000003A04050035040500300404002C040540
:1032A0000027040400230405001E0404001A04047B
:1032B0000016040500110404000D040400090405AF
:1032C000000404040000040400FC030400F80304E8
:1032D00000F4030400F0030400EC030400E803041A
:1032E00000E4030400E0030400DC030400D803044A
:1032F00000D4030400D0030400CC030400C803037B
:1033000000C5030300256C642E25696D004D6172B4
:103310006C696E20322E302E375F4457372E3300C3
:10332000417869732000206D696E3A00206D6178E4
:103330003A00416363656C65726174696F6E206CFD
:10334000696D697465642E0A004641535400534CFC
:103350004F570005000006010004000601000605A5
:10336000000000060004004572726F7220777269D7
:1033700074696E6720746F20454550524F4D210A85
:103380000053544F505045442E20005072696E74C3
:1033900065722073746F7070656420647565207445
:1033A0006F206572726F72732E2046697820746880
:1033B00065206572726F7220616E6420757365207E
:1033C0004D39393920746F20726573746172742EAF
:1033D000202854656D70657261747572652069731B
:1033E0002072657365742E205365742069742061A2
:1033F000667465722072657374617274696E672990
:103400000A004E6F20436865636B73756D207769A2
:103410007468206C696E65206E756D6265722C2013
:103420004C617374204C696E653A20004E6F2043E6
:103430006865636B73756D2077697468206C696E5D
:1034400065206E756D6265722C204C617374204C22
:10345000696E653A2000636865636B73756D206DF6
:1034600069736D617463682C204C617374204C69BE
:103470006E653A20004C696E65204E756D6265720E
:10348000206973206E6F74204C617374204C696ED8
:1034900065204E756D6265722B312C204C61737402
:1034A000204C696E653A20004D3131300053657211
:1034B00069616C20737461747573206D69736D61DB
:1034C0007463680A00776169740A00534420726566
:1034D0006164206572726F720A002121204B494C91
:1034E0004C2063617573656420627920746F6F206E
:1034F0006D75636820696E616374697665207469AF
:103500006D65202D2063757272656E7420636F6D1A
:103510006D616E643A2000486F74656E6420496482
:103520006C652054696D656F757400486F74656EC5
:10353000642049646C652054696D656F75740A0078
:103540003D3D6F6E46696C616D656E7452756E6F50
:1035500075743D3D007061757365004D3630300007
:103560002066696C616D656E745F72756E6F7574DF
:10357000200066696C616D656E745F72756E6F7543
:103580007420540046696C616D656E7452756E6F7F
:1035900075742054002A2A2A496E6974696E67205E
:1035A00063617264206973204F4B2A2A2A004D659B
:1035B00064696120496E736572746564004D656469
:1035C00069612052656D6F766564004D3130303031
:1035D0005300627573793A20706175736564206673
:1035E0006F7220696E7075740A00627573793A2083
:1035F00070617573656420666F7220757365720AF9
:1036000000627573793A2070726F63657373696EC7
:10361000670A002A2A2A6B696C6C2A2A2A00706FB2
:103620007765726F6666004B494C4C45442E20000E
:103630005072696E7465722068616C7465642E20C6
:103640006B696C6C28292063616C6C6564210A00CD
:1036500053544F505045442E20005072696E74658B
:10366000722073746F707065642064756520746F68
:10367000206572726F72732E2046697820746865B7
:10368000206572726F7220616E6420757365204DC3
:1036900039393920746F20726573746172742E2009
:1036A0002854656D70657261747572652069732048
:1036B00072657365742E2053657420697420616689
:1036C0007465722072657374617274696E67290A19
:1036D000006563686F3A004572726F723A00204A63
:1036E0000020204D3432312049002020473239203B
:1036F000493939390A006163746976650A00696E6F
:1037000000002053797374656D2076312E3031209E
:10371000002020207C0A004E414E0020202E202038
:103720002000207C004C43443A0A004353563A0A96
:103730000020666F7220003A0A0A000A426564207F
:10374000546F706F677261706879205265706F7224
:10375000740050726F62696E67204661696C6564BF
:103760000A0050726F62696E67204661696C656419
:1037700000205A3A200020593A200042656420581F
:103780003A20004732384C300047323800446F6EE0
:10379000652E0A003F496E76616C69642073746F10
:1037A0007261676520736C6F742E0A3F55736520D4
:1037B0003020746F20003F454550524F4D207374A8
:1037C0006F72616765206E6F7420617661696C61EC
:1037D000626C652E0A00446F6E652E0A003F496ECA
:1037E00076616C69642073746F7261676520736CB5
:1037F0006F742E0A3F557365203020746F20003F90
:10380000454550524F4D2073746F72616765206E4D
:103810006F7420617661696C61626C652E0A003F8D
:103820005034206973206F6E6C7920617661696C09
:1038300061626C65207768656E20616E204C434440
:103840002069732070726573656E742E0A003F5094
:1038500032206973206F6E6C7920617661696C61CA
:10386000626C65207768656E20616E204C43442051
:1038700069732070726573656E742E0A00292E0AB2
:103880000A0050726F62696E672061726F756E64B4
:103890002028004D65736820696E76616C696461EB
:1038A0007465642E2050726F62696E67206D657357
:1038B000682E0A004D657368207A65726F65642E04
:1038C0000A0044656661756C742073746F72616779
:1038D0006520736C6F7420302073656C656374654C
:1038E000642E0A004C6F6164696E6720746573749E
:1038F0005F7061747465726E2076616C7565732E8D
:103900000A0A00496E76616C696420746573745F9D
:103910007061747465726E2076616C75652E2028F6
:103920002D3120746F2032290A0A0020696E7661D9
:103930006C6964617465642E0A0A004C6F6361747B
:10394000696F6E7300456E74697265204D657368AA
:10395000005374616E6461726420446576696174B9
:10396000696F6E3A20004D65616E204D6573682069
:103970004865696768743A200023206F6620736188
:103980006D706C65733A200050726F62696E6720CB
:10399000506F696E740025532025692F2569002E0C
:1039A0000A002F0050726F62696E67206D65736840
:1039B00020706F696E742000496E76616C696420B6
:1039C0006D617020747970652E0A0A003F284629BF
:1039D0006164652068656967687420666F7220425B
:1039E0006564204C6576656C20436F727265637404
:1039F000696F6E206E6F7420706C61757369626C94
:103A0000652E0A0A003F43616E2774206163746962
:103A10007661746520616E642064656163746976A3
:103A2000617465206174207468652073616D652020
:103A300074696D652E0A0A00426F7468205820264A
:103A40002059206C6F636174696F6E73206D75739C
:103A500074206265207370656369666965642E0A07
:103A60000A003F496E76616C696420677269642060
:103A700073697A6520284A292073706563696669CD
:103A800065642028322D39292E0A0A003F28502942
:103A9000686173652076616C756520696E76616C0E
:103AA00069642028302D36292E0A0A003F2856291D
:103AB0006572626F7365206C6576656C20696D70E8
:103AC0006C61757369626C652028302D34292E0A6B
:103AD0000A003F285229657065746974696F6E2009
:103AE000636F756E7420696E76616C69642028312D
:103AF0002B292E0A0A0062335D33583353335D0A93
:103B00000062656420706C616E65206E6F726D611D
:103B10006C203D205B00436F756C64206E6F7420D9
:103B2000636F6D706C657465204C53462100436F64
:103B3000727265637465645F5A3D00255320256980
:103B40002F2569000A0A002F0054696C74696E679A
:103B5000206D65736820706F696E7420003F457238
:103B6000726F722070726F62696E6720706F696E1B
:103B7000742E2041626F7274696E67206F70657277
:103B80006174696F6E2E0A00436F727265637465AB
:103B9000645F5A3D00255320332F330054696C7401
:103BA000696E67206D6573682028332F33290A00FA
:103BB000436F727265637465645F5A3D00255320DC
:103BC000322F330054696C74696E67206D657368B9
:103BD0002028322F33290A00436F7272656374659F
:103BE000645F5A3D0054696C74696E6720506F6958
:103BF0006E7400255320312F330054696C74696E44
:103C000067206D6573682028312F33290A00646F9F
:103C10006E650A00496E73756666696369656E74E0
:103C200020646174610A000000803F3333914233A5
:103C3000331043CCCC574333B38F430080B343009E
:103C400000803F3333914233331043CCCC5743335E
:103C5000B38F430080B3434578747261706F6C61B9
:103C600074696E67206D6573682E2E2E00212120E9
:103C700053544F502063616C6C65642062656361CE
:103C8000757365206F6620424C546F7563682065BC
:103C900072726F72202D2072657374617274207756
:103CA000697468204D3939390A0021212053544F55
:103CB000502063616C6C6564206265636175736537
:103CC000206F6620424C546F756368206572726F76
:103CD00072202D2072657374617274207769746824
:103CE000204D3939390A002F2F616374696F6E3A9C
:103CF0000070726F6D70745F00656E640053656E66
:103D000064204D31303820746F20726573756D6595
:103D10000A00496E736572742066696C616D656E28
:103D20007420616E642073656E64204D3130380AF2
:103D3000005265686561742066696E6973686564C0
:103D40002E0052656865617420446F6E650052658F
:103D500068656174696E672E2E2E00526568656114
:103D600074004865617465722054696D656F75747F
:103D70000053656E64204D31303820746F206865C3
:103D80006174206E6F7A7A6C650A004E6F7A7A6C75
:103D900065205061726B656400486F74656E6420C5
:103DA000746F6F20636F6C640A0070617573656473
:103DB0000050617573650044697361626C6552758A
:103DC0006E6F75740050757267654D6F7265005047
:103DD00061757365640073686F7700627574746FE2
:103DE0006E00626567696E004C6F61642046696CA5
:103DF000616D656E74004C6F61642046696C616D25
:103E0000656E74205400496E736572742066696C27
:103E1000616D656E7420616E642073656E64204D03
:103E20003130380A00726573756D656400526573D0
:103E3000756D696E670057616974696E6720666F9A
:103E400072206865617475702E0A004C6561766930
:103E50006E6720473236003F537065636966696557
:103E60006420582C5920636F6F7264696E617465A9
:103E7000206F7574206F6620626F756E64732E0AF2
:103E8000003F28522965706561742076616C756504
:103E9000206E6F7420706C61757369626C653B2075
:103EA0006D757374206265206174206C6561737434
:103EB00020312E0A003F2852296570656174206DFB
:103EC00075737420626520737065636966696564E3
:103ED000207768656E206E6F74207573696E672039
:103EE000616E204C43442E0A003F5370656369663F
:103EF000696564206E6F7A7A6C652074656D706593
:103F0000726174757265206E6F7420706C61757368
:103F100069626C652E0A003F537065636966696566
:103F2000642066696C616D656E742073697A6520C2
:103F30006E6F7420706C61757369626C652E0A0017
:103F40003F537065636966696564207072696D6569
:103F5000206C656E677468206E6F7420706C61757C
:103F60007369626C652E0A003F5072696D65206C42
:103F7000656E677468206D75737420626520737058
:103F800065636966696564207768656E206E6F7425
:103F9000207573696E6720616E204C43442E0A00C1
:103FA0003F537065636966696564206E6F7A7A6CE9
:103FB000652073697A65206E6F7420706C6175730B
:103FC00069626C652E0A003F5265747261637469A0
:103FD0006F6E204D756C7469706C696572206D75BB
:103FE0007374206265207370656369666965642E09
:103FF0000A003F53706563696669656420526574A1
:1040000072616374696F6E204D756C7469706C6950
:104010006572206E6F7420706C61757369626C6577
:104020002E0A003F537065636966696564206C61A0
:1040300079657220686569676874206E6F74207096
:104040006C61757369626C652E0A0043292E0A0043
:104050003F537065636966696564206265642074B6
:10406000656D7065726174757265206E6F74207015
:104070006C61757369626C65202834302D0047329D
:1040800036207374617274696E672E2E2E0A004F8B
:1040900046460A0046616465204865696768742081
:1040A00000426564204C6576656C696E6720004649
:1040B00061696C656420746F20656E61626C652057
:1040C000426564204C6576656C696E670A00496ECE
:1040D00076616C6964206D6573682E0A0076616C88
:1040E00069640A53746F7261676520736C6F743A08
:1040F0002000696E004D65736820697320003F558C
:104100007365203020746F20003F496E76616C69C2
:10411000642073746F7261676520736C6F742E0A0C
:10412000003F454550524F4D2073746F7261676573
:10413000206E6F7420617661696C61626C652E0A15
:10414000004D65736820706F696E74206F75742000
:104150006F662072616E67650A004D3432312069E6
:104160006E636F727265637420706172616D6574E5
:1041700065722075736167650A00446576696174CC
:10418000696F6E0025533A2025730046696E697386
:10419000686564210A003A207A3A2000206F662080
:1041A00000476F696E6720746F3A20580043570AC2
:1041B00000206469723A0020616E676C653A0053B2
:1041C00074617274207261646975733A004D343899
:1041D00020506F696E740025533A2025642F2564A2
:1041E00000506F736974696F6E696E6720746865DB
:1041F0002070726F62652E2E2E0A003F4C65677329
:10420000206F66206D6F76656D656E7420696D70C8
:104210006C61757369626C652028302D3135292EEB
:104220000A003F2028582C5929206F7574206F668A
:1042300020626F756E64732E0A0050726F62652083
:104240006F7574206F6620626F756E6473003F53E4
:10425000616D706C652073697A65206E6F74207073
:104260006C61757369626C652028342D3530292E98
:104270000A004D3438205A2D50726F626520526505
:10428000706561746162696C6974792054657374D6
:104290000A003F2856296572626F7365206C657647
:1042A000656C20696D706C61757369626C6520283E
:1042B000302D34292E0A005374616E6461726420BB
:1042C000446576696174696F6E3A20002052616EB0
:1042D00067653A2000204D61783A2000204D696ED4
:1042E0003A2000205369676D613A20004D65616E88
:1042F0003A20005741524E494E4721204C6F7720BB
:104300005A204A65726B206D6179206C656164206A
:10431000746F20756E77616E74656420706175735B
:1043200065732E0A004F4646004F4E0020204D6117
:10433000783A2000200020204D696E3A2000536F0B
:10434000667420656E6473746F70733A20003D3D2F
:104350004F6E506F7765724C6F7373526573756DE6
:10436000653D3D004D32342053256C642054256C4E
:1043700064004739322E39204525730047312046E5
:104380002564004739322E39205A257300473120E1
:104390005A3020463230300047312058257320599A
:1043A0002573204633303030004D343230205325D1
:1043B00069205A2573004D3130362050256920532D
:1043C0002569004D32303020442573004732385281
:1043D000305859004739322E39204530205A300A9A
:1043E00047315A2573004D31303920532569004D2E
:1043F00031393020532569004D343230205330207C
:104400005A30000A20696E6974207A70726F626592
:104410005F7A6F6666736574203D20003D3D6F6E68
:10442000436F6E66696775726174696F6E53746FFE
:104430007265526561643D3D00454550524F4D20C7
:10444000496E697469616C697A65640A003F556EEA
:1044500061626C6520746F2073617665206D657391
:104460006820646174612E0A003F556E61626C655C
:1044700020746F206C6F6164206D657368206461C7
:1044800074612E0A00556E69666965642042656430
:10449000204C6576656C696E67003B20003A0A0027
:1044A00020204D363033200020440020204D343170
:1044B0003220530046696C616D656E742072756EB2
:1044C0006F75742073656E736F723A002055004CDF
:1044D0000046696C616D656E74206C6F61642F7548
:1044E0006E6C6F6164206C656E677468733A00204F
:1044F000204D393030204B004C696E65617220418F
:104500006476616E63653A0020204D38353120585D
:10451000005A2D50726F6265204F66667365740095
:1045200020204D343133205300506F7765722D4C6D
:104530006F7373205265636F766572793A00204419
:104540000020490020204D3330342050002044000A
:1045500020490020204D3330312050005049442064
:1045600073657474696E67733A00206D657368656E
:10457000732E0A0A00454550524F4D2063616E204C
:10458000686F6C642000416374697665204D6573C3
:104590006820536C6F743A200020204D3432302054
:1045A000530020204D323036205800486F6D652072
:1045B0006F66667365743A0020580020530020200F
:1045C0004D323035204200416476616E6365643A55
:1045D00020423C6D696E5F7365676D656E745F74D4
:1045E000696D655F75733E20533C6D696E5F6665EE
:1045F0006564726174653E20543C6D696E5F7472CF
:104600006176656C5F66656564726174653E2058AD
:104610003C6D61785F785F6A65726B3E20593C6DD6
:1046200061785F795F6A65726B3E205A3C6D617894
:104630005F7A5F6A65726B3E20453C6D61785F65AD
:104640005F6A65726B3E0020540020520020204DAE
:10465000323034205000416363656C657261746967
:104660006F6E2028756E6974732F7332293A20504B
:104670003C7072696E745F616363656C3E20523C8E
:10468000726574726163745F616363656C3E20542C
:104690003C74726176656C5F616363656C3E00209B
:1046A000204D3230312058004D6178696D756D2094
:1046B000416363656C65726174696F6E2028756E05
:1046C0006974732F7332293A0020204D3230332021
:1046D00058004D6178696D756D206665656472611D
:1046E0007465732028756E6974732F73293A0053AB
:1046F000746570732070657220756E69743A00205D
:10470000440020204D323030205300204469736132
:10471000626C65640A0046696C616D656E74207335
:10472000657474696E67733A0020286D6D290020E6
:1047300020473231202020203B20556E69747320A1
:10474000696E206D6D003F4D65736820746F6F203A
:1047500062696720666F7220454550524F4D2E0AA0
:10476000003D3D6F6E4C6F616453657474696E6794
:10477000733D3D0000803B4400803B4400002041ED
:10478000000096420000A0420000A0420000484401
:104790000000BE42D0070000D00700006400000007
:1047A0004B00000024F4D43050C38E20C2A2401726
:1047B000828B7011127A910D816CD90AA861E1087F
:1047C000C7586607615143061E4B5D05C145A704E6
:1047D0001A411104093D9803713931034036DB0257
:1047E00065339102D4305402802E1D02632CEE01F9
:1047F000752AC501B028A001102781018F25640109
:104800002B244B01E0223401AC211F018D200D012E
:10481000801FFC00841EED00971DDF00B81CD20035
:10482000E61BC600201BBC00641AB200B219A80027
:104830000A19A0006A189900D117910040178B003F
:10484000B516840031167E00B31579003A15730051
:10485000C7146F0058146A00EE13660088136300D3
:1048600025135E00C7125B006C125700151254002E
:10487000C111510070114F0021114B00D610490099
:104880008D1047004610440002104200C00F400047
:10489000800F3E00420F3C00060F3B00CB0E38005D
:1048A000930E37005C0E3500270E3400F30D3200F6
:1048B000C10D3100900D3000600D2E00320D2D0025
:1048C000050D2C00D90C2B00AE0C2900850C2900FD
:1048D0005C0C2700350C27000E0C2600E80B24008A
:1048E000C40B2400A00B23007D0B23005A0B2100D6
:1048F000390B2100180B2000F80A1F00D90A1E00EE
:10490000BB0A1E009D0A1D00800A1D00630A1C00D0
:10491000470A1B002C0A1B00110A1A00F7091A008B
:10492000DD091900C4091900AB0919009209170023
:104930007B091800630917004C0916003609160098
:10494000200916000A091500F5081500E0081400F2
:10495000CC081400B8081400A40814009008130030
:104960007D0812006B081300580812004608120058
:104970003408110023081100120811000108110069
:10498000F0071000E0071000D0071000C00710006B
:10499000B0070F00A107100091070E0083070F005A
:1049A00074070F0065070E0057070E0049070E0039
:1049B0003B070D002E070E0020070D0013070D000A
:1049C00006070D00F9060C00ED060D00E0060C00D0
:1049D000D4060C00C8060C00BC060C00B0060C0087
:1049E000A4060B0099060C008D060B0082060B0036
:1049F00077060B006C060B0061060A0057060B00D9
:104A00004C060A0042060A0038060A002E060A0072
:104A100024060A001A060A001006090007060A0002
:104A2000FD050900F4050900EB050900E205090090
:104A3000D9050900D0050900C7050900BE05090010
:104A4000B5050800AD050800A50509009C0508008E
:104A5000940508008C050800840508007C05080002
:104A6000740508006C050700650508005D05070072
:104A7000560508004E0507004705070040050800D9
:104A800038050700310507002A0507002305070040
:104A90001C050600160507000F050700080506009F
:104AA00002050700FB040600F5040700EE040600FB
:104AB000E8040600E2040700DB040600D504060053
:104AC000CF040600C9040600C3040600BD040600A6
:104AD000B7040600B1040500AC040600A6040600F5
:104AE000A00405009B040600950405009004060040
:104AF0008A04050085040500800406007A04050088
:104B000075040500700405006B04050066040500CB
:104B1000610405005C04050057040500520405000B
:104B20004D04050048040500430405003E0404004C
:104B30003A04050035040500300404002C04050087
:104B400027040400230405001E0404001A040400C2
:104B500016040500110404000D04040009040500F6
:104B60000404040000040400FC030400F80304002F
:104B7000F4030400F0030400EC030400E803040061
:104B8000E4030400E0030400DC030400D803040091
:104B9000D4030400D0030400CC030400C8030300C2
:104BA000C503030024F404D9201BC40C5C0E980434
:104BB000C4095F0265077101F405F900FB04B30045
:104BC00048048700C10369005803550003034500EA
:104BD000BE023A008402310053022A002902250055
:104BE00004022000E4011C00C8011900AF011700F5
:104BF000980114008401130071011000610110007C
:104C000051010E0043010D0036010B002B010B007A
:104C100020010B00150109000C0109000301080027
:104C2000FB000800F3000800EB000700E4000600AA
:104C3000DE000600D8000600D2000600CC00050009
:104C4000C7000500C2000500BD000400B900040053
:104C5000B5000400B1000400AD000400A900040088
:104C6000A5000300A20003009F0004009B000300B6
:104C700098000300950002009300030090000300D9
:104C80008D0002008B0003008800020086000200F5
:104C900084000300810002007F0002007D0002000A
:104CA0007B0002007900020077000100760002001C
:104CB0007400020072000100710002006F00020027
:104CC0006D0001006C0002006A0001006900020032
:104CD0006700010066000100650001006400020039
:104CE0006200010061000100600001005F0002003D
:104CF0005D0001005C0001005B0001005A00010042
:104D00005900010058000100570001005600010041
:104D10005500010054000100530000005300010041
:104D20005200010051000100500001004F0001003D
:104D30004E0000004E0001004D0001004C0001003B
:104D40004B0000004B0001004A0001004900010037
:104D50004800000048000100470001004600000034
:104D6000460001004500000045000100440001002C
:104D70004300000043000100420000004200010027
:104D80004100000041000100400001003F00000020
:104D90003F0001003E0000003E0001003D00000019
:104DA0003D0001003C0000003C0000003C00010010
:104DB0003B0000003B0001003A0000003A00010007
:104DC0003900000039000100380000003800000000
:104DD00038000100370000003700010036000000F5
:104DE00036000000360001003500000035000000EC
:104DF00035000100340000003400000034000100E0
:104E000033000000330000003300010032000000D6
:104E100032000000320001003100000031000000CB
:104E200031000100300000003000000030000100BF
:104E30002F0000002F0000002F0000002F000100B5
:104E40002E0000002E0000002E0001002D000000AA
:104E50002D0000002D0000002D0001002C0000009E
:104E60002C0000002C0000002C0001002B00000092
:104E70002B0000002B0000002B0001002A00000086
:104E80002A0000002A0000002A000100290000007A
:104E9000290000002900000029000000290001006D
:104EA0002800000028000000280000002800000062
:104EB0002800010027000000270000002700000054
:104EC0002700000027000100260000002600000047
:104ED000260000002600000026000100250000003A
:104EE000250000002500000025000000250000002E
:104EF0002500010024000000240000002400000020
:104F00002400000024000100230000002300000012
:104F10002300000023000000230000002300000005
:104F200023000100220000002200000022000000F7
:104F300022000000220000002200010021000000E9
:104F400021000000210000002100000021000000DD
:104F500021000000210001002000000020000000CE
:104F600020000000200000002000000020000000C1
:104F700020000000200001001F0000001F000000B2
:104F80001F0000001F0000001F0000001F000000A5
:104F90001F0001001E0000001E0000001E00000097
:104FA0001E000000232C0000B8220000561800004C
:104FB0003A0F0000B8080000B104000071020000C0
:104FC0003E01000020436F756E7420583A00236440
:104FD0006566696E652044454641554C545F000046
:104FE000626564004B6420004B6920004B70200018
:104FF000504944204175746F74756E652066696E02
:105000006973686564212050757420746865206C2C
:10501000617374204B702C204B6920616E64204BAF
:105020006420636F6E7374616E74732066726F6D4B
:105030002062656C6F7720696E746F20436F6E66B7
:10504000696775726174696F6E2E680A0050494411
:10505000204175746F74756E65206661696C656456
:10506000212074696D656F75740A005049442041B0
:1050700075746F74756E65206661696C6564212056
:1050800054656D706572617475726520746F6F2000
:10509000686967680A00204B643A2000204B693A2F
:1050A0002000204B703A200020436C6173736963C9
:1050B00020504944200A00204E6F206F766572739D
:1050C000686F6F740A002054753A2000204B753ABF
:1050D0002000206D61783A2000206D696E3A200032
:1050E00020643A200020626961733A2000504944EC
:1050F000204175746F74756E652073746172740AE3
:1051000000504944204175746F74756E6520666166
:10511000696C6564212054656D7065726174757287
:105120006520746F6F20686967680A0042656400D3
:10513000453100626564002C2073797374656D20BD
:1051400073746F7070656421204865617465725F67
:1051500049443A200048656174696E672046616978
:105160006C65640048656174696E67206661696C8E
:105170006564004D3131322053687574646F776E09
:10518000001000C90210012C014001220170011819
:1051900001B0010E01F00104015002FA00B002F06A
:1051A000003003E600D003DC009004D2007005C894
:1051B00000A006BE000008B400B009AA00D00BA0F1
:1051C00000600E960060118C000015820020197896
:1051D00000C01D6E00A0226400B0275A00902C5021
:1051E0000000314600E0343C0010383200903A288C
:1051F00000603C1E00A03D1400803E0A00203F00DD
:1052000000544845524D414C2052554E415741594A
:1052100000546865726D616C2052756E61776179BA
:10522000004572723A204D415854454D50004D4151
:105230005854454D50207472696767657265640003
:105240004572723A204D494E54454D50004D494EDD
:1052500054454D502074726967676572656400201B
:105260002F002042403A0020403A0020573A0020C8
:10527000573A00496E76616C69642065787472757E
:105280006465720A007C3C3E5E2B3D3F2F5B5D3BBC
:105290002C2A225C0043616E6E6F74206F70656E05
:1052A000207375626469722000534420496E6974EA
:1052B000204661696C0053442063617264206F6B07
:1052C0000A006F70656E526F6F74206661696C655D
:1052D000640A00766F6C756D652E696E6974206660
:1052E00061696C65640A004E6F20534420636172EB
:1052F000640A000A4D3234004D3233202573002EEB
:105300000A006F70656E206661696C65642C2046CA
:10531000696C653A200046696C652073656C65634D
:105320007465640A002053697A653A200046696C06
:1053300065206F70656E65643A2000454E442053C9
:105340005542524F5554494E450A002220706F7302
:10535000002220706172656E743A220053554252E9
:105360004F5554494E452043414C4C20746172675F
:1053700065743A220053756263616C6C204F7665E8
:1053800072666C6F77004578636565646564206D4F
:10539000617820535542524F5554494E452064651B
:1053A0007074683A002E0A0044656C6574696F6E0B
:1053B000206661696C65642C2046696C653A200042
:1053C00046696C652064656C657465643A00534495
:1053D000207072696E74696E67206279746520004E
:1053E0004E6F74205344207072696E74696E670A40
:1053F0000057726974696E6720746F2066696C6506
:105400003A2000667265736800646F696E670020F9
:1054100066696C653A20004E6F7720002F617574C5
:105420006F25632E67002020506C616E6E6572429E
:10543000756666657242797465733A20002046721B
:105440006565204D656D6F72793A2000436F6D7010
:10545000696C65643A2041707220323420323032F7
:10546000310A00204C617374205570646174656466
:105470003A20323032312D30342D3138207C2041E9
:105480007574686F723A2054696E794D616368690A
:105490006E657333440A00322E302E375F4457371F
:1054A0002E330A004D61726C696E0020536F667472
:1054B000776172652052657365740A0020576174C4
:1054C0006368646F672052657365740A00204272D6
:1054D0006F776E206F75742052657365740A0020B3
:1054E00045787465726E616C2052657365740A004C
:1054F000506F77657255700A0073746172740A0098
:105500004732385859004D31303031006572726F72
:10551000722077726974696E6720746F2066696C97
:10552000650A00446F6E6520736176696E67206658
:10553000696C652E0A004D323900456E6473746FD4
:1055400070730025532025632025632025632025C3
:105550006300205A3A0020593A0020583A00656EFC
:105560006473746F7073206869743A200070012C42
:105570000190012701B0012201C0011D01F00118B5
:10558000011002130130020E0160020901900204B1
:1055900001C002FF000003FA004003F5008003F0A1
:1055A00000D003EB002004E6007004E100E004DC1E
:1055B000004005D700C005D2004006CD00D006C887
:1055C000008007C3003008BE00F008B900C009B46D
:1055D00000B00AAF00B00BAA00D00CA500000EA0CE
:1055E00000500F9B00C01096005012910000148CC8
:1055F00000C0158700B0178200B0197D00D01B785D
:1056000000001E730040206E0090226900F02464A8
:105610000040275F0090295A00E02B5500102E50C3
:105620000020304B0010324600E033410090353C02
:10563000001037370070383200A0392D00B03A28FA
:1056400000A03B2300603C1E00103D1900903D145B
:1056500000103E0F00703E0A00C03E0500003F00F3
:1056600000403FFBFF803FF6FFC03FF1FF00000A14
:105670000B02090C0D0E08070304010000000000D6
:10568000000000000000000000000000000000001A
:1056900000000000000000000012111000000000D7
:1056A00000000000000000000000000000000000FA
:1056B0000000003D3D6F6E55736572436F6E666905
:1056C000726D52657175697265643D3D00220A0014
:1056D000556E6B6E6F776E20636F6D6D616E643AA1
:1056E0002022002042002050006F6B002045002047
:1056F0005A00205900204D393220580020453A00E8
:10570000205A3A0020593A00583A0020746F6F200E
:105710006C6F6E6720657874727573696F6E207038
:10572000726576656E7465640A0020636F6C642030
:10573000657874727573696F6E2070726576656EC8
:105740007465640A0043616E6E6F7420656E7465E3
:1057500072207375626469723A20004D32352050B0
:105760000A4D323400526573756D650055492050FD
:1057700061757365004E6F204D61746368203A0057
:1057800050675570005067446F776E00497320462C
:10579000696C6520004973204469722000476F5589
:1057A0007044697200486173204D65646961004608
:1057B000696C656E616D652053656C6563746564C5
:1057C000004D3130303043004D31303030004669CB
:1057D0006C616D656E7420537461742030202D20CF
:1057E000330046696C616D656E742053746174207A
:1057F00030202D20320046696C616D656E74205337
:105800007461742030202D2031002046696C616D58
:10581000656E7420526573706F6E7365204E6F00F5
:10582000526573756D652059657320647572696E74
:1058300067207072696E74000A204E6F2046696C92
:10584000616D656E7400496E76616C6964204F709D
:1058500074696F6E004D3530300053746F7265207F
:1058600053657474696E67730042656420504944DF
:105870002053746172746564004D3939390A4D32B0
:10588000383050305331363000424C546F756368B5
:10589000205265736574004D3530320A4D35303015
:1058A00000496E697420454550524F4D00486F7451
:1058B000656E6420504944205374617274656400BD
:1058C000456E676C69736820416C7265616479200C
:1058D000536574004368696E657365204E6F74206C
:1058E000537570706F7274656400496E4C616E67B9
:1058F00043686F696365000A202A2A2A7265636417
:1059000061742E646174615B305D203D0047323804
:105910000A4731204631303030205A313000556E40
:10592000737570706F72746564204F7074696F6EF8
:105930002053656C656374656400473236523235B6
:1059400035004D3139305335350A4732380A473240
:105950003950310A47323950330A47323953310A04
:1059600047323953300A47323946302E300A4732EF
:1059700039410A4D313034533231350A4732380A11
:105980004D313039533231350A473158313530597C
:1059900031353046353030300A47315A300A4D35CE
:1059A00030300A4D3430300A4D3131372053657470
:1059B000205A204F666673657400473120463130A7
:1059C0003030205A302E30004732380A47312046D6
:1059D00031303030205A302E30004D353030005AC2
:1059E000204F6666736574203A202573004D35306C
:1059F00030005A204F6666736574203A2025730084
:105A00004732380A473146313530305A302E30006F
:105A10004732385A0A473146313530305A302E3005
:105A2000004D383400473146313030305A302E3056
:105A3000004732380A473146313030305A302E3044
:105A4000004D616E75616C53657454656D70005ADC
:105A5000204F6666736574203A2025730053746F77
:105A600070205472696767657265640053746F7063
:105A7000204E6F0053746F705072696E74004861ED
:105A80006E646C6520446174612041646A7573744E
:105A900020322053657474696E67205363726565A4
:105AA0006E200048616E646C652044617461205012
:105AB00072696E7446696C6520332053657474692D
:105AC0006E672053637265656E200048616E646C7A
:105AD000652044617461205072696E7446696C651A
:105AE00020322053657474696E6720536372656554
:105AF0006E20004D38340048616E646C652044614E
:105B00007461205072696E7446696C6520506F73C1
:105B1000740048616E646C65204461746120507249
:105B2000696E7446696C65205072650042656769EC
:105B30006E537769746368003D3D20436865636B0D
:105B40006B65793D3D007265636461742E616464C8
:105B500072203D3D007265636461742E64617461FE
:105B60005B305D203D3D0077616974776179203D50
:105B70003D0020202A2A2A2A2A2A2A5254535F48E2
:105B8000616E646C65446174612A2A2A2A2A2A2A71
:105B90002A2000526573656E643A200000002200DE
:105BA000250028002B002E003100340002010000E7
:105BB000050108010B0100002100240027002A0034
:105BC0002D003000330001010000040107010A012B
:105BD00005050505070508080808020202020A0A69
:105BE0000808040404040101010101010101030387
:105BF000030303030303040707070C0C0C0C0C0C32
:105C00000C0C0202020206060606060606060B0B2E
:105C10000B0B0B0B0B0B010210202008081020406F
:105C20001020408002010201080402010102040860
:105C300010204080804020100804020180040201EE
:105C40008040201008040201080402010102040837
:105C5000102040800102040810204080544D33443D
:105C600020453520506C75732052656164792E0093
:105C70005072696E74696E672E2E2E005072696EB6
:105C80007420506175736564006E6F746966696332
:105C90006174696F6E20005049442054756E652010
:105CA00046696E69736865640000950159011124A5
:105CB0001FBECFEFD1E2DEBFCDBF00E00CBF19E0C9
:105CC000A0E0B2E0E4ECF8ED02E00BBF02C0079008
:105CD0000D92A031B107D9F72BE1A0E1B9E001C0E5
:105CE0001D92AA3BB207E1F71EE2C6E5DEE200E044
:105CF00006C021970109802FFE010F943C67C5352E
:105D0000D10780E00807A9F70F948A540D94506CCE
:105D10000C9400009F92AF92BF92CF92DF92EF92CD
:105D2000FF920F931F93CF93DF9300D01F921F9288
:105D3000CDB7DEB7EAEDFFE00027BB27462F572F90
:105D4000A82FAA2341F4A52F542FB85FAA2319F432
:105D5000A52F5527B85FA03138F45295A295452F4D
:105D60004F70507FA42BBC5FA03428F4550FAA1F9E
:105D7000550FAA1FBE5FA03818F4550FAA1FB39580
:105D8000550FAA1FEA0FF01F449151E0AA27B850FF
:105D900081F1C8F0B0FF02C0440F551FB1FF04C02D
:105DA000440F551F440F551FB2FF06C05295429530
:105DB000142F1F70407F512BB3FF1BC0A52F542FF2
:105DC00044270C94F92EB195B0FF02C05595479524
:105DD000B1FF04C05595479555954795B2FF05C04D
:105DE0005295407F4295452B5F70B3FF02C0452F0F
:105DF0005527DD24CC24BB24B2E0649FD018C10811
:105E0000B00AB00B749FC018B108B00B849FB018D3
:105E1000B109659FC018B108B00B759FB018B109E2
:105E2000859FB0196A9FB018B1097A9FB0194D9D2E
:105E3000A12C99243327992722275D9DA00C911C22
:105E4000301F901F201FAD9D900C311D901F201FF3
:105E50004C9DA00C911C301F901F201F5C9D900C2E
:105E6000311D901F201FAC9D300D911D201F4B9D9B
:105E7000900C311D901F201F5B9D300D911D201F28
:105E8000AB9D900D211D4B9F300D911D201F5B9FE1
:105E9000900D211DAB9F200DB1E0BB24CC24DD244F
:105EA000639FD018C108B00AB00B739FC018B10827
:105EB000B00B839FB018B109699FC018B108B00B2F
:105EC000799FB018B109899FB019629FB018B109C4
:105ED000729FB019D61AC70AB80A20F0B1E03B0F7A
:105EE000901F201F1124792F632F90E0822F0F9095
:105EF0000F900F900F900F90DF91CF911F910F9106
:105F0000FF90EF90DF90CF90BF90AF909F9008955B
:105F1000AF92BF92CF92DF92EF92FF920F931F93B7
:105F2000CF93DF93C5EBD1E108E01EE085ECA82E0E
:105F300081E1B82EC12CD12C7601C394699179915D
:105F4000899199910F947A60288939894A895B8966
:105F50000F94DB600F94B868F8016193719381939B
:105F600091938F01C616D706E806F90610F46B0167
:105F70007C01AC16BD0611F76FEF7FEFCB01A701D7
:105F800096010F94B9662093180E3093190E409322
:105F90001A0E50931B0EDF91CF911F910F91FF901E
:105FA000EF90DF90CF90BF90AF900895809102184E
:105FB00090910318891B877089F4809108138111CF
:105FC0000DC08091FD119091FE11892B39F481E073
:105FD0009091A80B911103C080E0089581E008958D
:105FE00090E080E00895CF93C82FCB010E94909E4F
:105FF0008EE49DE00E94909E8FE39DE0CC2311F003
:1060000084E49DE00E94909E8AE0CF910C94059ECE
:106010000F931F93CF938C01C62F81EA98E00E94C3
:10602000909EC8010E94909E8AE30E94059E80E394
:106030008C0F0E94059E8AE0CF911F910F910C94C6
:10604000059E84E29AE00E94909E60E084E19AE0DE
:106050000E94083060E08FEF99E00E94083061E014
:1060600088EF99E00E94083061E08DEE99E00E948F
:10607000083061E08DED99E00E94083060E084ED29
:1060800099E00E94083061E08AEC99E00E940830B3
:1060900061E080EC99E00E94083061E089EB99E0D2
:1060A0000E94083061E081EB99E00E94083061E0D5
:1060B00083EA99E00E94083061E085E999E00E9456
:1060C000083060E086E899E00E94083060E088E7E8
:1060D00099E00E94083060E082E699E00E94083072
:1060E00061E081E599E00E94083061E082E499E096
:1060F0000E94083061E08BE399E00E94083060E084
:1061000084E399E00E94083061E08BE299E00E940C
:10611000083061E086E199E00E94083061E088E0A3
:1061200099E00E94083061E085EF98E00E94083015
:1061300060E088EE98E00E94083061E083EE98E02D
:106140000E94083061E086ED98E00E94083060E02F
:1061500082EC98E00E94083060E08FEA98E00E94AC
:10616000083060E08DEB99E10E94F02F682F61709C
:1061700086EA98E00C940830CF93DF938091021860
:1061800090910318891B8095877019F40E9405BCB3
:10619000F5CF809102188F5F8770A091021897E663
:1061A000A99FD0011124FD01ED5CF14FEF0119927F
:1061B0009A95E9F798E09083A85BB14F90E1E4E10C
:1061C000F8E101900D929A95E1F7209102189091D3
:1061D0000318291303C094E69093FF1780930218C5
:1061E000DF91CF910C94339990910218809103180C
:1061F000981308C080916C1190916D11892B11F446
:106200000C94439A80E00E9405BCEECF2F923F92FF
:106210004F925F926F927F928F929F92AF92BF92B6
:10622000CF92DF92EF92FF920F931F93CF93DF9362
:10623000D62FC72FFC0180809180A280B380C5013A
:10624000B40120E831E541E050E00F94B966C9019E
:106250006DE671E00F9428676B017C01C501B40104
:1062600020E13EE040E050E00F94B966CA01B90178
:1062700028E130E040E050E00F94B966362E272E3A
:10628000062F172F8CE3482E512C612C712CC50141
:10629000B401A30192010F94B966B62EA72ECA01CC
:1062A000B901A30192010F94B966CB01C114D104C5
:1062B00079F1AF92BF927F936F932F923F92FF92AB
:1062C000EF92DF92CF9281EE9BE09F938F93CF93DB
:1062D000DF930F940C608DB79EB70E960FB6F894AF
:1062E0009EBF0FBE8DBF8D2F9C2FDF91CF911F9131
:1062F0000F91FF90EF90DF90CF90BF90AF909F9065
:106300008F907F906F905F904F903F902F90089567
:10631000E114F104C9F0AF92BF927F936F932F9273
:106320003F92FF92EF9281ED9BE09F938F93CF93EB
:10633000DF930F940C60EDB7FEB73C960FB6F89460
:10634000FEBF0FBEEDBFCFCF012BB9F0AF92BF9212
:106350007F936F932F923F9285EC9BE09F938F9357
:10636000CF93DF930F940C608DB79EB70A960FB64C
:10637000F8949EBF0FBE8DBFB6CF892BA9F0AF9208
:10638000BF927F936F938DEB9BE09F938F93CF93FF
:10639000DF930F940C60EDB7FEB738960FB6F89404
:1063A000FEBF0FBEEDBF9FCFAF92BF9289EB9BE0C8
:1063B0009F938F93CF93DF930F940C600F900F9068
:1063C0000F900F900F900F908ECFCF93DF9300D050
:1063D0001F92CDB7DEB784EF91E0A0E0B0E08983F3
:1063E0009A83AB83BC83BE016F5F7F4F8CE30E94B7
:1063F000C99B8CE69DE00E94909E8CB166E67DE094
:1064000085FB882780F90E94F32F8091030160E6C5
:106410007DE0869581700E94F32F89B16AE57DE069
:1064200083FB882780F90E94F32F8CB161E57DE022
:10643000829581700E94F32F4B9909C00E94049CA1
:106440000F900F900F900F90DF91CF9108950E94C1
:10645000E99B0F900F900F900F90DF91CF910895CF
:106460008091E80B882319F01092E80B089540E022
:1064700070E060E081E39DE00E9434BBCF93C09167
:106480009709CF7739F50E945C9A882319F180919A
:10649000B2199091B319A091B419B091B5190097A0
:1064A000A105B105B9F0BC01CD016D597F4F8F4FEA
:1064B0009F4F24E630E040E050E00F94B9666091D1
:1064C000B6197091B7198091B8199091B9190F94B4
:1064D000B966C22F8C2FCF9108954F925F926F9221
:1064E0007F928F929F92AF92BF92CF92DF92EF9264
:1064F000FF921F93CF93DF9300D01F92CDB7DEB7EB
:1065000019821A821B821C82CE0101964C018CE7F3
:10651000C82E8CE0D82E9FE5E92E92E0F92E2BEFC5
:10652000A22E2DE0B22E10E088E5810F0E948A8F06
:10653000F40181934F01882309F4E0C00E94128F77
:106540002B013C01812F0E94D48B882309F4CCC0FD
:10655000F7012081318142815381C301B2010F943F
:106560004567F60160837183828393831F5FF4E044
:10657000CF0ED11C84E0E80EF11C94E0A90EB11CF2
:10658000133091F685E40E948A8F8C83882309F466
:10659000C0C00E94128F6B017C0183E00E94D48BEB
:1065A000882371F020916B0230916C0240916D0252
:1065B00050916E02C701B6010F9445676B017C01D3
:1065C000C092880CD092890CE0928A0CF0928B0CCD
:1065D0008091DB0A882359F18091BA1982FF27C084
:1065E0008C81882321F18981811103C08A818823CC
:1065F000F1F02DEC3CEC4CE45DE36091520D7091B8
:10660000530D8091540D9091550D0F9445679B014A
:10661000AC0160916702709168028091690290916B
:106620006A020F94A569181614F40F945D3340E0C4
:1066300050E0BA0186E40E94B18F20E030E0A90169
:106640000F94A569181684F40E94128F20E030E0A0
:1066500040E752E40F943F6860933F02709340021A
:10666000809341029093420280916B1183FD28C078
:106670008091920B882321F120916B0230916C0262
:1066800040916D0250916E026091880C7091890C5E
:1066900080918A0C90918B0C0F94446720919F0BF2
:1066A0003091A00B4091A10B5091A20B0F94456724
:1066B00060939F0B7093A00B8093A10B9093A20B00
:1066C0000F900F900F900F90DF91CF911F91FF903F
:1066D000EF90DF90CF90BF90AF909F908F907F9082
:1066E0006F905F904F900895F50120813181428134
:1066F0005381C301B2010F94446733CFF701808106
:106700009181A281B381F60180839183A283B383B7
:106710002DCF80916B0290916C02A0916D02B0918F
:106720006E028093880C9093890CA0938A0CB0938E
:106730008B0C4ECF84E690E09093D20A8093D10ADE
:106740001092E30A1092E20A0D94C0140F93AB0169
:106750000091E10A21E0022722EE3AE0BC0181ED3E
:106760009AE00E94869A0F910895CF93DF9300D00C
:106770001F92CDB7DEB78091920B8823C1F083E3DF
:1067800090E09C838B831A8219829E012F5F3F4F7A
:1067900040E150E063E97BE0CE0103960E94C4BA79
:1067A0008EE191E10E94909E8AE00E94059E0F90EA
:1067B0000F900F900F90DF91CF910895CF93DF93BB
:1067C00000D01F921F92CDB7DEB781E08093920B6D
:1067D00080E1E3E9FBE0DF011D928A95E9F70E9481
:1067E000B53386E18D8382E390E09C838B831A82AC
:1067F00019829E012F5F3F4F41E050E0BE016B5F69
:106800007F4FCE0103960E94C4BA0F900F900F9055
:106810000F900F90DF91CF910895CF92DF92EF927A
:10682000FF92CF93DF93EC0108960E94CD8D6B0110
:106830007C0120E030E0A9010F94756020E030E099
:10684000A901882371F0BE016C5F7F4FCE010E94C9
:106850005F959B01AC01C701B6010F94DB609B0102
:10686000AC01688579858A859B850F944467688724
:1068700079878A879B87DF91CF91FF90EF90DF9098
:10688000CF9008958C3221E0920714F08CE291E0D1
:1068900090936517809364170D9432380F931F936C
:1068A000CF93DF9309EC11E1CDEDD6E1F801219111
:1068B0003191419151918F0160E070E080E89FE358
:1068C0000F943F686993799389939993F6E1CD3E4C
:1068D000DF0761F70F941A32DF91CF911F910F916B
:1068E0000C94882F9091021880910318981306C079
:1068F00080916C1190916D11892B21F080E00E94A4
:1069000005BCF0CF0895CF92DF92EF92FF92CF9324
:10691000DF932091B011222341F1EC0108960E94EF
:10692000CD8D6B017C0120E030E0A9010F947560F2
:1069300020E030E0A901882371F0BE016C5F7F4F39
:10694000CE010E945F959B01AC01C701B6010F9477
:10695000DB609B01AC01688579858A859B850F94F6
:106960004567688779878A879B87DF91CF91FF90FA
:10697000EF90DF90CF900895CF92DF92EF92FF9249
:106980008091300D882309F457C0C0902C0DD09011
:106990002D0DE0902E0DF0902F0D20E030E0A9019C
:1069A000C701B6010F947560882309F445C020E043
:1069B00030E040E05FE3C701B6010F94DB609B016C
:1069C000AC010F94DB602BED3FE049E450E40F9401
:1069D000DB609B01AC0160E070E080E89FE30F9416
:1069E0003F686B017C01C092B111D092B211E0926C
:1069F000B311F092B4116091730270917402072E7A
:106A0000000C880B990B0F947C602AE037ED43E271
:106A10005CE30F94DB60A70196010F94DB60609349
:106A20006F02709370028093710290937202FF90D4
:106A3000EF90DF90CF900895C12CD12C80E8E82E04
:106A40008FE3F82ED0CF0F931F93CF93DF9350E0B7
:106A5000FC01E40FF51F8081440F551F440F551FA3
:106A60004255564FEA01882329F188819981AA81EC
:106A7000BB81EB01088119812A813B810097A10527
:106A8000B10569F40C591F4F2F4F3F4FDA010D9399
:106A90001D932D933C9313978FEF808306C0081BA3
:106AA000190B2A0B3B0B37FDF7CFDF91CF911F91CD
:106AB0000F910895188219821A821B82F6CF2F92A5
:106AC0003F924F925F926F927F928F929F92AF927E
:106AD000BF92CF92DF92EF92FF920F931F93CF93CB
:106AE000DF93CDB7DEB76C970FB6F894DEBF0FBE5D
:106AF000CDBF8C015B015A834983FC01EF5AFF4FE4
:106B0000208131814281538129873A874B875C8775
:106B1000CA01B9010F947A606B017C01D5012D91F6
:106B20003D914D915C910F94DB600F9423682B0194
:106B30003C01E981FA812081318142815381C70181
:106B4000B6010F94DB600F9423684B015C01C30115
:106B5000B2010F94B868698B7A8B8B8B9C8B6837EA
:106B600071058105910540F428E730E040E050E0F0
:106B7000298B3A8B4B8B5C8BC501B4010F94B868A1
:106B80006D877E878F87988B6837710581059105A2
:106B900040F448E750E060E070E04D875E876F8723
:106BA000788BF801E35AFF4F4080518062807380F8
:106BB000C301B2010F947C6069837A838B839C83C9
:106BC00069897A898B899C890F947A606D8B7E8B19
:106BD0008F8B988F20E030E0A90169817A818B81C9
:106BE0009C810F947560882309F4E1C1A701960187
:106BF000C701B6010F94DB604B015C012D893E8912
:106C00004F89588DCA01B9010F94DB609B01AC011B
:106C1000C501B4010F9444674B015C0129813A819D
:106C20004B815C81CA01B9010F9445679B01AC019E
:106C3000C501B4010F943F680F9423680F94B8689E
:106C40006D837E838F83988766277727CB016419AE
:106C50007509860997090F947C604B015C016D856D
:106C60007E858F8598890F947A602B013C0120E006
:106C700030E0A901C501B4010F947560882309F4BF
:106C80009AC1A3019201C301B2010F94DB60698F25
:106C90007A8F8B8F9C8FA7019601C701B6010F9445
:106CA000DB609B01AC01698D7A8D8B8D9C8D0F947F
:106CB00044676B017C01A5019401C501B4010F94E7
:106CC00045679B01AC01C701B6010F943F680F9463
:106CD000E768D80195968D909D90AD90BC9098975F
:106CE000750164012D813E814F815885C21AD30AF6
:106CF000E40AF50A0F94B868C61AD70AE80AF90A2E
:106D0000F7FE8EC02D893E894F89588DCA01B90181
:106D10000F94DB606B017C0129813A814B815C819E
:106D2000CA01B9010F94456769877A878B879C8769
:106D300020E030E0A90169817A818B819C810F94E8
:106D40007560882309F43BC1C501B4010F947A60D2
:106D500029853A854B855C850F94DB60A7019601F8
:106D60000F9444676D837E838F839887A30192017C
:106D7000C301B2010F94DB609B01AC016D817E8188
:106D80008F8198850F9445672B013C0120E030E00E
:106D900040E850E469817A818B819C810F94DB60AB
:106DA0009B01AC01C301B2010F943F680F942368AB
:106DB0002B013C0120E030E0A9010F94A5691816D1
:106DC0001CF0412C512C3201C301B2010F94B86860
:106DD0006D837E838F83988786169706A806B906EB
:106DE00020F48D829E82AF82B8866D817E818F81F4
:106DF00098850F947A6029853A854B855C850F9438
:106E0000DB60A70196010F9445670F94436A0F94C6
:106E1000B86869877A878B879C87C12CD12C7601CB
:106E200069857A858B859C8529893A894B895C8916
:106E3000621B730B840B950B0F947A6029813A8146
:106E40004B815C810F943F6820E034E244EF59E4C9
:106E50000F94DB600F94B8684B015C0169857A85FB
:106E60008B859C852D853E854F855889621B730BCC
:106E7000840B950B0F947A6029813A814B815C8158
:106E80000F943F6820E034E244EF59E40F94DB6054
:106E90000F94B8682B013C013FE683169104A104CE
:106EA000B10408F090C0F401EE0FFF1FEE0FFF1FBA
:106EB000E25EF14F85919591A591B4918983292E38
:106EC0003A2EBD8B4FE6441651046104710408F05C
:106ED00083C0F201EE0FFF1FEE0FFF1FE25EF14FC6
:106EE00045915591659174919A01CB014D815E81D7
:106EF0006F817885D80199964D935D936D937C93BE
:106F00009C974C0D5D1D6E1D7F1DF80145A756A772
:106F100067A770ABEB5AFF4F49895A896B897C8907
:106F20004083518362837383D5968D929D92AD92F7
:106F3000BC92D897F80141AE52AE63AE74AEFD96E6
:106F400049814083218232825D8953833496208334
:106F500031838283938369857A858B859C85D196DD
:106F60006D937D938D939C93D49778962D853E85D4
:106F70004F85588920833183428353836C960FB6A3
:106F8000F894DEBF0FBECDBFDF91CF911F910F915F
:106F9000FF90EF90DF90CF90BF90AF909F908F9039
:106FA0007F906F905F904F903F902F90089560E09A
:106FB00070E0CB0141CE60E070E0CB0188CE60E0B4
:106FC00070E0CB01F3CEC501B4010E948A2E698323
:106FD000272E382E9D8B76CFC301B2010E948A2EB8
:106FE0009B0184CF8091021890910318891B8770B0
:106FF00019F490E080E008959091FF17992351F0E3
:10700000833030F48FEF890F19F08093FF17F1CFA1
:107010001092FF178091031827E6829FC001112468
:107020008D5C914FFC01208120FDE3CF209103185E
:107030002F5F2770209300183091031820910118BA
:10704000321304C0209100182093011808959091E4
:107050006F0081E091FD02C080E0089590916F0083
:107060009D7F90936F000895CF92DF92EF92FF92F1
:10707000FC01C080D180E280F3802091D511309155
:10708000D6114091D7115091D811C701B6010F9474
:10709000DB600F94B269609320187093211880937D
:1070A000221890932318C0921018D0921118E092D1
:1070B0001218F092131890910218809103189817E3
:1070C00031F0FF90EF90DF90CF900C94BC300E9495
:1070D00072340E94273840912018509121186091F5
:1070E00022187091231840930B0B50930C0B609354
:1070F0000D0B70930E0B882331F0FF90EF90DF9013
:10710000CF900C943399FF90EF90DF90CF9008953B
:107110004F925F926F927F928F929F92AF92BF92A7
:10712000CF92DF92EF92FF920F931F93CF93DF9353
:10713000EC018B017A016901F90180819181A281C1
:10714000B381FA014081518162817381F8018080AD
:107150009180A280B380488059806A807B80409271
:1071600004185092051860920618709207188092C1
:10717000081890920918A0920A18B0920B18409320
:107180000C1850930D1860930E1870930F1880937D
:10719000101890931118A0931218B09313182091FF
:1071A000D5113091D6114091D7115091D811F601D7
:1071B00060817181828193810F94DB600F94B26949
:1071C0004B015C012091D1113091D2114091D3112A
:1071D0005091D411F70160817181828193810F9464
:1071E000DB600F94B2696B017C012091CD1130916D
:1071F000CE114091CF115091D011F8016081718171
:10720000828193810F94DB600F94B2692B013C0162
:107210002091C9113091CA114091CB115091CC11DC
:10722000688179818A819B810F94DB600F94B269B8
:10723000609314187093151880931618909317186C
:10724000409218185092191860921A1870921B18D0
:10725000C0921C18D0921D18E0921E18F0921F18B0
:107260008092201890922118A0922218B092231890
:107270009091021880910318981791F0DF91CF91A7
:107280001F910F91FF90EF90DF90CF90BF90AF9044
:107290009F908F907F906F905F904F900C94BC3038
:1072A0000E9472340E94273840911C1850911D187A
:1072B00060911E1870911F180091181810911918DC
:1072C00020911A1830911B18C0901418D0901518DE
:1072D000E0901618F0901718C092FF0AD092000B99
:1072E000E092010BF092020B0093030B1093040B3E
:1072F0002093050B3093060B4093070B5093080B1C
:107300006093090B70930A0B40912018509121183B
:10731000609122187091231840930B0B50930C0B23
:1073200060930D0B70930E0B882391F0DF91CF913A
:107330001F910F91FF90EF90DF90CF90BF90AF9093
:107340009F908F907F906F905F904F900C943399A7
:10735000DF91CF911F910F91FF90EF90DF90CF9031
:10736000BF90AF909F908F907F906F905F904F9065
:107370000895CF92DF92EF92FF92CF93DF93C82FC1
:107380000E94273894E0C99FE0011124FE01E150DA
:10739000F54FC080D180E280F38081110E94339943
:1073A000C352D94EC701B6010F947C602881398140
:1073B0004A815B810F94DB60DF91CF91FF90EF906A
:1073C000DF90CF9008953F924F925F926F927F929D
:1073D0008F929F92AF92BF92CF92DF92EF92FF92E5
:1073E0000F931F93CF93DF93CDB7DEB768970FB698
:1073F000F894DEBF0FBECDBFD82E2A013B01480155
:1074000059013E2C20E030E0A901C501B8010F94DC
:107410007560811110C081E08D1508F0B0C060E08A
:1074200070E080E793E420E030E040E752E40F941E
:107430003F684B015C018D8A9E8AAF8AB88E0D2D04
:1074400010E0F801E55EF14FE491BB24B3941E1601
:107450000CF4B12CCC24C39420E030E0A901C3018A
:10746000B2010F94A56918160CF0C12CBC1471F070
:1074700092E0D9120BC0332049F081E00F942435FB
:1074800069E170E080E090E00E94509980E00E9405
:10749000B93969837A838B839C8381E00E94B939EF
:1074A0006D837E838F83988782E00E94B9396987D4
:1074B0007A878B879C8783E00E94B9396D877E87A6
:1074C0008F87988B000F111F000F111FE1E0F0E074
:1074D000EC0FFD1F0E0F1F1FF80110821182128288
:1074E00013829E01235F3F4FAE01475F5F4FBE0196
:1074F0006B5F7F4FCE0101960E948838F801408271
:10750000518262827382198A1A8A1B8A1C8ACE016E
:1075100041967C018E010B5E1F4F9E01235F3F4F02
:10752000AE01475F5F4FBE016B5F7F4F40970F9487
:10753000AE210E947234BC1451F092E0D91205C001
:10754000332019F080E00F9424350E943032689681
:107550000FB6F894DEBF0FBECDBFDF91CF911F9164
:107560000F91FF90EF90DF90CF90BF90AF909F90E2
:107570008F907F906F905F904F903F90089560E064
:1075800070E88BE395E44FCFCF92DF92EF92FF92BA
:10759000CF93DF93C82F0E94273894E0C99FE00162
:1075A0001124FE01ED50F54FC080D180E280F380C0
:1075B00081110E943399C352D94EC701B6010F946D
:1075C0007C60288139814A815B810F94DB60DF9187
:1075D000CF91FF90EF90DF90CF9008950E942738D1
:1075E00090910318909302189093011890930018AB
:1075F00094E69093FF1720ED33E030936D112093C4
:107600006C1181110E94339981E08093F20A0895F0
:10761000CF93DF9324E0829FC0011124EC01C55079
:10762000D24FFC01E35CF24F8F5C924FDC012D9155
:107630003D914D915C9160817181828193810F9424
:107640004567688379838A839B83DF91CF9108950F
:1076500080FF04C09091AF1190FD8E7F81FF05C027
:107660009091AF11969590FD8D7F82FF06C090910D
:10767000AF119695969590FD8B7F08958F929F926E
:10768000AF92BF92CF92DF92EF92FF92CF93DF93B0
:1076900020914302222309F49EC0EC0180918409C9
:1076A000C82ED12CF12CE12C80FF2CC080904502FB
:1076B00090904602A0904702B090480228813981FC
:1076C0004A815B81C501B4010F94A569181624F4A1
:1076D00088829982AA82BB82809051029090520245
:1076E000A0905302B0905402288139814A815B8175
:1076F000C501B4010F94756087FF04C08882998228
:10770000AA82BB82D701C601B695A79597958795A2
:1077100080FF2CC08090490290904A02A0904B02BA
:10772000B0904C022C813D814E815F81C501B40136
:107730000F94A569181624F48C829D82AE82BF82B4
:107740008090550290905602A0905702B090580237
:107750002C813D814E815F81C501B4010F9475601C
:1077600087FF04C08C829D82AE82BF8282E0F69445
:10777000E794D794C7948A95D1F7C0FE2CC0C090E7
:107780004D02D0904E02E0904F02F09050022885BA
:1077900039854A855B85C701B6010F94A56918161E
:1077A00024F4C886D986EA86FB86C0905902D09018
:1077B0005A02E0905B02F0905C02288539854A8588
:1077C0005B85C701B6010F94756087FF04C0C8864A
:1077D000D986EA86FB86DF91CF91FF90EF90DF900C
:1077E000CF90BF90AF909F908F9008952F923F922F
:1077F0004F925F926F927F928F929F92AF92BF92C1
:10780000CF92DF92EF92FF920F931F93CF93DF936C
:10781000CDB7DEB7C257D1090FB6F894DEBF0FBEA1
:10782000CDBF8CE79CE00E943E3B80916B1183FDB5
:107830007EC020916B0230916C0240916D0250919C
:107840006E026091880C7091890C80918A0C9091E5
:107850008B0C0F947560882309F469C01091320E67
:10786000111161C080915D0290915E02019720919B
:10787000621730916317281739073CF40E94CEB87D
:1078800085EA9DE00E94909E11E020916B0230916C
:107890006C0240916D0250916E026091880C709163
:1078A000890C80918A0C90918B0C0F9444676B012A
:1078B0007C0120E030E0A9010F94A56987FF04C096
:1078C000F7FAF094F7F8F09420916F02309170027B
:1078D0004091710250917202C701B6010F94DB60B2
:1078E00020E030E84BE354E40F94A5691816ECF45B
:1078F0000E94CEB886E89DE00E94909E8091880C00
:107900009091890CA0918A0CB0918B0C80936B02A2
:1079100090936C02A0936D02B0936E0288E89CE095
:107920000E94343804C010E0B0CF1111E7CF2AE034
:1079300037ED43E25CE360913F0270914002809139
:107940004102909142020F94DB606B017C016091D7
:10795000750270917602072E000C880B990B0F941C
:107960007C609B01AC01C701B6010F94DB602196DE
:107970006CAF7DAF8EAF9FAF21978091B011882300
:1079800001F1C090280DD090290DE0902A0DF090C3
:107990002B0D20E030E0A901C701B6010F947560FE
:1079A000882309F43EC02091840C3091850C4091CD
:1079B000860C5091870CC701B6010F94A569181663
:1079C00084F18E01035C1F4F28E83CE044E85CE052
:1079D00060E87CE08CE79CE00F94263180E1ECE7E6
:1079E000FCE0AFE5B2E001900D928A95E1F7CE5848
:1079F000DF4F0FB6F894DEBF0FBECDBFDF91CF9142
:107A00001F910F91FF90EF90DF90CF90BF90AF90BC
:107A10009F908F907F906F905F904F903F902F90AE
:107A2000089580E1EFE5F2E0DE01519601900D92BC
:107A30008A95E1F780E1ECE7FCE0DE011196019028
:107A40000D928A95E1F7CE0141960E94478E182F3C
:107A5000092FCE0101960E94478E6C968FAF6C97CE
:107A60006D969FAF6D97181303C0091709F426C4CC
:107A700089899A89AB89BC896B968CAF9DAFAEAF73
:107A8000BFAF6B979C01AD0169817A818B819C812D
:107A90000F9444672A966FAF2A972C967FAF2C9746
:107AA00064968FAF649766969FAF66978D899E891F
:107AB000AF89B88DE3968CAF9DAFAEAFBFAFE39704
:107AC0009C01AD016D817E818F8198850F94446703
:107AD000362E272E22968FAF229726969FAF269777
:107AE000298D3A8D4B8D5C8D69857A858B859C853A
:107AF0000F944467A1966CAF7DAF8EAF9FAFA197F7
:107B00002D8D3E8D4F8D58A16D857E858F859889F1
:107B10000F9444672B013C0120E030E0A901632D64
:107B2000722D22968FAD229726969FAD26970F94A1
:107B30007560881F8827881FA2968FAFA29720E0C4
:107B400030E0A9012A966FAD2A972C967FAD2C972D
:107B500064968FAD649766969FAD66970F94756037
:107B6000812C912C70E8A72E7FEBB72E87FD06C0E5
:107B7000812C912C20E8A22E2FE3B22E20E030E0C1
:107B8000A901632D722D22968FAD229726969FAD67
:107B900026970F947560C12CD12C90E8E92E9FE3B5
:107BA000F92E87FF06C0C12CD12C80E8E82E8FEB80
:107BB000F82E6C969FAD6C97191709F410C2C50189
:107BC000B4010F94B1682E966FAF2E976D96AFAD3E
:107BD0006D970A1709F407C2C701B6010F94B1687F
:107BE00062966FAF6297A50194012A966FAD2A97AE
:107BF0002C967FAD2C9764968FAD649766969FAD5B
:107C000066970F94DB60A7966CAF7DAF8EAF9FAF8A
:107C1000A797A7019601632D722D22968FAD22970B
:107C200026969FAD26970F94DB60AB966CAF7DAF29
:107C30008EAF9FAFAB979B01AC01A7966CAD7DADAE
:107C40008EAD9FADA7970F94A56918160CF0CFC104
:107C50002A96EFAC2A972C96FFAC2C976496CFAC63
:107C600064976696DFAC669749AE5AAE6BAE7CAE53
:107C70009701A601C301B2010F943F68AF966CAFA4
:107C80007DAF8EAF9FAFAF979701A601A1966CAD68
:107C90007DAD8EAD9FADA1970F943F68A1966CAF5F
:107CA0007DAF8EAF9FAFA1972A962FAD2A972C96C6
:107CB0003FAD2C9764964FAD649766965FAD66971F
:107CC000632D722D22968FAD229726969FAD269713
:107CD0000F943F6829966CAF7DAF8EAF9FAF299709
:107CE0009B01AC016B966CAD7DAD8EAD9FAD6B977E
:107CF0000F94DB609B01AC01E3966CAD7DAD8EAD66
:107D00009FADE3970F9444676B966CAF7DAF8EAFDA
:107D10009FAF6B97AF968CAD9DADAEADBFADAF973E
:107D2000BF7725968CAF9DAFAEAFBFAF25972E9690
:107D30009FAD2E9791118DC1A2963FACA297300EA8
:107D4000A296AFADA2978A2F90E09C016D964FADA1
:107D50006D97240F311D47FD3A952D963FAF2EAFFD
:107D60002D9729968CAD9DADAEADBFAD2997BF7750
:107D700061968CAF9DAFAEAFBFAF6197A12F110FD2
:107D8000BB0B2B96BFAFAEAF2B97832D032C000CF4
:107D9000990B2D962EAD3FAD2D978217930709F4C1
:107DA0006CC262963FAD6297330E832D0E94F090B5
:107DB0006B017C012FEF3FEF4FE75FE761966CAD02
:107DC0007DAD8EAD9FAD61970F94926A811118C100
:107DD0002FEF3FEF4FE75FE761966CAD7DAD8EAD66
:107DE0009FAD61970F94756018160CF009C16989F1
:107DF0007A898B899C896DA77EA78FA798AB2B96D4
:107E00008EAD9FAD2B978630910508F00CC1432DA8
:107E1000032C000C550B4630510508F004C1BC0181
:107E2000CE018D960E94FD926B017C01CE010996D8
:107E30000E94CD8DA70196010F94DB606B017C0140
:107E4000AC019B010F94926A882319F0C12CD12CAC
:107E50007601832D0E94F0904B015C0189A69AA6C1
:107E6000ABA6BCA64D885E886F88788CA301920172
:107E70000F947560882309F488CF2FEF3FEF4FE709
:107E80005FE725966CAD7DAD8EAD9FAD25970F94C8
:107E9000926A81110FC02FEF3FEF4FE75FE7259602
:107EA0006CAD7DAD8EAD9FAD25970F9475601816A6
:107EB0000CF4C2C0AB962CAD3DAD4EAD5FADAB97F3
:107EC000A7966CAD7DAD8EAD9FADA7970F94A569BC
:107ED00018160CF0ACC029893A894B895C896DA5CC
:107EE0007EA58FA598A90F9444674B015C01AC0156
:107EF0009B01AF966CAD7DAD8EAD9FADAF970F94EE
:107F0000DB609B01AC016D8D7E8D8F8D98A10F94F0
:107F1000456769AF7AAF8BAF9CAFA5019401A1967D
:107F20006CAD7DAD8EAD9FADA1970F94DB60298DBB
:107F30003A8D4B8D5C8D0F9445671DA21EA21FA22A
:107F400018A6A70196010F94456769A37AA38BA38E
:107F50009CA3DE0195967D018E01035C1F4F9E015F
:107F6000275C3F4FAE014F5D5F4FBE01675D7F4FA6
:107F7000CE018D960F94AE2108CF20E030E0A9010C
:107F800069857A858B859C850F94456769877A8793
:107F90008B879C8719A21AA21BA21CA29E012F5D8F
:107FA0003F4F79018E01035C1F4F24513109AE010F
:107FB000475F5F4FBE016B5F7F4FCE0101960F940D
:107FC000AE210CCDA701960169857A858B859C85AC
:107FD0000F94456769877A878B879C874BC22E965B
:107FE0001FAE2E97F3CD62961FAE6297FCCDE32CA9
:107FF000F22C2296CFAC22972696DFAC269734CE71
:108000006B962CAD3DAD4EAD5FAD6B97C701B60124
:108010000F94446729962CAD3DAD4EAD5FAD2997C9
:108020000F943F68E8CEC12CD12C7601FFCEA3017E
:108030009201C501B40157CF8D859E85AF85B88962
:1080400089AF9AAFABAFBCAF69857A858B859C85CC
:1080500074CF20E030E0A9012A966FAD2A972C96C4
:108060007FAD2C9764968FAD649766969FAD6697AB
:108070000F947560482E441C4424441C342C310E4B
:108080006296BFAD6297B11124C2512C92016C96D9
:108090004FAD6C97240F311D47FD3A952B963FAF9E
:1080A0002EAF2B97802F000F990B63969FAF8EAF4B
:1080B0006397832D032C000C990B2B96AEADBFADAF
:1080C0002B978A179B0709F4D8C02E96BFAD2E9721
:1080D0003B0E832D0E9486919B01AC012DA73EA7EC
:1080E0004FA758AB29966CAD7DAD8EAD9FAD29974E
:1080F0000F94DB606B962CAD3DAD4EAD5FAD6B97D5
:108100000F94456769A77AA78BA79CA7632D032CBB
:10811000000C770B6630710508F0C1C163962EAD77
:108120003FAD63972630310508F0B9C1A901CE01F2
:1081300089960E941F916B017C01CE0109960E94D5
:10814000CD8DA70196010F94DB606B017C01AC0122
:108150009B010F94926A882319F0C12CD12C7601CF
:1081600049885A886B887C888DA49EA4AFA4B8A83F
:10817000A5019401C301B2010F947560882309F42D
:1081800098CF2FEF3FEF4FE75FE725966CAD7DADC2
:108190008EAD9FAD25970F94926A81110FC02FEF7E
:1081A0003FEF4FE75FE725966CAD7DAD8EAD9FADA0
:1081B00025970F94756018160CF47EC1AB962CAD04
:1081C0003DAD4EAD5FADAB97A7966CAD7DAD8EADC1
:1081D0009FADA7970F94A56918160CF064C1A30171
:1081E0009201C501B4010F9444674B015C01AC01DD
:1081F0009B01AF966CAD7DAD8EAD9FADAF970F94EB
:10820000DB609B01AC016D8D7E8D8F8D98A10F94ED
:10821000456769AF7AAF8BAF9CAFA5019401A1967A
:108220006CAD7DAD8EAD9FADA1970F94DB60298DB8
:108230003A8D4B8D5C8D0F9445671DA21EA21FA227
:1082400018A6A70196010F94456769A37AA38BA38B
:108250009CA3CE0185967C018E01035C1F4F9E017D
:10826000275C3F4FAE014F5D5F4FBE01675D7F4FA3
:1082700008960F94AE2181111CCF20915F0230919E
:108280006002409161025091620269817A818B8122
:108290009C810F947560811111C02091630230910F
:1082A000640240916502509166026D817E818F81EA
:1082B00098850F947560882309F490CBC980DA8083
:1082C000EB80FC80C701B6010E94B88D882309F4B9
:1082D00054CE6D817E818F8198850E94B88D8823D0
:1082E00009F44BCE6C968FAD6C970E9486919B01E2
:1082F000AC01C701B6010F9444672BEA33ED44E6A5
:108300005CE30F94DB602B013C018D819E81AF818A
:10831000B88525968CAF9DAFAEAFBFAF25976D9654
:108320008FAD6D970E94F09029966CAF7DAF8EAFA8
:108330009FAF29976C96AFAD6C978A2FAA0F990BB8
:108340006D96BFAD6D97AB2EBB0FBB0826E0289F87
:108350004001299F900C1124F401EA0DFB1DEE0F42
:10836000FF1FEE0FFF1FE956F34FC080D180E28060
:10837000F3800196289F8001299F100D1124F80198
:10838000EA0DFB1DEE0FFF1FEE0FFF1FE956F34F27
:10839000A701960160817181828193810F94446766
:1083A000A30192010F94DB60A70196010F9445672A
:1083B0006B017C01F5013196D401AE0FBF1FAA0FEE
:1083C000BB1FAA0FBB1FA956B34F8D909D90AD90B8
:1083D000BC90E00FF11FEE0FFF1FEE0FFF1FE956DD
:1083E000F34FA501940160817181828193810F9483
:1083F0004467A30192010F94DB60A50194010F94DF
:108400004567A70196010F9444674B015C012996CB
:108410002CAD3DAD4EAD5FAD299725966CAD7DADD4
:108420008EAD9FAD25970F9444672BEA33ED44E65C
:108430005CE30F94DB609B01AC01C501B4010F94B8
:10844000DB60A70196010F9445676B017C01CE01AB
:1084500009960E94CD8D9B01AC01C701B6010F9416
:10846000DB606B017C01AC019B010F94926A882355
:1084700009F4A8CD19A21AA21BA21CA2CE018196B2
:108480007C018E01035C1F4F9E01235F3F4FAE01B5
:10849000475F5F4FBE016B5F7F4F809790CDC12CD0
:1084A000D12C76014ACE2D893E894F89588D69A5F8
:1084B0007AA58BA59CA597CE8D859E85AF85B8891D
:1084C00089AF9AAFABAFBCAF69857A858B859C8548
:1084D000B4CE812F6C969FAD6C97891B082E000C33
:1084E000990B97FF03C0919581959109682E202ED5
:1084F0006D96AFAD6D972A1A822D220C990B97FFBE
:1085000003C0919581959109282EA2967FACA297E0
:10851000700E2E962FAD2E97022E000C330B2D963B
:108520003FAF2EAF2D97A2969FADA297892F90E0D7
:1085300065969FAF8EAF6597A42DB0E06796BFAFED
:10854000AEAF679762962FAD6297022E000C330B89
:10855000A3963FAF2EAFA397611003C0222009F46A
:108560008CCE2E965FAC2E97530C852D0E94869153
:108570006DAB7EAB8FAB98AF62963FAD6297370D18
:108580002A963FAF2A97832F0E94F0906B017C01BF
:10859000C9AADAAAEBAAFCAA8DA89EA8AFA8B8AC73
:1085A000A501940129966CAD7DAD8EAD9FAD299747
:1085B0000F94DB606B962CAD3DAD4EAD5FAD6B9710
:1085C0000F9445676DA77EA78FA798AB6B962CADD0
:1085D0003DAD4EAD5FAD6B97C701B6010F944467DB
:1085E00029962CAD3DAD4EAD5FAD29970F943F68F8
:1085F0009B01AC0129A73AA74BA75CA7E72C072C46
:10860000000CFF08032D032C000C110BC501B40155
:108610000F947560881F8827881F4812D3C0B8013F
:1086200067968EAD9FAD6797681B790B66307105B5
:1086300008F0AEC0A3964EAD5FADA3974E0D5F1D83
:108640004630510508F0A4C0CE0189960E94FD92E3
:108650006B017C01CE0109960E94CD8DA701960188
:108660000F94DB606B017C01AC019B010F94926A5B
:10867000882319F0C12CD12C76012FEF3FEF4FE763
:108680005FE725966CAD7DAD8EAD9FAD25970F94C0
:10869000926A81110FC02FEF3FEF4FE75FE72596FA
:1086A0006CAD7DAD8EAD9FAD25970F94756018169E
:1086B0000CF47BC0AB962CAD3DAD4EAD5FADAB9732
:1086C000A7966CAD7DAD8EAD9FADA7970F94A569B4
:1086D00018160CF061C029893A894B895C8969A513
:1086E0007AA58BA59CA50F9444674B015C01AC0156
:1086F0009B01AF966CAD7DAD8EAD9FADAF970F94E6
:10870000DB609B01AC016D8D7E8D8F8D98A10F94E8
:10871000456769AF7AAF8BAF9CAFA5019401A19675
:108720006CAD7DAD8EAD9FADA1970F94DB60298DB3
:108730003A8D4B8D5C8D0F9445671DA21EA21FA222
:1087400018A6A70196010F94456769A37AA38BA386
:108750009CA3DE0195967D018E01035C1F4F9E0157
:10876000275C3F4FAE014F5D5F4FBE016F5C7F4F97
:10877000CE0189960F94AE21882309F47ECD2A96E6
:108780007FAC2A972A9467FC78CD27FEE5CE75CD7D
:10879000C12CD12C76015ECF2D893E894F89588D11
:1087A00069A97AA98BA99CA99ECF8D859E85AF8545
:1087B000B88989AF9AAFABAFBCAF69857A858B8535
:1087C0009C85BBCF2D966EAD7FAD2D97600F711F31
:1087D0006630710508F0A8C0A70165962EAD3FADC3
:1087E0006597421B530B4630510508F09DC0CE01E2
:1087F0008D960E941F916B017C01CE0109960E940B
:10880000CD8DA70196010F94DB606B017C01AC015B
:108810009B010F94926A882319F0C12CD12C760108
:108820002FEF3FEF4FE75FE725966CAD7DAD8EAD47
:108830009FAD25970F94926A81110FC02FEF3FEFE4
:108840004FE75FE725966CAD7DAD8EAD9FAD25976B
:108850000F94756018160CF474C0AB962CAD3DAD3A
:108860004EAD5FADAB97A7966CAD7DAD8EAD9FADB8
:10887000A7970F94A56918160CF05AC029893A8950
:108880004B895C896DA97EA98FA998AD0F94446727
:108890004B015C01AC019B01AF966CAD7DAD8EAD23
:1088A0009FADAF970F94DB609B01AC016D8D7E8D0A
:1088B0008F8D98A10F94456769AF7AAF8BAF9CAF4E
:1088C000A5019401A1966CAD7DAD8EAD9FADA19734
:1088D0000F94DB60298D3A8D4B8D5C8D0F9445672D
:1088E0001DA21EA21FA218A6A70196010F944567FC
:1088F00069A37AA38BA39CA3CE0185967C018E01EC
:10890000035C1F4F9E01275C3F4FAE014F5D5F4FE1
:10891000BE01635D7F4F40960F94AE21882309F41A
:10892000ACCC352C6A942FCFC12CD12C760165CFDD
:108930002D893E894F89588D6DA57EA58FA598A953
:10894000A5CF8D859E85AF85B88989AF9AAFABAF2E
:10895000BCAF69857A858B859C85C2CF8091AA0939
:108960009091AB09A091AC09B091AD0980933F0201
:1089700090934002A0934102B09342028091A809D3
:108980009091A90990937602809375020895809141
:108990003F0290914002A0914102B0914202809327
:1089A000AA099093AB09A093AC09B093AD0980914B
:1089B0007502909176029093A9098093A80984E6A4
:1089C00090E0909376028093750208958F929F9223
:1089D000AF92BF92CF92DF92EF92FF92CF93DF934D
:1089E00080903F0290904002A0904102B0904202DD
:1089F000FC01C080D180E280F38020E030E0A9015A
:108A0000C701B6010F947560882341F0C0923F0200
:108A1000D0924002E0924102F0924202C09175026F
:108A2000D091760284E690E090937602809375026E
:108A3000C0906F02D0907002E0907102F0907202CC
:108A400080E090E0A0E8BFE380936F029093700213
:108A5000A0937102B09372020E94F63B80923F0293
:108A600090924002A0924102B0924202D0937602CC
:108A7000C0937502C0926F02D0927002E0927102B0
:108A8000F0927202DF91CF91FF90EF90DF90CF9044
:108A9000BF90AF909F908F9008950F931F938C017C
:108AA0002BE632E047E652E063E672E08FE592E0C3
:108AB0000F9426311F910F9108954F925F926F92FC
:108AC0007F928F929F92AF92BF92CF92DF92EF925E
:108AD000FF920F931F93CF93DF93CDB7DEB72C9701
:108AE0000FB6F894DEBF0FBECDBF2B013C01298726
:108AF0003A874B875C8747015801F601E080F18097
:108B00000281138120E030E0A901B701C8010F9470
:108B10007560882309F484C05E2D4F2D302F212FDE
:108B2000852F942FA32FB22F89839A83AB83BC8385
:108B300020E030E0A901B701C8010F9475608111F0
:108B400004C0E12CF12C08E413E4C701D8018D83A3
:108B50009E83AF83B887A5019401609167027091ED
:108B600068028091690290916A020F94756087FF94
:108B70000CC08092670290926802A0926902B09243
:108B80006A02CE0101960E944D4540925F025092CA
:108B90006002609261027092620289859A85AB855B
:108BA000BC858093630290936402A0936502B093A6
:108BB0006602CE0105960E944D45A5019401609183
:108BC0006702709168028091690290916A020F9425
:108BD000A569181664F48092670290926802A092C8
:108BE0006902B0926A02CE0101960E944D450E9430
:108BF00072342C960FB6F894DEBF0FBECDBFDF9156
:108C0000CF911F910F91FF90EF90DF90CF90BF9089
:108C1000AF909F908F907F906F905F904F9008954E
:108C200050E040E030E820E47BCFCF92DF92EF923B
:108C3000FF920F931F936A01E0906702F090680221
:108C40000091690210916A02FB0120813181428109
:108C50005381FC0160817181828193810E945D4515
:108C60001F910F91FF90EF90DF90CF900895CF92DA
:108C7000DF92EF92FF920F931F936B01FC01E08054
:108C8000F18002811381EFE5F2E024813581468194
:108C9000578160817181828193810E945D451F911E
:108CA0000F91FF90EF90DF90CF900895AF92BF9219
:108CB000CF92DF92EF92FF920F931F93CF93DF93A8
:108CC00000D01F92CDB7DEB7FC01E080F1800281B9
:108CD0001381611112C0A0906702B0906802C09029
:108CE0006902D0906A029501A601B701C8010F94EC
:108CF000756087FF02C07501860120E030E048EC16
:108D000053E4B701C8010F94756087FD04C0E12CDE
:108D1000F12C08EC13E4C701D80189839A83AB8353
:108D2000BC8368ED72E0CE0101960E9437460F9039
:108D30000F900F900F90DF91CF911F910F91FF90A7
:108D4000EF90DF90CF90BF90AF900895EF92FF9299
:108D50000F931F93CF93DF937C018B010E94109A96
:108D6000CFE5D2E020916F02309170024091710204
:108D700050917202F70160817181828193810F9419
:108D80003F682C853D854E855F850F9445676C87D0
:108D90007D878E879F87C8010E944D45DF91CF91C7
:108DA0001F910F91FF90EF900C947234CF92DF924D
:108DB000EF92FF921F93CF93DF93CDB7DEB760970B
:108DC0000FB6F894DEBF0FBECDBF182F80E00E9413
:108DD000B93960939C0970939D0980939E09909383
:108DE0009F0981E00E94B9396093A0097093A1099D
:108DF0008093A2099093A30982E00E94B9396093FD
:108E0000A4097093A5098093A6099093A7091D86CC
:108E10001E861F86188AC0909C09D0909D09E090FC
:108E20009E09F0909F09C982DA82EB82FC82C09091
:108E3000A009D090A109E090A209F090A309CD82E9
:108E4000DE82EF82F88669877A878B879C8783E04A
:108E50000E94B9396D877E878F87988B8091B0117A
:108E6000882321F0CE0101960E940D341E3FB9F4F3
:108E700080E1FE013196AFE5B2E001900D928A9556
:108E8000E1F760960FB6F894DEBF0FBECDBFDF915D
:108E9000CF911F91FF90EF90DF90CF90089584E0E5
:108EA000189FF0011124DF01A15ABD4F81E090E02D
:108EB0008C0F9D1FE80FF91F4081518162817381E2
:108EC0004D935D936D937C931397DBCF0D941A3282
:108ED0000F931F93CF93DF93EC018B0181E00F94ED
:108EE000243569E170E080E090E00E945099B8017B
:108EF000CE010E943746C091E80B80E00F942435E4
:108F00001092E80B82E00E94D6460E946647C2FBA0
:108F1000CC27C0F981E08C27DF91CF911F910F9171
:108F200008952F923F924F925F926F927F928F920D
:108F30009F92AF92BF92CF92DF92EF92FF920F93E8
:108F40001F93CF93DF93CDB7DEB766970FB6F89434
:108F5000DEBF0FBECDBFF82E282E312CF101E55E0D
:108F6000F14FD49022E0821332C00E94F58F81111C
:108F70003DC10E947BBA811139C187E19EE00E9408
:108F8000FE8B20E030E0A9010F9475608823F9F092
:108F90006D2DDD0C770B880B990B0F947C602B01EA
:108FA0003C0187E19EE00E94FE8B4B015C0120E0CA
:108FB00030E040EA50E40F94756011E087FF1CC078
:108FC000812C912C90EAA92E90E4B92E15C06D2D1C
:108FD000DD0C770B880B990B0F947C602B013C0107
:108FE000C101880F991F880F991F815F914F0E94BF
:108FF000FE8B4B015C0110E0A3019201C501B4019D
:109000000F94DB604B015C016101CC0CDD1CCC0CCE
:10901000DD1CC6018D5F914F0E94FE8BEE24E39410
:10902000E12620E030E040EC5FE30F94DB60A30139
:1090300092010F94DB60AB01BC0100E010E09801ED
:109040008F2D0E94E33920E030E0A901C501B40171
:109050000F947560F601E950F24FFA8BE98B882383
:1090600009F44DC0F2E000E010E020E431E4FF1626
:1090700019F000E010E09801B501A4017058E12C4E
:109080008F2D0E94E339A5019401C501B4010F940D
:1090900045676B8B7C8B8D8B9E8B22E0F216E9F003
:1090A000F101EC50F24F6491611107C00E94CEB8FB
:1090B00082ED9DE00E94909E6AE070E090E080E08A
:1090C0000F947A609B01AC0160E070E088E492E468
:1090D0000F943F688B019C0104C000E010E020EC7D
:1090E00030E4EE24E3944B895C896D897E898F2D71
:1090F0000E94E33932E0F312D0C00E9438BA81E016
:1091000090E0A0E0B0E00F2C04C0880F991FAA1FC8
:10911000BB1F0A94D2F72091AF11282B2093AF11D7
:1091200020918409822B8093840989899A890E94DD
:10913000FE8BF601E15AFD4F608371838283938336
:1091400082E0F8121AC02091F9173091FA17409175
:10915000FB175091FC176091670270916802809133
:10916000690290916A020F9444676093670270935A
:1091700068028093690290936A02F601EF5CF24FF5
:1091800010821182128213828F2D0E94083B0E944E
:109190006647F601E15AFD4F80819181A281B3813A
:1091A000F601E458F34F80839183A283B38392E066
:1091B000F916A9F18CE0E9E8F2E0DE0111960190E0
:1091C0000D928A95E1F7E1E0F0E0EC0FFD1FEC0D68
:1091D000FD1D80809180A280B38020E030E0A90155
:1091E000C501B4010F94756081111EC066960FB65B
:1091F000F894DEBF0FBECDBFDF91CF911F910F91CD
:10920000FF90EF90DF90CF90BF90AF909F908F90A6
:109210007F906F905F904F903F902F9008950E94A5
:10922000EC8F8111E3CFC6CF20E030E0A901C5016A
:10923000B4010F94A56987FF04C0B7FAB094B7F8DA
:10924000B094F601E15AFD4F6F01A3019201C501EF
:10925000B4010F94DB609B01AC01F6016081718168
:10926000828193810F944467F601608371838283C6
:109270009383F2E080E090E0A0E4B1E4FF1621F0F7
:1092800080E090E0A8E4B2E48D879E87AF87B88B3A
:10929000CE010D960E944D45A9CF81E090E0A0E05F
:1092A000B0E00F2C04C0880F991FAA1FBB1F0A949F
:1092B000D2F72091AF11282B2093AF112091840970
:1092C000822B8093840989899A890E94FE8BF601FA
:1092D000E15AFD4F60837183828393834ECFCF9396
:1092E000DF93CDB7DEB72C970FB6F894DEBF0FBE75
:1092F000CDBF0F94F8320E9427389CE0EFEFFAE0E0
:10930000DE01119601900D929A95E1F781110E946C
:109310003399CE0101960E9417FD2C960FB6F89452
:10932000DEBF0FBECDBFDF91CF9108952F923F9248
:109330004F925F926F927F928F929F92AF92BF9265
:10934000CF92DF92EF92FF920F931F93CF93DF9311
:1093500000D0CDB7DEB780905F0290906002A09001
:109360006102B0906202409063025090640260908B
:10937000650270906602C0906702D0906802E0902B
:109380006902F0906A020E94882F0E94BC340EEF9E
:1093900010E185E492E09B838A8382EF282E80E1AE
:1093A000382E198289810E94083BC8010E94FE8BD9
:1093B000EA81FB816193719381939193FB83EA83AB
:1093C000C1010E94FE8BEA81FB81608771878287E1
:1093D0009387F981FF5FF9830C5F1F4F84E0280EAC
:1093E000311CF330F9F660E08DED9AE00E942B9885
:1093F0000E944E34A501940160915F027091600259
:1094000080916102909162020F94756081111CC07D
:10941000A3019201609163027091640280916502E0
:10942000909166020F94756081110EC020916702C1
:10943000309168024091690250916A02C701B601F9
:109440000F9475608823B9F00F900F900F90DF9103
:10945000CF911F910F91FF90EF90DF90CF90BF9031
:10946000AF909F908F907F906F905F904F903F90C4
:109470002F900C946F490F900F900F90DF91CF9128
:109480001F910F91FF90EF90DF90CF90BF90AF9022
:109490009F908F907F906F905F904F903F902F9014
:1094A000089580919B09659B6EC0806180939B09A4
:1094B0009091030180919B0991FF67C08062809326
:1094C0009B0980919B094B9B62C0846080939B09A0
:1094D00080919B0990919A09981709F45AC092E0DB
:1094E0009093990980939A098091A40B811105C0EA
:1094F0008091A60B882309F459C08091F10A80FF5E
:1095000010C08091A50B80FD0CC08091980984FF4C
:1095100008C08091E80B80618093E80B80E00E9496
:1095200037FD8091F10A869580FF11C08091A50BCF
:10953000869580FD0CC08091980985FF08C08091B8
:10954000E80B80628093E80B81E00E9437FD8091F8
:10955000F10A8695869580FF29C08091A50B869596
:10956000869580FF23C08091A60B8823F9F0809117
:10957000980982FF1BC08091E80B84608093E80B00
:1095800082E00C9437FD8F7E91CF8F7D98CF8B7FBB
:109590009DCF80919909882309F4A6CF81508093AB
:1095A00099098111A1CF909398099ECF0895809138
:1095B000A40B811104C08091A60B882331F062E0D6
:1095C00070E080E090E00C94509908953F924F92A3
:1095D0005F926F927F928F929F92AF92BF92CF9243
:1095E000DF92EF92FF920F931F93CF93DF9300D000
:1095F0001F92CDB7DEB7382E80E090E0A0E2B1E454
:1096000089839A83AB83BC83C090F917D090FA17F3
:10961000E090FB17F090FC1720E030E0A901C701B3
:10962000B6010F94756087FF0CC0A701960160E03A
:1096300070E080E291E40F94446769837A838B83BE
:109640009C8360E0CE0101960E94564640905F02E6
:10965000509060026090610270906202809063029C
:1096600090906402A0906502B0906602332089F168
:109670000E947BBA19821A821B821C82E0906702C8
:10968000F09068020091690210916A02CE01019681
:109690006C01A5019401C301B2010E945D453092A5
:1096A000A60B0E94D74A0F900F900F900F90DF915A
:1096B000CF911F910F91FF90EF90DF90CF90BF90CF
:1096C000AF909F908F907F906F905F904F903F9062
:1096D00008950E9438BACECF4F925F926F927F92D8
:1096E0008F929F92AF92BF92CF92DF92EF92FF92B2
:1096F000CF93DF9300D000D0CDB7DEB79E838D83AC
:10970000DC014D905D906D907C90139714968D9038
:109710009D90AD90BC90179718968D919D910D904E
:10972000BC91A02D89839A83AB83BC83A301920152
:10973000C301B2010F94DB606B017C01A5019401B0
:10974000C501B4010F94DB609B01AC01C701B601F8
:109750000F9445676B017C0129813A814B815C81C3
:10976000CA01B9010F94DB609B01AC01C701B601CE
:109770000F9445670F94436A9B01AC0160E070E071
:1097800080E89FE30F943F686B017C01AC019B0173
:10979000C301B2010F94DB60ED81FE8160837183B0
:1097A00082839383A7019601C501B4010F94DB6006
:1097B000AD81BE8114966D937D938D939C93179785
:1097C000A701960169817A818B819C810F94DB606E
:1097D000ED81FE81608771878287938726960FB619
:1097E000F894DEBF0FBECDBFDF91CF91FF90EF9019
:1097F000DF90CF90BF90AF909F908F907F906F90B1
:109800005F904F9008950F931F9380919B16813026
:1098100019F50F9426380091B6091091B7092091D7
:10982000B8093091B909601B710B820B930B28EEBC
:1098300033E040E050E00F94B9666091BA0970914E
:10984000BB098091BC099091BD09620F731F841FF1
:10985000951F1F910F9108956091BE097091BF09E6
:109860008091C0099091C109D6CF10929B16109299
:10987000B6091092B7091092B8091092B90910925E
:10988000BE091092BF091092C0091092C10910922E
:10989000BA091092BB091092BC091092BD09089533
:1098A0008F929F92AF92BF92CF92DF92EF92FF92F0
:1098B0000F931F93CF93DF93CDB7DEB72C970FB6DF
:1098C000F894DEBF0FBECDBF8B0140E050E068E4EE
:1098D00072E44D835E836F83788740E050E060EAF6
:1098E00070E449875A876B877C878130B9F1823071
:1098F00009F459C020E030E040E050E46091670294
:10990000709168028091690290916A020F94456794
:109910004B017C0120E030E048EC53E40F94A56952
:10992000181634F4812C912C88ECE82E93E4F92E4F
:10993000F801A084B184C284D3849401A701B50145
:10994000C6010F94A569181614F054016701C501EA
:10995000D60189839A83AB83BC8348C0BE01675F0D
:109960007F4FC80108960E943746B8016C5F7F4F51
:10997000AE014B5F5F4FC8010E9415460E946F49C0
:109980002C960FB6F894DEBF0FBECDBFDF91CF91FE
:109990001F910F91FF90EF90DF90CF90BF90AF900D
:1099A0009F908F900895F8012085318542855385D9
:1099B00060916702709168028091690290916A02D9
:1099C0000F9445676B017C0120E030E048EC53E4E4
:1099D0000F94756087FD06C0C12CD12C28ECE22EB7
:1099E00023E4F22EC982DA82EB82FC82BE01675F39
:1099F0007F4FCE010196B7CF4F925F926F927F92C9
:109A00008F929F92AF92BF92CF92DF92EF92FF928E
:109A1000CF93DF93CDB7DEB76E970FB6F894DEBF66
:109A20000FBECDBF9E8F8D8FFC01C4A8D5A8E6A820
:109A3000F7A820E030E0A901C701B6010F947560D6
:109A4000882309F497C1A701960160E070E080E8DF
:109A50009FE30F943F686B017C01ED8DFE8D2081AB
:109A60003181428153810F94DB606D837E838F83CC
:109A70009887ED8DFE8D2481358146815781C70100
:109A8000B6010F94DB602B013C01ED8DFE8D24852A
:109A9000358546855785C701B6010F94DB604B01BC
:109AA0005C012D813E814F815885CA01B9010F9417
:109AB000DB609B01AC01C501B4010F944467698B65
:109AC0007A8B8B8B9C8BED8DFE8D20893189428921
:109AD0005389C701B6010F94DB604B015C01A30100
:109AE0009201C301B2010F94DB609B01AC01C5017F
:109AF000B4010F9444676D8B7E8B8F8B988FED8DA7
:109B0000FE8D2489358946895789C701B6010F948E
:109B1000DB604B015C01A30192016D817E818F812D
:109B200098850F94DB609B01AC01C501B4010F94D3
:109B3000446769837A838B839C832D893E894F890F
:109B4000588D69897A898B899C890F94DB604B01D8
:109B50005C0129813A814B815C81CA01B9010F9472
:109B6000DB609B01AC01C501B4010F9444676987B8
:109B70007A878B879C8720E030E0A9010F94A56944
:109B800089849A84AB84BC8487FF04C0B7FAB094FC
:109B9000B7F8B094ED8DFE8D24A135A146A157A153
:109BA00060A171A182A193A10F9445672FEF36EEBA
:109BB0004BED5EE20F94DB60A50194010F94A56963
:109BC00087FFD8C0ED8DFE8D208531854285538578
:109BD000C701B6010F94DB606D877E878F87988BF6
:109BE000ED8DFE8D248D358D468D578DC701B601C7
:109BF0000F94DB604B015C012D853E854F855889B4
:109C0000C301B2010F94DB609B01AC01C501B4013B
:109C10000F9444674B015C01ED8DFE8D208D318DDD
:109C2000428D538DC701B6010F94DB606B017C013F
:109C30002D853E854F8558896D817E818F819885E0
:109C40000F94DB609B01AC01C701B6010F94446720
:109C5000698F7A8F8B8F9C8FA501940169817A819E
:109C60008B819C810F94DB606B017C01298D3A8D87
:109C70004B8D5C8D6D897E898F89988D0F94DB600B
:109C80009B01AC01C701B6010F94446729853A8551
:109C90004B855C850F943F686B017C01ED8DFE8DDB
:109CA000C0A6D1A6E2A6F3A6298D3A8D4B8D5C8D78
:109CB00069817A818B819C810F94DB6069837A83CF
:109CC0008B839C83A501940169897A898B899C89FE
:109CD0000F94DB609B01AC0169817A818B819C814F
:109CE0000F94446729853A854B855C850F943F68BE
:109CF0004B015C01ED8DFE8D84A695A6A6A6B7A6A8
:109D00002D813E814F815885C701B6010F94DB60DC
:109D10002D853E854F8558890F9445676B017C01E1
:109D2000A3019201C501B4010F94DB609B01AC015A
:109D3000C701B6010F9445679058ED8DFE8D60AB5D
:109D400071AB82AB93AB90E080E06E960FB6F89467
:109D5000DEBF0FBECDBFDF91CF91FF90EF90DF90C0
:109D6000CF90BF90AF909F908F907F906F905F90BB
:109D70004F90089581E090E0E8CFCF93DF93EC011E
:109D80008991882319F00E94059EFACFDF91CF9127
:109D90000895AF92BF92CF92DF92EF92FF920F930E
:109DA0001F93CF93DF93CDB7DEB7E6970FB6F89446
:109DB000DEBF0FBECDBF00918D0910918E09F80155
:109DC00001900020E9F731976F01C01AD10AF8011C
:109DD000CF01801B910B8C159D053CF481918F3236
:109DE000B9F7DF0111971C92F3CF8BE1EAEDF9E1AE
:109DF000DE015C9601900D928A95E1F7F12CE12C41
:109E0000EC14FD040CF05DC0F801EE0DFF1D808127
:109E1000811103C08FEFE81AF80A5801AE0CBF1C7D
:109E2000F5018081882309F44CC0FFEFEF1AFF0A87
:109E3000F801EE0DFF1D7F01E01AF10A81918111F9
:109E4000FACFCE014C960E944EEB8BE1FE017C9640
:109E5000DE01119601900D928A95E1F7B501CE01D0
:109E600001960E9468E3CE0101960E94B28D8FE2B6
:109E70000E94059E8091161781113BC082EA98E0EE
:109E80000E94BD4E8091BA1984FF1BC019821C82AA
:109E900021E0A501BE01645E7F4FCE0101960E94C4
:109EA00090ED811129C08AE00E94059E0E94CEB8E3
:109EB000B50185EA9BE00E940EACCE0101960E949E
:109EC000B28D8AE00E94059ECE014C960E94B28D12
:109ED000E6960FB6F894DEBF0FBECDBFDF91CF91EF
:109EE0001F910F91FF90EF90DF90CF90BF90AF90B8
:109EF000089586E197E1C4CFCE014C960E94BDEA59
:109F00008BE1FE013196DE015C9601900D928A95FF
:109F1000E1F7CE0101960E94B28D72CFCF92DF920F
:109F2000EF92FF92CF93DF93C62FFC01C080D180C8
:109F3000E280F38020E030E0A901C701B6010F9470
:109F4000756020E030E0A90187FD14C020E030E01A
:109F500048EC52E4C701B6010F94A56924E630E04D
:109F600040E050E0181634F0C701B6010F94B16814
:109F70009B01AC01C230A0F4D0E0C05DD14FAFEF87
:109F8000B0E00F94FA6624E630E040E050E00F9431
:109F9000DB662F3F310519F010F02FEF30E02883FA
:109FA000DF91CF91FF90EF90DF90CF900895E1E1A6
:109FB000FBE0108211821282138214820D943238D7
:109FC000EF92FF920F931F93CF93DF93CDB7DEB73E
:109FD0008C01EDB6FEB60F94C25F01962DB73EB769
:109FE000281B390B0FB6F8943EBF0FBE2DBF8DB79F
:109FF0009EB70196B8010F94BB5F0F946A350FB6F8
:10A00000F894FEBE0FBEEDBEDF91CF911F910F9170
:10A01000FF90EF9008958091090180FD06C0809126
:10A02000BA1983FB882780F9089580E00895CF92BC
:10A03000DF92EF92FF92FC01C080D180E280F3803A
:10A04000663019F51092160B1092170B1092180B20
:10A050001092190B10921A0B0E945DF520E030E06F
:10A06000A901C701B6010F94756087FF1DC0C12CFF
:10A07000D12C7601C701B6010F94B269CB01FF90D4
:10A08000EF90DF90CF900C947F8D0E94D74F20E00F
:10A0900030E0A901C701B6010F94756087FF15C0B4
:10A0A000C12CD12C760121C020E030E04CE053E4FB
:10A0B000C701B6010F94A5691816E4F6C12CD12C7E
:10A0C0009CE0E92E93E4F92ED5CF20E030E046E97C
:10A0D00053E4C701B6010F94A569181634F4C12CD6
:10A0E000D12C86E9E82E83E4F82EC701B6010F943F
:10A0F000B269CB01FF90EF90DF90CF900C94423487
:10A100009091AF11977081E0973009F080E0089549
:10A110002091830920FF14C020E83EE3629FA00144
:10A12000639F500D729F500D1124CA01969587951B
:10A1300096958795009731F08A950000E9F7089584
:10A140000C9450990895CF93DF9310926E11109252
:10A15000011210920312109202121092960910929C
:10A160009509CFEFDFEF8091BA1985FD07C00E94F6
:10A1700069E2D0933918C0933818F5CF8FEF9FEF6D
:10A180009093391880933818DF91CF9108958F926A
:10A190009F92AF92BF92CF92DF92EF92FF920F9376
:10A1A0001F93CF93DF937C0121E5E20EF11CD701D1
:10A1B0004C914A3509F0A4C06C01B2E5CB0ED11C1C
:10A1C000F6013081353A09F09BC0EC01C05BDF4FEE
:10A1D0002881233008F494C08C0100561F4FD80109
:10A1E0004C93E15BFF4F308331962083EF54F109AC
:10A1F0003081E05BFF4F30833038B1F43196AC549E
:10A20000B1093C913083E854F109AF5ABF4F50E097
:10A2100040E02250330B42175307CCF48081329632
:10A220008D934F5F5F4FF7CF233031F5313809F011
:10A2300074C0FC01EC55FF4FDC01AC5ABF4F2C91B0
:10A2400020833196885A9F4FDC018C91808348018E
:10A25000B12CA12C888190E002968A159B050CF404
:10A260003FC0F40181914F010E94969C0F94F31A14
:10A27000FFEFAF1ABF0AEECF323821F5FC01EC5ADE
:10A28000FF4F30814181E05BFF4F40833196308347
:10A29000DC01AA55BF4F50E040E02350330B42177A
:10A2A0005307ACF6FA01EE7FE45AFF4FE80FF91FAF
:10A2B000608171817C9311966C9311974E5F5F4F13
:10A2C0001296EDCF243019F6333809F6FC01EC5A1A
:10A2D000FF4F20813181E05BFF4F30833196B0CF5B
:10A2E00080E5DE011D928A95E9F78AE1F801119275
:10A2F0008A95E9F78AE5D7018C9385EAF601808390
:10A30000DF91CF911F910F91FF90EF90DF90CF9051
:10A31000BF90AF909F908F900895323809F097CFFB
:10A32000ADCFCF93DF93D0919B168AED90E10E9441
:10A33000909E8AE00E94059E80911A12873009F44F
:10A3400049C083E08093181281E080937C0280E111
:10A3500090E0909351198093501985E080934419AF
:10A36000C2E8C093471984E190E1A0E0B0E0809397
:10A37000481990934919A0934A19B0934B1984EF47
:10A3800098E10E94C75061E070E080E090E00E9498
:10A39000885081E09AE5909351198093501985E394
:10A3A00090E0909353198093521987E08093441959
:10A3B000C093471984E890E0A0E0B0E0809348198A
:10A3C00090934919A0934A19B0934B1984EF98E1DF
:10A3D0000E94C75080919B16813089F1823061F5CF
:10A3E0000E94034C6093BA097093BB098093BC0927
:10A3F0009093BD0981E080939B160F94263860935B
:10A40000B6097093B7098093B8099093B909D2300F
:10A4100089F08091930B9091940B01969093940BFB
:10A420008093930B109285091092860910928709E8
:10A430001092880981E004C00E94354CDBCF80E097
:10A44000DF91CF9108950F948D1E1092AE1110924E
:10A450003E020E945C9A882351F08091BA1982FDD5
:10A4600006C085E09DE09093FE118093FD1161E0B0
:10A470008EEF9CE00E94EBA10C94915180919B1671
:10A480008130C1F58AE19DE00E94909E8AE00E94A1
:10A49000059E81E09AE5909351198093501987E5C4
:10A4A00090E0909353198093521987E08093441958
:10A4B00082E88093471984E890E0A0E0B0E08093C0
:10A4C000481990934919A0934A19B0934B1984EFF6
:10A4D00098E10E94C75082E080939B160F94263823
:10A4E0006093BE097093BF098093C0099093C1091E
:10A4F00081E0089580E008950F931F930F9426380C
:10A5000000918E0B10918F0B2091900B3091910B3D
:10A51000011511052105310509F067C020912618A4
:10A52000222309F45FC0E0912418215020932618BB
:10A5300021E02E0F2093241830912718231302C0F6
:10A540001092241824E0E29FF0011124E85DF74EF8
:10A55000008111812281338100938A0B10938B0B30
:10A5600020938C0B30938D0B600F711F811D911DFB
:10A5700060938E0B70938F0B8093900B9093910B45
:10A5800080918C0B90918D0B892B61F11FB7F89402
:10A5900089E09DE00E94909E8AE00E94059E84E0F2
:10A5A00096E0909351198093501980EA90E8909327
:10A5B00053198093521987E08093441982E880935D
:10A5C000471980EA90E0A0E0B0E0809348199093AA
:10A5D0004919A0934A19B0934B1984EF98E10E944E
:10A5E000C7501FBF1F910F910895601B710B820B05
:10A5F000930B97FDF7CF409810928E0B10928F0B14
:10A600001092900B1092910BEDCF0F931F93CF935D
:10A61000DF938C01EB01909126182091271892135B
:10A6200005C00E947C520E94D7F8F5CF8091251872
:10A6300034E0839FF0011124E85DF74E118300831D
:10A64000D383C2839F5F909326188F5F281739F0BA
:10A6500080932518DF91CF911F910F91089510924B
:10A660002518F8CF2F923F924F925F926F927F9270
:10A670008F929F92AF92BF92CF92DF92EF92FF9212
:10A680000F931F93CF93DF93009709F0AAC1109205
:10A690000312109202129093960980939509BAE0E2
:10A6A000CB2EB0E2DB2EE12CF12C15E002E84601C6
:10A6B0005701C4E1D0E010929718109296181093A9
:10A6C0008A1800938D1880928E1890928F18A092FD
:10A6D0009018B09291188AE398E10E94C750219790
:10A6E0002FEF821A920AA20AB20A209721F744E1B8
:10A6F000C40ED11CE11CF11C8AE5C81680E2D80604
:10A70000E104F104A1F6C12CA0E2DA2EE12CF12C37
:10A71000D5E0C2E81092971810929618D0938A1834
:10A72000C0938D18C0928E18D0928F18E092901816
:10A73000F09291188AE398E10E94C75010929718FE
:10A7400010929618D0938A18C0938D18D701C6011D
:10A750008C529F4FAF4FBF4F80938E1890938F189E
:10A76000A0939018B09391188AE398E10E94C75083
:10A77000EFEFCE1ADE0AEE0AFE0AFAE0CF16F0E29A
:10A78000DF06E104F10431F6FEEDCF2EF0E2DF2E1C
:10A79000E12CF12CD5E0C2E810929718109296188F
:10A7A000D0938A18C0938D18C0928E18D0928F18AB
:10A7B000E0929018F09291188AE398E10E94C750B5
:10A7C0002FEFC21AD20AE20AF20A46EEC41640E29B
:10A7D000D406E104F10401F7CC24C394E2E1DE2EB7
:10A7E000E12CF12C0AE010E0D5E0C2E810939718B4
:10A7F00000939618D0938A18C0938D18C0928E1823
:10A80000D0928F18E0929018F09291188AE398E114
:10A810000E94C7501093971800939618D0938A18E7
:10A82000C0938D18D701C6018096A11DB11D8093DC
:10A830008E1890938F18A0939018B09391188AE374
:10A8400098E10E94C7508FEFC81AD80AE80AF80AA0
:10A85000E5E0CE16E2E1DE06E104F10439F600910E
:10A860000212109103120115110509F0D6C0809152
:10A870000112882309F4E1C02AE030E240E050E010
:10A8800066EA78E08AE398E10F94F81AC1E0D0E034
:10A8900003E010E0E0900212F090031235E0332E56
:10A8A00042E8242E44244A94542C64E0662E712CF1
:10A8B0007FE1C72E74E0D72E80910212909103128F
:10A8C000800F911FE816F90608F0D5C0C7010F9454
:10A8D0000F1C882309F481C08091161769E077E185
:10A8E000882311F066E177E1FB0101900020E9F790
:10A8F000CF010197861B970BF4E1FC9F9001FD9F10
:10A90000300D1124265F3F4D50E040E0459710F098
:10A91000FB01128A8AE398E10F94F81ACE018F5F47
:10A920009D4EB0E0A0E021964E0124E0880C991CD9
:10A930002A95E1F7FDEF8F1AFFE99F0AB12CA12CB0
:10A940002091BA1924FF7EC07092971860929618D1
:10A9500030928A1820928D1880938E1890938F18B9
:10A96000A0939018B09391188AE398E10E94C75081
:10A97000D0929718C092961830928A1820928D180B
:10A9800080928E1890928F18A0929018B092911881
:10A990008AE398E10E94C750B70186EC9CE00E94D0
:10A9A00078A48091161766E177E1811102C069E011
:10A9B00077E183EC9CE00E940EAC6EE671E18FEBD8
:10A9C0009CE00E940EAC69E077E18EEB9CE00E9477
:10A9D0000EAC8AEB9CE00E94909E2FEFE21AF20AE6
:10A9E0006BCF2091021230910312A90141505109FD
:10A9F00060919509709196096817790738F42C5F72
:10AA00003F4F309303122093021245CE443051053C
:10AA100008F43DCE24503109F4CF0430110569F417
:10AA200080910112882331F083E090E0909303122B
:10AA300080930212D0E0C0E02DCFD0E0C0E004E06F
:10AA400010E028CF109297181092961830928A181A
:10AA500020928D1880938E1890938F18A093901841
:10AA6000B09391188AE398E10E94C75050929718CA
:10AA70004092961881CFDF91CF911F910F91FF9057
:10AA8000EF90DF90CF90BF90AF909F908F907F908E
:10AA90006F905F904F903F902F900895AF92BF922C
:10AAA000CF92DF92EF92FF920F931F93CF93DF939A
:10AAB000EC0184E6C82E80E2D82EE12CF12C02E8CD
:10AAC000A12C90E2B92E15E000934719C0924819C5
:10AAD000D0924919E0924A19F0924B19B09251194B
:10AAE000A09250191093441984EF98E10E94C75026
:10AAF0008FEFC81AD80AE80AF80A88E7C81680E271
:10AB0000D806E104F10401F724E630E240E050E029
:10AB1000BE0184EF98E1DF91CF911F910F91FF90DB
:10AB2000EF90DF90CF90BF90AF900D94F81ACF9335
:10AB3000DF93CDB7DEB78E819091DC16891788F050
:10AB40008093DC169E01275F3F4F4F8158856FE34E
:10AB500070E08CE996E10F943C608CE996E10E94EC
:10AB60004E55DF91CF9108950F931F93CF93DF93AD
:10AB70008C016F3F19F41092DC1660E02091DC1616
:10AB8000862F062E000C990B2817190609F08CF554
:10AB90006093DC1660E088EC9CE00E94EBA1C801A9
:10ABA0000E94909E8AE00E94059EC8010F94C25F99
:10ABB000800F911FEC01C01BD10BC034D1053CF0BC
:10ABC0000197FC012491207C2038D1F3F3CFDD27BD
:10ABD000AE01B8018CE996E10F94E35FC456D94EFB
:10ABE00018828CE996E1DF91CF911F910F910C941F
:10ABF0004E55DF91CF911F910F910895CF92DF9223
:10AC0000EF92FF920F931F93CF93DF93CDB7DEB7F1
:10AC1000CA5AD1090FB6F894DEBF0FBECDBFCF55CB
:10AC2000DF4F188219821A821B82C15AD04080914C
:10AC3000B3089091B408A091B508B091B608CB556F
:10AC4000DF4F88839983AA83BB83C55AD04084E6AB
:10AC500090E09093D20A8093D10A1092E30A109266
:10AC6000E20A1092E40A22EE3AE044E050E0BE012B
:10AC70006B557F4F81ED9AE00E94C4BA8091D10A52
:10AC80009091D20A02969093D20A8093D10A1092A0
:10AC9000E30A1092E20A81E0C655DF4F8883CA5A60
:10ACA000D040CE0186559F4F0F94380A22EE3AE0ED
:10ACB00048E450E065EB71E181ED9AE00E94C4BA8E
:10ACC00022EE3AE040E150E06CE17EE081ED9AE076
:10ACD0000E94C4BA8AE097EDA3EABCE3CF55DF4FE8
:10ACE00088839983AA83BB83C15AD040CE018F55F4
:10ACF0009F4F0F942F0A8DE39DE00F944A0A80E244
:10AD000092E00F94410A8CE192E00F942F0A809117
:10AD1000280D9091290DA0912A0DB0912B0D8983BA
:10AD20009A83AB83BC838E010F5F1F4FC8010F94C2
:10AD30002F0ACF55DF4F188219821A821B82C15AFF
:10AD4000D0407E018DE6E80EF11C83E0D7018C93A4
:10AD50008983CE018F559F4F0F942F0AC7010F94FF
:10AD6000380AC8010F94380A4AE0D42EDA94DD205C
:10AD700031F0CE018F559F4F0F942F0AF7CF81EFFF
:10AD800097E10F944A0ACF55DF4F188219821A8231
:10AD90001B82C15AD0403AE0D32EDA94DD2031F044
:10ADA000CE018F559F4F0F942F0AF7CF88E0F70100
:10ADB000982F11929A95E9F7D8011D928A95E9F793
:10ADC00083E0C755DF4F8883C95AD040C356DF4F51
:10ADD0008883CD59D040CE0187559F4F0F94380AB4
:10ADE000CE0183569F4F0F94380A22EE3AE048E096
:10ADF00050E0B80181ED9AE00E94C4BA22EE3AE038
:10AE000048E050E0B70181ED9AE00E94C4BACF5506
:10AE1000DF4F188219821A821B82C15AD0402AE061
:10AE2000C22ED12CB1E0CB1AD10831F0CE018F5512
:10AE30009F4F0F942F0AF6CF8091B0118983809194
:10AE4000DC0AF7018083C8010F94410AC7010F94FF
:10AE5000380A22EE3AE044E050E06CED72E081ED19
:10AE60009AE00E94C4BA8091A70B8983C8010F940D
:10AE7000410A198A1A8A1B8A1C8A80E090E0A0E89D
:10AE8000BFE38D879E87AF87B88B809167179091BE
:10AE90006817A0916917B0916A1789839A83AB8369
:10AEA000BC832CEA35EC47E25EE360916B1770914E
:10AEB0006C1780916D1790916E170F943F686D839A
:10AEC0007E838F8398872CEA35EC47E25EE36091BE
:10AED0006F177091701780917117909172170F947E
:10AEE000DB6069877A878B879C8722EE3AE044E1B2
:10AEF00050E0B80181ED9AE00E94C4BA84E190E08C
:10AF00009A838983C8010F941D0A8091FC16909141
:10AF1000FD16A091FE16B091FF1689839A83AB832C
:10AF2000BC832CEA35EC47E25EE360910017709138
:10AF3000011780910217909103170F943F686D835A
:10AF40007E838F8398872CEA35EC47E25EE360913D
:10AF500004177091051780910617909107170F94A9
:10AF6000DB6069877A878B879C87C8010F94260AE4
:10AF70008CE0E5E9F2E0D80101900D928A95E1F7C5
:10AF8000C8010F94260A1982C8010F94380A8FE766
:10AF900090E09A838983C8010F941D0A85E0E1EA55
:10AFA000F2E0D80101900D928A95E1F722EE3AE0A5
:10AFB00045E050E0B80181ED9AE00E94C4BA80916A
:10AFC000DB0A8983C8010F94410A80E2E6EAF2E0D5
:10AFD000D80101900D928A95E1F722EE3AE040E225
:10AFE00050E0B80181ED9AE00E94C4BAD7011C92EA
:10AFF000C7010F94410A80E39DE00F94410A8CE25F
:10B000009DE00F942F0ACF55DF4F188219821A82C4
:10B010001B82C15AD040CE018F559F4F0F942F0AEB
:10B0200080E2F80111928A95E9F722EE3AE040E2D7
:10B0300050E0B80181ED9AE00E94C4BAFE01F99691
:10B0400088E0DF011D928A95E9F744E650E060E070
:10B0500070E049835A836B837C834D835E836F8367
:10B06000788783E090E0A0E0B0E089879A87AB879B
:10B07000BC874D875E876F87788B498B5A8B6B8B2C
:10B080007C8B8D8B9E8BAF8BB88F898F9A8FAB8F7C
:10B09000BC8F8D8F9E8FAF8FB8A38EE190E0A0E024
:10B0A000B0E089A39AA3ABA3BCA38DA39EA3AFA337
:10B0B000B8A789A79AA7ABA7BCA78DA79EA7AFA73C
:10B0C000B8AB89AB9AABABABBCAB8DAB9EABAFAB0C
:10B0D000B8AF22EE3AE040E450E0B80181ED9AE0EA
:10B0E0000E94C4BA80E1D82EF8018D2D11928A9564
:10B0F000E9F722EE3AE040E150E0B80181ED9AE054
:10B100000E94C4BAD8011D92DA94E9F722EE3AE01F
:10B1100040E150E0B80181ED9AE00E94C4BA8CE2AF
:10B120009EE00F942F0A9CE0D92EF8018D2D1192EC
:10B130008A95E9F722EE3AE04CE050E0B80181ED63
:10B140009AE00E94C4BA8CE6D8011D928A95E9F76C
:10B1500022EE3AE04CE650E0B80181ED9AE00E9420
:10B16000C4BA82EC99E00F94260A22EE3AE048E055
:10B1700050E063ED7AE081ED9AE00E94C4BAF701F5
:10B180001192DA94E9F7C755DF4F1882C95AD040B7
:10B1900080E090E0A0E4B0E4C356DF4F8883998359
:10B1A000AA83BB83CD59D040C7010F944A0ACE0170
:10B1B00087559F4F0F94380ACE0183569F4F0F94A7
:10B1C0002F0A80E3D7011D928A95E9F78AE091E181
:10B1D0000E94909E8AE00E94059E22EE3AE040E3A3
:10B1E00050E0B70181ED9AE00E94C4BA8091E40A70
:10B1F000811128C00091D10A1091D20A8091E20AEF
:10B200009091E30AF7019183808384E690E0909324
:10B21000D20A8093D10A22EE3AE044E050E063E0A3
:10B2200078E081ED9AE00E94C4BAC7010F941D0A2C
:10B2300091E00532134009F490E08091E40A892BF3
:10B240008093E40A8091DC0A87FF0F94410C80917F
:10B25000E40A811105C060E08EE391E10E94B455DB
:10B260008EE191E10E94909E8AE00E94059E90915D
:10B27000E40A81E08927C655DF4F0FB6F894DEBF98
:10B280000FBECDBFDF91CF911F910F91FF90EF9037
:10B29000DF90CF9008951092AE1110923E028091EF
:10B2A000BA1980648093BA1961E086ED9CE00E942F
:10B2B000EBA14BEE5CE063EF7CE085E00F94121DA8
:10B2C00060E08DED9CE00C94B455CF92DF92EF924C
:10B2D000FF920F931F93CF93DF93CDB7DEB77C011F
:10B2E000CDB6DEB60F94C25F01962DB73EB7281BD0
:10B2F000390B0FB6F8943EBF0FBE2DBF0DB71EB76A
:10B300000F5F1F4FB701C8010F94BB5FF801019099
:10B310000020E9F73197E01BF10B759720F086ECE0
:10B3200092E0F801848BC8010E944E550FB6F89444
:10B33000DEBE0FBECDBEDF91CF911F910F91FF906A
:10B34000EF90DF90CF900895CF93DF9300D01F92BE
:10B35000CDB7DEB78FE89CE00E94909E8AE00E9405
:10B36000059E80911A128330D9F119821A821B82AC
:10B370001C8260E0CE0101960E948E4F19821A82D3
:10B380001B821C8261E0CE0101960E948E4F81E0FB
:10B3900080937B021092171280937C0281E09AE5E1
:10B3A000909351198093501983E390E0909353192F
:10B3B0008093521987E08093441982E8809347195B
:10B3C00084E890E0A0E0B0E0809348199093491998
:10B3D000A0934A19B0934B1984EF98E10E94C7508B
:10B3E0000F900F900F900F90DF91CF910895CF9213
:10B3F000DF92EF92FF92CF93C82F80919B168150DE
:10B40000823008F069C00E94A45910929B160F94D4
:10B4100026386093BE097093BF098093C00990934A
:10B42000C109C0908509D0908609E0908709F09005
:10B4300088090E94034CAB01BC01409385095093DD
:10B44000860960938709709388098091970B909182
:10B45000980BA091990BB0919A0B8C199D09AE098C
:10B46000BF09840F951FA61FB71F8093970B90935A
:10B47000980BA093990BB0939A0BC1110AC0C1E02D
:10B480000E94B5338C2FCF91FF90EF90DF90CF903B
:10B4900008958091950B9091960B01969093960B41
:10B4A0008093950B0E94034CC0909B0BD0909C0BFB
:10B4B000E0909D0BF0909E0BC616D706E806F906A5
:10B4C000F0F60E94034C60939B0B70939C0B80934F
:10B4D0009D0B90939E0BD3CFC0E0D2CF8F929F92C3
:10B4E000AF92BF92CF92DF92EF92FF920F931F9392
:10B4F000CF93DF930E94A3503AE0C32E30E2D32EC5
:10B50000E12CF12C15E002E846015701CAE0D0E039
:10B510001092511910925019109344190093471921
:10B520008092481990924919A0924A19B0924B19E9
:10B5300084EF98E10E94C75021978FEF881A980AEC
:10B54000A80AB80A209721F78AE0C80ED11CE11C8E
:10B55000F11C82EDC81680E2D806E104F104A1F6E0
:10B56000C12C20E2D22EE12CF12CD5E0C2E81092C1
:10B57000511910925019D0934419C0934719C09291
:10B580004819D0924919E0924A19F0924B1984EF68
:10B5900098E10E94C7501092511910925019D093FF
:10B5A0004419C0934719D701C6018C529F4FAF4F22
:10B5B000BF4F8093481990934919A0934A19B093AB
:10B5C0004B1984EF98E10E94C7508FEFC81AD80A30
:10B5D000E80AF80A8AE0C81680E2D806E104F10415
:10B5E00031F69EEDC92E90E2D92EE12CF12CD5E05A
:10B5F000C2E81092511910925019D0934419C09377
:10B600004719C0924819D0924919E0924A19F0920C
:10B610004B1984EF98E10E94C7508FEFC81AD80ADF
:10B62000E80AF80A86EEC81680E2D806E104F104BA
:10B6300001F7CC24C39482E1D82EE12CF12C0AE04E
:10B6400010E0D5E0C2E81093511900935019D0933F
:10B650004419C0934719C0924819D0924919E092F1
:10B660004A19F0924B1984EF98E10E94C750109349
:10B67000511900935019D0934419C0934719D70119
:10B68000C6018096A11DB11D809348199093491958
:10B69000A0934A19B0934B1984EF98E10E94C750C8
:10B6A0008FEFC81AD80AE80AF80A85E1C81682E1BD
:10B6B000D806E104F10439F682E190E09093511943
:10B6C00080935019D0934419C093471984E190E1B5
:10B6D000A0E0B0E08093481990934919A0934A19CB
:10B6E000B0934B1984EF98E1DF91CF911F910F91A7
:10B6F000FF90EF90DF90CF90BF90AF909F908F9092
:10B700000C94C7504F925F926F927F928F929F924C
:10B71000AF92BF92CF92DF92EF92FF920F931F935F
:10B72000CF93DF9300D000D01F921F92CDB7DEB72A
:10B730008091810981110AC48091930990919409A3
:10B740009C012F5F3F4F30939409209393098E3EC5
:10B75000924008F4FBC38091621790916317909315
:10B7600051198093501905E00093441912E8109381
:10B77000471986E390E1A0E0B0E0809348199093E8
:10B780004919A0934A19B0934B1984EF98E10E948C
:10B79000C7508091F7169091F816909351198093A5
:10B7A000501900934419109347198CE390E1A0E0DD
:10B7B000B0E08093481990934919A0934A19B09327
:10B7C0004B1984EF98E10E94C750809164179091C3
:10B7D0006517909351198093501900934419109351
:10B7E000471984E390E1A0E0B0E08093481990937A
:10B7F0004919A0934A19B0934B1984EF98E10E941C
:10B80000C7508091F9169091FA1690935119809330
:10B81000501900934419109347198AE390E1A0E06E
:10B82000B0E08093481990934919A0934A19B093B6
:10B830004B1984EF98E10E94C75081E08093810901
:10B84000109294091092930980911A12882339F169
:10B850000E94D62F811123C0809192098F5F80931F
:10B86000920980919209853620F0109292091092E7
:10B870001A12E0911A12E150E73008F06AC00E2E59
:10B88000000CFF0B8827E85BF34A8F4F0D943C6751
:10B89000525CA15C6D5E995EDA5E125FA55C1092EF
:10B8A0009209DFCF0E948050882309F452C081E0C2
:10B8B00080937C0281E89CE00E94909E8AE00E9436
:10B8C000059E80E190E0909351198093501985E096
:10B8D0008093441912E81093471984E190E1A0E0A5
:10B8E000B0E08093481990934919A0934A19B093F6
:10B8F0004B1984EF98E10E94C75081E09AE590933C
:10B9000051198093501986E390E0909353198093D6
:10B91000521987E0809344191093471984E890E006
:10B92000A0E0B0E08093481990934919A0934A1978
:10B93000B0934B1984EF98E10E94C75010921A12ED
:10B9400008C00E948050882321F00E94D62F8823AF
:10B95000A9F380917C02882309F433C7809182097E
:10B960008111C0C284E096E09093511980935019E0
:10B9700080EA90E8909353198093521917E010933E
:10B98000441902E80093471980EA90E0A0E0B0E093
:10B990008093481990934919A0934A19B0934B1971
:10B9A00084EF98E10E94C7508091770290917802CD
:10B9B000A0917902B0917A020097A105B10509F032
:10B9C0003FC2109251191092501915E0109344196A
:10B9D000009347198AE890E1A0E0B0E0809348190D
:10B9E00090934919A0934A19B0934B1984EF98E1A9
:10B9F0000E94C75089E090E09093511980935019AC
:10BA000010934419009347198CE890E1A0E0B0E04E
:10BA10008093481990934919A0934A19B0934B19F0
:10BA200084EF98E10E94C75080917702909178024C
:10BA3000A0917902B0917A020097F1E0AF07B105C9
:10BA400008F441C2B0935119A0935019909353191F
:10BA50008093521987E08093441982E880934719B4
:10BA600088E890E1A0E0B0E08093481990934919EC
:10BA7000A0934A19B0934B1984EF98E10E94C750E4
:10BA80008091770290917802A0917902B0917A0228
:10BA9000BA2FA92F982F8827009721E0A207B10578
:10BAA00008F417C2B0935119A093501990935319E9
:10BAB0008093521987E08093441912E81093471934
:10BAC00081EA90E0A0E0B0E0809348199093491992
:10BAD000A0934A19B0934B1984EF98E10E94C75084
:10BAE0008091B011882309F4FAC183E090E090932B
:10BAF00051198093501985E0809344191093471988
:10BB000085E490E1A0E0B0E0809348199093491952
:10BB1000A0934A19B0934B1984EF98E10E94C75043
:10BB200080918209875E8093820920918209822F09
:10BB300090E0253608F021C2909351198093501956
:10BB400085E08093441982E88093471980E090E172
:10BB5000A0E0B0E08093481990934919A0934A1946
:10BB6000B0934B1984EF98E10E94C7500E94D62FE2
:10BB7000811114C20E945C9A811105C090918309C1
:10BB800091FD0E94D62F9091830980FB91F99093AB
:10BB9000830991FD03C28091BA1982FDFFC1809192
:10BBA0009B168150823008F4F9C16091F9167091AA
:10BBB000FA16072E000C880B990B0F947C606B0112
:10BBC0007C0120E030E0A9010F947560882309F41E
:10BBD000BBC66091F7167091F816072E000C880B03
:10BBE000990B0F947C602B013C0120E030E040E099
:10BBF00050E4C701B6010F944467A30192010F946A
:10BC0000A56918160CF4C2C660916217709163178B
:10BC1000072E000C880B990B0F947C606D837E833C
:10BC20008F8398876091641770916517072E000CB9
:10BC3000880B990B0F947C604B015C0120E030E095
:10BC400040E251E40F9444672D813E814F81588535
:10BC50000F94A56918160CF499C620E030E040E076
:10BC600050E4C701B6010F944567A30192010F94F8
:10BC7000756087FD10C020E030E040E251E4C5016E
:10BC8000B4010F9445672D813E814F8158850F94F3
:10BC9000756087FF6AC684E190E0909351198093A4
:10BCA000501985E08093441982E88093471984E114
:10BCB00090E1A0E0B0E08093481990934919A093D7
:10BCC0004A19B0934B1984EF98E10E94C7508091B4
:10BCD000181281117CC682E07AC683E79CE00E943C
:10BCE000909E8AE00E94059E81E09AE5909351190A
:10BCF0008093501980E490E09093531980935219E7
:10BD000017E01093441982E88093471984E890E083
:10BD1000A0E0B0E08093481990934919A0934A1984
:10BD2000B0934B1984EF98E10E94C75010931A12F8
:10BD300010CE80910712882309F40BCE0E94805008
:10BD4000882309F406CE0E94D62F811102CE85E603
:10BD50009CE00E94909E8AE00E94059E80910812BD
:10BD600090E0B0E0A0E0895B9F4FAE4FB54A21E084
:10BD70003AE53093511920935019909353198093B9
:10BD8000521987E08093441982E88093471984E828
:10BD900090E0A0E0B0E08093481990934919A093F7
:10BDA0004A19B0934B1984EF98E10E94C750109242
:10BDB0000712C4CD0E948050882309F4CACD0E9486
:10BDC000D62F8111C6CD81E080937C0210921A1289
:10BDD00087E59CE00E94909E8AE00E94059E81E09B
:10BDE0009AE590935119809350198EE490E09093C6
:10BDF00053198093521987E08093441982E8809305
:10BE0000471984E890E0A0E0B0E08093481990934F
:10BE10004919A0934A19B0934B1984EF98E10E94F5
:10BE2000C75097CD0E94D62F811193CD19821A82C7
:10BE30001B821C8262E0CE0101960F9478317ECD88
:10BE40000196A11DB11D35E0B695A79597958795EB
:10BE50003A95D1F70197A109B1090097E1E0AE0742
:10BE6000B10548F1B0935119A0935019909353190B
:10BE7000809352191093441912E8109347198AE8D5
:10BE800090E1A0E0B0E08093481990934919A09305
:10BE90004A19B0934B1984EF98E10E94C75088E08B
:10BEA00090E0909351198093501985E08093441944
:10BEB00010934719A9CD909351198093501985E09B
:10BEC00080934419D9CF909351198093501985E0EC
:10BED000C2CD909351198093501985E0ECCD82E04A
:10BEE00090E005CE8A3F08F020CE8EEF8093820945
:10BEF00086E49CE00E94909E8AE00E94059E81E07C
:10BF000080937C0281E09AE59093511980935019B7
:10BF10008DE290E0909353198093521987E08093BB
:10BF2000441982E88093471984E890E0A0E0B0E0EB
:10BF30008093481990934919A0934A19B0934B19CB
:10BF400084EF98E10E94C7501092810928960FB69D
:10BF5000F894DEBF0FBECDBFDF91CF911F910F913F
:10BF6000FF90EF90DF90CF90BF90AF909F908F9019
:10BF70007F906F905F904F900895845691099093B1
:10BF800051198093501985E08093441982E8809379
:10BF9000471981E090E1A0E0B0E0DCCD8CE090E0DA
:10BFA000909351198093501915E01093441982E829
:10BFB0008093471984E190E1A0E0B0E080934819B4
:10BFC00090934919A0934A19B0934B1984EF98E1C3
:10BFD0000E94C7500E94034C20E13EE040E050E048
:10BFE0000F94B9662115310581E04807510508F421
:10BFF00070C05093511940935019309353192093A6
:10C00000521987E08093441912E81093471980E190
:10C0100090E1A0E0B0E08093481990934919A09373
:10C020004A19B0934B1984EF98E10E94C7500E94BF
:10C03000034C20E13EE040E050E00F94B9662CE371
:10C0400030E040E050E00F94B966309351192093EE
:10C05000501905E0009344191093471982E190E1CB
:10C06000A0E0B0E08093481990934919A0934A1931
:10C07000B0934B1984EF98E10E94C7500E943E3262
:10C08000882309F45CC48F5F80939109E82EF12C1A
:10C09000833330F5EE0CFF1CF0925119E0925019E9
:10C0A00000934419109347198EE090E1A0E0B0E0AE
:10C0B0008093481990934919A0934A19B0934B194A
:10C0C00084EF98E10E94C7501092511910925019B4
:10C0D0002BC030935119209350191093441994CFC9
:10C0E00084E690E09093511980935019009344197D
:10C0F000109347198EE090E1A0E0B0E080934819DA
:10C1000090934919A0934A19B0934B1984EF98E181
:10C110000E94C750A2E3EA1AA0E8FA0AEE0CFF1C3C
:10C12000F0925119E0925019009344191093471955
:10C130008FE090E1A0E0B0E0809348199093491916
:10C14000A0934A19B0934B1984EF98E10E94C7500D
:10C150000E943E3290E0909351198093501985E0EF
:10C160008093441982E88093471986E190E1A0E02A
:10C17000B0E08093481990934919A0934A19B0935D
:10C180004B1984EF98E10E94C75020E030E0A901EC
:10C190006091F9177091FA178091FB179091FC1735
:10C1A0000F94456720E030E048EC52E40F94DB60E8
:10C1B0000F94B168709351196093501905E0009382
:10C1C000441912E81093471986E290E1A0E0B0E02C
:10C1D0008093481990934919A0934A19B0934B1929
:10C1E00084EF98E10E94C75080917302909174028D
:10C1F0009093511980935019009344191093471943
:10C2000080E093E1A0E0B0E0809348199093491951
:10C21000A0934A19B0934B1984EF98E10E94C7503C
:10C2200020E030E040E251E46091C9117091CA1100
:10C230008091CB119091CC110F94DB600F94B86872
:10C240007093511960935019009344191093471932
:10C2500082E492E1A0E0B0E08093481990934919FC
:10C26000A0934A19B0934B1984EF98E10E94C750EC
:10C2700020E030E040E251E46091CD117091CE11A8
:10C280008091CF119091D0110F94DB600F94B8681A
:10C2900070935119609350190093441910934719E2
:10C2A00086E492E1A0E0B0E08093481990934919A8
:10C2B000A0934A19B0934B1984EF98E10E94C7509C
:10C2C00020E030E040E251E46091D1117091D21150
:10C2D0008091D3119091D4110F94DB600F94B868C2
:10C2E0007093511960935019009344191093471992
:10C2F0008AE492E1A0E0B0E0809348199093491954
:10C30000A0934A19B0934B1984EF98E10E94C7504B
:10C3100020E030E040E251E46091D5117091D611F7
:10C320008091D7119091D8110F94DB600F94B86869
:10C330007093511960935019009344191093471941
:10C340008EE492E1A0E0B0E08093481990934919FF
:10C35000A0934A19B0934B1984EF98E10E94C750FB
:10C3600020E030E048EC52E46091F1177091F21750
:10C370008091F3179091F4170F94DB600F94B168DC
:10C3800070935119609350190093441910934719F1
:10C3900086E392E1A0E0B0E08093481990934919B8
:10C3A000A0934A19B0934B1984EF98E10E94C750AB
:10C3B00020E030E048EC52E46091F5177091F617F8
:10C3C0008091F7179091F8170F94DB600F94B16884
:10C3D00070935119609350190093441910934719A1
:10C3E0008AE392E1A0E0B0E0809348199093491964
:10C3F000A0934A19B0934B1984EF98E10E94C7505B
:10C4000080918302909184029093511980935019E6
:10C41000009344191093471982E592E1A0E0B0E03F
:10C420008093481990934919A0934A19B0934B19D6
:10C4300084EF98E10E94C75080918102909182021E
:10C4400090935119809350190093441910934719F0
:10C4500084E592E1A0E0B0E08093481990934919F7
:10C46000A0934A19B0934B1984EF98E10E94C750EA
:10C4700020E030E040E251E4609167177091681766
:10C480008091691790916A170F94DB600F94B868D8
:10C4900070935119609350190093441910934719E0
:10C4A00086E592E1A0E0B0E08093481990934919A5
:10C4B000A0934A19B0934B1984EF98E10E94C7509A
:10C4C0002CEA35EC47E25EE360916B1770916C17D4
:10C4D00080916D1790916E170F943F6820E030E0C7
:10C4E00040E251E40F94DB600F94B86870935119E7
:10C4F0006093501900934419109347198AE592E10B
:10C50000A0E0B0E08093481990934919A0934A198C
:10C51000B0934B1984EF98E10E94C7502CEA35EC98
:10C5200047E25EE360916F17709170178091711709
:10C53000909172170F94DB6020E030E040E251E40C
:10C540000F94DB600F94B868709351196093501981
:10C5500000934419109347198EE592E1A0E0B0E0F2
:10C560008093481990934919A0934A19B0934B1995
:10C5700084EF98E10E94C75020E030E040E251E4AF
:10C580006091FC167091FD168091FE169091FF1639
:10C590000F94DB600F94B868709351196093501931
:10C5A000009344191093471982E692E1A0E0B0E0AD
:10C5B0008093481990934919A0934A19B0934B1945
:10C5C00084EF98E10E94C7502CEA35EC47E25EE325
:10C5D00060910017709101178091021790910317D5
:10C5E0000F943F6820E030E040E251E40F94DB60BC
:10C5F0000F94B868709351196093501900934419BF
:10C600001093471986E692E1A0E0B0E080934819C4
:10C6100090934919A0934A19B0934B1984EF98E16C
:10C620000E94C7502CEA35EC47E25EE360910417A4
:10C630007091051780910617909107170F94DB6092
:10C6400020E030E040E251E40F94DB600F94B868E2
:10C65000709351196093501900934419109347191E
:10C660008AE692E1A0E0B0E08093481990934919DE
:10C67000A0934A19B0934B1984EF98E10E94C750D8
:10C6800080911112811105C080911312882309F441
:10C690006DC06091621770916317072E000C880BB4
:10C6A000990B0F947C6020E030E048EC52E40F944A
:10C6B000DB606B017C016091641770916517072E38
:10C6C000000C880B990B0F947C609B01AC01C70197
:10C6D000B6010F943F680F94B8686536710510F085
:10C6E00064E670E0709351196093501905E000936F
:10C6F000441912E81093471984E290E1A0E0B0E0F9
:10C700008093481990934919A0934A19B0934B19F3
:10C7100084EF98E10E94C75060916217709163178F
:10C72000072E000C880B990B0F947C606B017C0129
:10C7300020E030E04AE253E40F94A569181624F48F
:10C7400080911112811146C1609164177091651733
:10C75000072E000C880B990B0F947C609B01AC0199
:10C76000C701B6010F94A56987FFAFC18091071279
:10C77000882339F18091061291E0980F9093061268
:10C7800090E0909351198093501985E0809344195B
:10C7900082E88093471982E490E1A0E0B0E08093C2
:10C7A000481990934919A0934A19B0934B1984EFF3
:10C7B00098E10E94C750809106128A3010F01092C2
:10C7C00006120E940B50882309F4B5C16091FF1135
:10C7D00070910012EE24E394F12C61157105A9F01B
:10C7E00090E080E00F947A6020E030E040E85EE383
:10C7F0000F94DB600F94236820E030E040E85FE3B3
:10C800000F9445670F94B8687B0101E010E08091B8
:10C810000112811102C010E000E08091381890915F
:10C8200039188F3F980711F40E9453EB90933918F1
:10C8300080933818080F191FB80190E080E00F941A
:10C840007A6020E030E040E85EE30F94DB600F9414
:10C8500023684B015C01F0925119E092501905E0F8
:10C860000093441912E81093471980E193E1A0E086
:10C87000B0E08093481990934919A0934A19B09356
:10C880004B1984EF98E10E94C750C501B4010F9481
:10C89000B86870935119609350190093441910931C
:10C8A000471982E193E1A0E0B0E0809348199093AA
:10C8B0004919A0934A19B0934B1984EF98E10E944B
:10C8C000C75004E919E1AAE1FA2E80913F0990913D
:10C8D000400920918F0930919009891B8F7309F4C9
:10C8E00049C12A3131050CF0DBC190913F0980919B
:10C8F00040094FEF5FEF981749F0E82FF0E0E15C57
:10C90000F64F42818F5F8F7380934009F901EC5697
:10C91000F64E4083809194198A3509F0B3C162E0E4
:10C9200070E080E090E00E94885080918F099091A3
:10C93000900901969093900980938F09C6CF109229
:10C94000511910925019ACCB609164177091651712
:10C95000072E000C880B990B0F947C6020E030E0D0
:10C96000A9010F947560811134C98CE090E0909317
:10C9700051198093501985E08093441982E880937F
:10C98000471984E190E1A0E0B0E0F3CB8DE090E0C6
:10C99000909351198093501985E08093441982E84F
:10C9A0008093471984E190E1A0E0B0E080934819BA
:10C9B00090934919A0934A19B0934B1984EF98E1C9
:10C9C0000E94C75080911812811101C081E08093AC
:10C9D0001812DBCB1092111220E030E040E251E45B
:10C9E0006091091270910A1280910B1290910C12B1
:10C9F0000F94DB600F94B1687093511960935019D4
:10CA0000009344191093471984E590E1A0E0B0E049
:10CA10008093481990934919A0934A19B0934B19E0
:10CA200084EF98E10E94C75020E030E040E251E4FA
:10CA300060910D1270910E1280910F129091101250
:10CA40000F94DB600F94B168709351196093501983
:10CA5000009344191093471988E590E1A0E0B0E0F5
:10CA60008093481990934919A0934A19B0934B1990
:10CA700084EF98E10E94C75085E29CE00E94909E5E
:10CA80008AE00E94059E81E09AE590935119809377
:10CA9000501981E490E0909353198093521987E0E4
:10CAA000809344191093471984E890E0A0E0B0E027
:10CAB0008093481990934919A0934A19B0934B1940
:10CAC00084EF98E10E94C75051CE60911312662303
:10CAD00009F44CCE062E000C770B8CE09CE00E94F3
:10CAE000A3A48AE00E94059E1092131284E090E0B5
:10CAF000909351198093501985E08093441912E85E
:10CB0000109347198EE890E1A0E0B0E080934819B7
:10CB100090934919A0934A19B0934B1984EF98E167
:10CB20000E94C75081E09AE5909351198093501963
:10CB300083E590E0B0CF109251191092501905E0A2
:10CB40000093441912E81093471980E193E1A0E0A3
:10CB5000B0E08093481990934919A0934A19B09373
:10CB60004B1984EF98E10E94C7501092511910920E
:10CB7000501993CE121613060CF492C08091F81837
:10CB80009091F918A091FA18B091FB188C34E0E15B
:10CB90009E07A105B10509F4D7C98A349041A105C2
:10CBA000B10509F4D1C920E030E040E251E46091E0
:10CBB0005F027091600280916102909162020F9415
:10CBC000DB600F94B168709351196093501905E0C0
:10CBD0000093441912E81093471988E490E1A0E00B
:10CBE000B0E08093481990934919A0934A19B093E3
:10CBF0004B1984EF98E10E94C75020E030E040E2FA
:10CC000051E4609163027091640280916502909199
:10CC100066020F94DB600F94B168709351196093B2
:10CC2000501900934419109347198AE490E1A0E049
:10CC3000B0E08093481990934919A0934A19B09392
:10CC40004B1984EF98E10E94C75020E030E040E2A9
:10CC500051E460916702709168028091690290913D
:10CC60006A020F94DB600F94B1687093511960935E
:10CC7000501900934419109347198CE490E1A0E0F7
:10CC8000B0E056C9121613060CF01FCEF8012F2D76
:10CC900011922A95E9F71092900910928F0915CEFA
:10CCA0009091F51880919419981321C09091F618DD
:10CCB0008091951998131BC023303105C4F09091D1
:10CCC00096199093F418809197198093F7189330E0
:10CCD000D1F4982F9D7F9038B1F4909198199F349A
:10CCE00009F059C0909199199B3409F054C0E4E9B6
:10CCF000F9E18AE1DF011D928A95E9F71092900926
:10CD000010928F093BCF833809F045C08091981964
:10CD100090919919982789279827B0E0A0E08093EF
:10CD2000F8189093F918A093FA18B093FB18C090D4
:10CD30009A19D12CF12CE12CC092FC18D092FD183C
:10CD4000E092FE18F092FF182BE939E140E050E044
:10CD5000BA014C155D056E057F0508F04AC0DB0180
:10CD6000CA01B695A795979587950696880F991F3E
:10CD7000FC01EC50F74ED9018C9111969C918927BA
:10CD800098278927918380834E5F5F4F6F4F7F4F36
:10CD90002E5F3F4FDECF813861F58091981990E08A
:10CDA000B0E0A0E08093F8189093F918A093FA18D7
:10CDB000B093FB1880919919482F50E070E060E023
:10CDC0004093FC185093FD186093FE187093FF1861
:10CDD000AAE9B9E1E0E0F9E190E030E020E0821773
:10CDE000930739F04D9150E0419351932F5F3F4F9E
:10CDF000F6CFE4E9F9E18AE1DF011D928A95E9F7CE
:10CE00001092900910928F090F94D638B7CE6F9276
:10CE10007F928F929F92AF92BF92CF92DF92EF92CA
:10CE2000FF920F931F93CF93DF93CDB7DEB7649735
:10CE30000FB6F894DEBF0FBECDBF1092D000809128
:10CE4000D00082608093D0001092D50080E1809362
:10CE5000D4008091D10080618093D1008091D10075
:10CE600088608093D1008091D10080688093D10048
:10CE70008091D1008F7D8093D1008AE58093451900
:10CE80008093F51885EA809346198093F618E4E9B3
:10CE9000F9E18AE1DF011D928A95E9F78091161286
:10CEA000882309F473C283E090E090935119809332
:10CEB000501985E08093441982E8809347198FE1E7
:10CEC00090E1A0E0B0E08093481990934919A093B5
:10CED0004A19B0934B1984EF98E10E94C75084E639
:10CEE00090E0909351198093501905E000934419F4
:10CEF00012E81093471986E090E1A0E0B0E080933B
:10CF0000481990934919A0934A19B0934B1984EF8B
:10CF100098E10E94C7508BE090E090935119809364
:10CF20005019009344191093471980E092E1A0E052
:10CF3000B0E08093481990934919A0934A19B0938F
:10CF40004B1984EF98E10E94C7501092511910922A
:10CF50005019009344191093471984E390E1A0E01D
:10CF6000B0E08093481990934919A0934A19B0935F
:10CF70004B1984EF98E10E94C750109251191092FA
:10CF8000501900934419109347198AE390E1A0E0E7
:10CF9000B0E08093481990934919A0934A19B0932F
:10CFA0004B1984EF98E10E94C750809162179091CD
:10CFB000631790935119809350190093441910935B
:10CFC000471986E390E1A0E0B0E080934819909380
:10CFD0004919A0934A19B0934B1984EF98E10E9424
:10CFE000C7508091F7169091F8169093511980933D
:10CFF000501900934419109347198CE390E1A0E075
:10D00000B0E08093481990934919A0934A19B093BE
:10D010004B1984EF98E10E94C75082E090E0909312
:10D0200051198093501900934419109347198EE1B8
:10D0300090E1A0E0B0E08093481990934919A09343
:10D040004A19B0934B1984EF98E10E94C75081E0D0
:10D0500080937B0270E6C72E70E1D72EE12CF12C75
:10D0600010925119109250190093441910934719B6
:10D07000C0924819D0924919E0924A19F0924B197E
:10D0800084EF98E10E94C750BFEFCB1ADB0AEB0A8E
:10D09000FB0AE4E7CE16E0E1DE06E104F10401F765
:10D0A000CE0101967C0184E1D7011D928A95E9F7B2
:10D0B00081E08F9390E99F938F9398E69F938F934E
:10D0C0009F9387EB98E09F938F93FF92EF920F943B
:10D0D000206C20E630E140E050E064EC78E084EF42
:10D0E00098E10F94F81A2AE630E140E050E061ED53
:10D0F00078E084EF98E10F94F81A24E730E140E0FB
:10D1000050E0B70184EF98E10F94F81A2EE730E170
:10D1100040E050E06DED78E084EF98E10F94F81A6C
:10D1200010925119109250190093441910934719F5
:10D130008EE090E1A0E0B0E0809348199093491907
:10D14000A0934A19B0934B1984EF98E10E94C750FD
:10D1500010925119109250190093441910934719C5
:10D160008FE090E1A0E0B0E08093481990934919D6
:10D17000A0934A19B0934B1984EF98E10E94C750CD
:10D180000FB6F894DEBF0FBECDBF4AE0C42E40E21A
:10D19000D42EE12CF12C55E0752E62E8662E460166
:10D1A00057010AE010E01092511910925019709234
:10D1B0004419609247198092481990924919A09297
:10D1C0004A19B0924B1984EF98E10E94C750015060
:10D1D0001109FFEF8F1A9F0AAF0ABF0A0115110547
:10D1E00011F78AE0C80ED11CE11CF11C92EDC916A2
:10D1F00090E2D906E104F10491F6C12C30E2D32E7D
:10D20000E12CF12C05E012E81092511910925019FE
:10D210000093441910934719C0924819D0924919A4
:10D22000E0924A19F0924B1984EF98E10E94C7509E
:10D2300010925119109250190093441910934719E4
:10D24000D701C6018C529F4FAF4FBF4F80934819F3
:10D2500090934919A0934A19B0934B1984EF98E120
:10D260000E94C750AFEFCA1ADA0AEA0AFA0ABAE00D
:10D27000CB16B0E2DB06E104F10431F62EEDC22E4E
:10D2800020E2D22EE12CF12C05E012E81092511987
:10D29000109250190093441910934719C0924819DD
:10D2A000D0924919E0924A19F0924B1984EF98E113
:10D2B0000E94C750EFEFCE1ADE0AEE0AFE0AF6EE23
:10D2C000CF16F0E2DF06E104F10401F7CC24C394A9
:10D2D00082E1D82EE12CF12C9AE0A92EB12C05E0A8
:10D2E00012E8B0925119A09250190093441910936A
:10D2F0004719C0924819D0924919E0924A19F09200
:10D300004B1984EF98E10E94C750B0925119A09236
:10D3100050190093441910934719D701C6018096FC
:10D32000A11DB11D8093481990934919A0934A19E2
:10D33000B0934B1984EF98E10E94C7508FEFC81A41
:10D34000D80AE80AF80A95E1C91692E1D906E1047B
:10D35000F10439F685EF9BE00E94909E8AE00E94DE
:10D36000059E64960FB6F894DEBF0FBECDBFDF9169
:10D37000CF911F910F91FF90EF90DF90CF90BF90D2
:10D38000AF909F908F907F906F90089582E090E093
:10D390008CCD0E9407671092820981E080937C0205
:10D3A00087EA9CE00E94909E8AE00C94059EAB0167
:10D3B000BC014093B6195093B7196093B819709394
:10D3C000B9198EE19BE10C94FCE6CF93DF93DB016E
:10D3D000F9019C919130C1F0943080F094509C936D
:10D3E0008830D1F480819181009771F00197918309
:10D3F0008083480F591FEA01188206C08C3539F422
:10D400009C5F9C93943041F4DF91CF9108958B33CE
:10D4100039F781E08C93F8CF20813181B9016F5FBA
:10D420007F4F71836083420F531FEA01888380819D
:10D4300091818F3591056CF7E7CF0F931F9381E0B2
:10D440000091B6191091B7192091B8193091B919F6
:10D450004091B2195091B3196091B4197091B519F6
:10D46000041715072607370708F480E01F910F916E
:10D4700008954F925F926F927F928F929F92AF9298
:10D48000BF92CF92DF92EF92FF920F931F93CF93B1
:10D4900010928E0910928D092FE320938C0910921F
:10D4A0008B0910928A091092890910923A091092F8
:10D4B0003B0910923C0910923D099C01F9019081B1
:10D4C0002F5F3F4F9032D1F39E34C9F4818190EDAC
:10D4D000980F9A3020F08D3211F08B3281F4329611
:10D4E0009F012F5F3F4F808180538A3008F47EC0B8
:10D4F0009F012F5F3F4F8081803209F479C0F09304
:10D500008E0CE0938D0C8F010F5F1F4FC0816AE27C
:10D5100070E0C8010F94E66B009731F0FC01319781
:10D5200080818032E1F31182CD3429F0C43519F0C5
:10D53000C73409F04BC0F80180810F5F1F4F803264
:10D54000D1F380538A3008F041C0C0938C0990E039
:10D5500080E04AE0DF011196489F9001499F300D1D
:10D560001124C901C0972081820F911D27FD9A9532
:10D57000218130ED320F3A30E8F190938B0980939E
:10D580008A092E3261F4329630E04AE0DF013196AA
:10D590002C9150ED520F5A3078F1309389099D014A
:10D5A000D9012F5F3F4F4C914032D1F3CD34A1F5DB
:10D5B0008E31910539F030F58731910519F08C31B4
:10D5C000910551F5B0938E09A0938D09CF911F91CC
:10D5D0000F91FF90EF90DF90CF90BF90AF909F9012
:10D5E0008F907F906F905F904F900895F90178CF62
:10D5F000F9017ECFFD01AECF349F200D112430ED17
:10D60000320FC4CF8537910538F087379105D0F2B6
:10D61000803A23E09207B1F250918D0C70E060E007
:10D62000C12CD12C7601C394FD0131964C91442339
:10D6300009F492C04132A1F4CD3491F480329105C5
:10D6400079F4F0938E09E0938D0963E270E0CF01E5
:10D650000F94E66B009709F4B9CFFC011082B6CFA6
:10D6600041544A3108F073C0DF012D91203209F492
:10D6700059C030ED320F3A3008F465C02E3209F04F
:10D6800053C0218120532A3008F45DC030E020E0EF
:10D690006115710519F4BF0161507109A42FB0E043
:10D6A0002601370104C0440C551C661C771C4A95A2
:10D6B000D2F780903A0990903B09A0903C09B09035
:10D6C0003D0984289528A628B72880923A09909287
:10D6D0003B09A0923C09B0923D0921153105A9F101
:10D6E000251BA05EB64F2C9320812154DF012A31E7
:10D6F00008F49ACFDF012191222309F495CF30ED70
:10D70000320F3A30B8F333ED320F323098F32B3218
:10D7100089F39D012F5F3F4F4C91403209F084CF38
:10D72000D901F7CFFD01A0CF2D3219F02B3209F02E
:10D73000ADCF218130ED320F3A3028F02E3209F092
:10D74000A5CF22819FCF9F01A9CF20E0CACF61152D
:10D75000710551F6BD01C8CF70938E0960938D0994
:10D7600035CFCF93DF93EC018991882319F00E9484
:10D77000059EFACF8DE00E94059E8AE0DF91CF9151
:10D780000C94059EEF92FF920F931F93CF93DF931C
:10D79000CDB7DEB762970FB6F894DEBF0FBECDBF30
:10D7A0000E94283B882309F43FC047EF58E082FFDE
:10D7B00002C040EF58E027EF38E081FF02C022EFBF
:10D7C00038E080FD2EC087EF98E05F934F933F9342
:10D7D0002F939F938F9380EC9DE09F938F938E0167
:10D7E0000F5F1F4F1F930F930F940C600E94CEB8D2
:10D7F000C8010E94B16BC8010F94551E0FB6F89472
:10D80000DEBF0FBECDBF81E062960FB6F894DEBFDB
:10D810000FBECDBFDF91CF911F910F91FF90EF9081
:10D82000089584EF98E0D1CF80E0EECFCF9384E5E8
:10D830000E948A8FC0E08823D9F00E94EA8EC82F08
:10D840001816B4F40E94CEB88DE40E94059E809113
:10D850008A0990918B090F94091C6C2FCC0F770BC0
:10D8600085E195E00E94A3A48AE00E94059ECFEF87
:10D870008C2FCF9108953F924F925F926F927F923B
:10D880008F929F92AF92BF92CF92DF92EF92FF92D0
:10D890000F931F93CF93DF9380913C0987FD38C08E
:10D8A00080913D098370A1F5C091FD17D091FE17BD
:10D8B000488159816A817B8186E99BE00E9482A42C
:10D8C0004C815D816E817F8182EF96E50E9482A40A
:10D8D0004091F9175091FA176091FB177091FC175E
:10D8E0008FEE96E50E9482A48AE0DF91CF911F918E
:10D8F0000F91FF90EF90DF90CF90BF90AF909F90EF
:10D900008F907F906F905F904F903F900C94059E0A
:10D910006090F1177090F2178090F3179090F417C1
:10D92000A090F517B090F6170091F7171091F8171F
:10D93000C090F917D090FA17E090FB17F090FC1701
:10D9400088E50E948A8FC82F882309F49AC00E9414
:10D95000128F362E472E582ED92F20E030E044EB80
:10D9600053EC0F94A56987FD0DC020E030E044EB37
:10D9700053E4632D742D852D9D2F0F94756018161B
:10D980000CF081C068E671E083E89BE00E94A3A4EC
:10D9900068E671E08EE79BE00E94A3A48BE79BE022
:10D9A0000E94909EC0E089E50E948A8F882361F1E1
:10D9B0000E94128F362E472E582ED92F20E030E0AD
:10D9C00044EB53EC0F94A56987FD0DC020E030E0D7
:10D9D00044EB53E4632D742D852D9D2F0F947560BA
:10D9E00018160CF055C068E671E088E69BE00E94CE
:10D9F000A3A468E671E083E69BE00E94A3A480E60E
:10DA00009BE00E94909EC0E08AE50E948A8F882356
:10DA100009F443C00E94128F6B017C0120E030E0CA
:10DA200040E151EC0F94A56987FD0AC020E030E089
:10DA300040E151E4C701B6010F94756018166CF50A
:10DA400067EF7FEF8EE49BE00E94A3A469E070E0A3
:10DA500089E49BE00E94A3A486E49BE0DF91CF9140
:10DA60001F910F91FF90EF90DF90CF90BF90AF90FC
:10DA70009F908F907F906F905F904F903F900C940D
:10DA8000909EC1E090CF632C742C852C9D2E8BCF63
:10DA9000A32CB42C052D1D2FB7CFCC23E1F0C3014F
:10DAA000D4018093F1179093F217A093F317B093DA
:10DAB000F417C501D8018093F5179093F617A0933A
:10DAC000F717B093F817C092F917D092FA17E092AF
:10DAD000FB17F092FC17DF91CF911F910F91FF90F0
:10DAE000EF90DF90CF90BF90AF909F908F907F90FE
:10DAF0006F905F904F903F900895CF92DF92EF929A
:10DB0000FF928AE50E948A8F882309F45AC00E94F6
:10DB1000128F20E030E040E050EC0F947560C12C93
:10DB2000D12CE12C90ECF92E87FD0FC00E94128FB2
:10DB300020E030E040E050E40F94A56918160CF4A2
:10DB400062C00E94128F6B017C012091D111309133
:10DB5000D2114091D3115091D411C701B6010F9445
:10DB6000DB600F94B168CB010F945F3880E50E94B1
:10DB70003C8F81114EC0A70196016091F9177091F9
:10DB8000FA178091FB179091FC170F9445676093EB
:10DB9000F9177093FA178093FB179093FC170E9464
:10DBA000CEB84091F9175091FA176091FB17709118
:10DBB000FC1787E39BE00E9482A48AE00E94059EF6
:10DBC00005C083E50E948A8F8111A1CF80913C0915
:10DBD00087FD24C080913D09837001F50E94CEB875
:10DBE0004091F9175091FA176091FB177091FC174B
:10DBF00088E29BE00E9482A48AE0FF90EF90DF9091
:10DC0000CF900C94059EC12CD12CE12C80E4F82EF1
:10DC10009CCF0E94FE8E8111AECFD8CF82E50E94AC
:10DC20003C8F8111DBCFFF90EF90DF90CF90089574
:10DC30002F923F924F925F926F927F928F929F921C
:10DC4000AF92BF92CF92DF92EF92FF920F931F930A
:10DC5000CF93DF93CDB7DEB7E5970FB6F894DEBF6D
:10DC60000FBECDBF8DAB20911F092CAB81E08093FF
:10DC70001F0980918C098D3409F47EC5843511F417
:10DC80000C946583873409F091C180918A09909141
:10DC90008B098B31910509F4DDC108F079C184301D
:10DCA000910508F030C12091E90B8230910508F40C
:10DCB0008EC1213009F091C111E0029709F010E006
:10DCC0000E946D3219821A821B821C821D821E8262
:10DCD0001F82188682E50E948A8F882309F490C1EA
:10DCE0000E94128F6B017C0120E030E0A9010F94AB
:10DCF0007560882309F4EAC040905F02509060028A
:10DD0000609061027090620280916302909164025F
:10DD1000A0916502B09166028CA79DA7AEA7BFA790
:10DD200080907C0C90907D0CA0907E0CB0907F0C2D
:10DD30008091800C9091810CA091820CB091830C09
:10DD400088AB99ABAAABBBABA5019401C301B201EF
:10DD50000F94756081110DC028A939A94AA95BA942
:10DD60006CA57DA58EA59FA50F947560882309F4E9
:10DD7000ADC0A3019201C501B4010F94446720E036
:10DD800030E040E05FE30F94DB6068A779A78AA7E3
:10DD90009BA72CA53DA54EA55FA568A979A98AA931
:10DDA0009BA90F94446720E030E040E05FE30F94CC
:10DDB000DB602B013C0120E030E0A901C701B60186
:10DDC0000F947560881F8827881F181709F40FC1E2
:10DDD00080E090E0A0E8BFEB8CA79DA7AEA7BFA70F
:10DDE00028A539A54AA55BA5CA01B9010F94DB6036
:10DDF0004B015C01A3019201C301B2010F94DB60EE
:10DE00009B01AC01C501B4010F9445670F94436AAF
:10DE10004B015C01AC019B01C701B6010F94446743
:10DE200068AB79AB8AAB9BABA5019401C701B60186
:10DE30000F9445679B01AC0168A979A98AA99BA9A0
:10DE40000F94DB606B017C0120E030E0A9010F94AE
:10DE5000A56987FDD1C0C701B6010F94436A6B0164
:10DE60007C01C301B2019058A50194010F943F6851
:10DE70002CA53DA54EA55FA50F94DB60A7019601DB
:10DE80000F94DB6028A539A54AA55BA50F944567CB
:10DE900069837A838B839C83A501940168A579A506
:10DEA0008AA59BA50F943F682CA53DA54EA55FA50F
:10DEB0000F94DB60A70196010F94DB60A301920130
:10DEC0000F9445676D837E838F83988720E030E0D1
:10DED000A90169817A818B819C810F947560811180
:10DEE000A3C020E030E0A9016D817E818F819885FB
:10DEF0000F947560811198C00E9418AC88E295E07B
:10DF00000E94909E6AC08531910509F466C08A31ED
:10DF1000910509F49CC0049709F048C080E50E946F
:10DF20008A8FC12CD12C7601882321F00E94EE8BA0
:10DF30006B017C0183E50E948A8F882361F00E9437
:10DF4000128F20E030E04AE754E40F94DB600F9436
:10DF5000B8686B017C010E94723480919C1681111B
:10DF600005C060E08EE395E00E94B4550F9426381A
:10DF7000C60ED71EE81EF91E0F9426386C197D09AF
:10DF80008E099F0997FF29C080E00E9405BCF4CF4D
:10DF90008A32910509F494C260F48D31910509F437
:10DFA00013C208F470C04E9709F411C20F945C3587
:10DFB00014C08B35910509F437C38C35910509F4EC
:10DFC00037C38A35910591F71092270D06C021308D
:10DFD00021F40E946D320E94F63B3DA9311102C02E
:10DFE0000F94314F8CA980931F090C94237B80E000
:10DFF00090E0A0E8BFE3F0CEC12CD12C760131CF68
:10E0000089E40E948A8F882331F00E94128F6983ED
:10E010007A838B839C838AE40E948A8F882309F405
:10E0200055CF0E94128F4ECF412FBE016F5F7F4FA1
:10E030008CE79CE00F94874F0F9426386093ED1681
:10E040007093EE168093EF169093F016C6CF0E9451
:10E05000ADA4C3CF87E00E94C26B8111BECF8CE01C
:10E06000E8ECF2E0DE01119601900D928A95E1F75D
:10E0700070E060E080E50E94978FBE016F5F7F4F88
:10E080000E94504CAACF87E00E94283B811106C015
:10E0900060E08FE40E94C88F81119FCF0E9472348C
:10E0A000109244026091B0118CE40E94C88FE82E57
:10E0B00080E00E94BC970F9426386093ED16709311
:10E0C000EE168093EF169093F0160E94C74481E0FD
:10E0D0008093A40B0E94D74A8AE50E943C8FF82EB9
:10E0E000882369F081E00E94283B182F82E00E947B
:10E0F000283B11110C94808311E0811101C010E0C4
:10E1000088E50E943C8F082F81110C947A831111AD
:10E110000CC089E50E943C8F81133DC1012FF11293
:10E1200004C001E011E0FF24F39482E50E948A8F8D
:10E13000882309F433C10E94128F6CA37DA38EA3A0
:10E140009FA320E030E0A9010F947560882381F03F
:10E15000011105C0111103C0FF2009F40EC160E0D8
:10E16000CE0184960E9456460E941F9C0E94E99B05
:10E17000002309F47DC0112309F477C010925F02D7
:10E180001092600210926102109262021092630279
:10E190001092640210926502109266020E94664715
:10E1A00083E09EE00E94FE8B4B015C0187E09EE0D5
:10E1B0000E94FE8B2B013C01AC019B01C501B40107
:10E1C0000F94A56918160CF0EEC0A5019401C301C7
:10E1D000B2010F943F689B01AC010F94DB6020E01B
:10E1E00030E040E85FE30F9445670F94436A20E016
:10E1F00030E048E452E40F94DB6068A379A38AA37B
:10E200009BA320E030E040EC5FE3C301B2010F9438
:10E21000DB6069837A838B839C8320E030E040EC71
:10E220005FE3C501B4010F94DB606C8F7D8F8E8F2F
:10E230009F8FAE01405E5F4FBE016F5F7F4FCE018B
:10E240004C960E9415460E94303210925F02109246
:10E2500060021092610210926202109263021092A8
:10E260006402109265021092660280E00E9491475B
:10E27000112319F081E00E949147FF2009F47DC02D
:10E2800083E00E94C26B811178C00E946647209192
:10E290003D0D30913E0D40913F0D5091400D60E09D
:10E2A00070E084E393E40F9444672B013C012091D8
:10E2B000410D3091420D4091430D5091440D60E06D
:10E2C00070E084E393E40F9444674B015C01809118
:10E2D000670290916802A0916902B0916A028093EE
:10E2E000840C9093850CA093860CB093870C0091BE
:10E2F000FD171091FE17D8012D913D914D915C9124
:10E30000C301B2010F94446760937C0C70937D0C41
:10E3100080937E0C90937F0CF80124813581468197
:10E320005781C501B4010F9444676093800C7093CA
:10E33000810C8093820C9093830C8CE79CE00E946C
:10E34000FA968823A9F11C8E1D8E1E8E1F8E88E0E2
:10E35000ECE7FCE0DE01119601900D928A95E1F761
:10E36000AE01445E5F4FBE016B5F7F4FCE010196F1
:10E370000E94154682E00E9491470E946647809164
:10E38000A30B8093A40B8E2D0E94BC970E94AE44D9
:10E390000E946F4922CE012F182FC7CE60E070E097
:10E3A00080E890E4CACEA3019201C501B40111CF67
:10E3B00060E089E595E00E94B4550E94CEB887E4FC
:10E3C00095E00E94909ED9CF0E9431D206CE009156
:10E3D000FD171091FE17D8012D913D914D915C9143
:10E3E00060915F027091600280916102909162027F
:10E3F0000F944567AB01BC0188E50E94B18F69832A
:10E400007A838B839C83F8012481358146815781EF
:10E41000609163027091640280916502909166023E
:10E420000F944567AB01BC0189E50E94B18F6D83F4
:10E430007E838F839887BE016B5F7F4FCE010196ED
:10E440000E941890882309F4C8CD80E00E94BC97F0
:10E450000E94C74461E085E40E94C88F182F01E044
:10E4600021E041E0682FCE0101960E94E0AC6B01F3
:10E470007C01AC019B010F94926A811119C0498102
:10E480005A816B817C8184E795E00E9482A44D8152
:10E490005E816F8178858FE695E00E9482A4B70146
:10E4A000A6018AE695E00E9482A48AE00E94059E69
:10E4B0000E94AE4411110E94FE8F0E946F498DCDC3
:10E4C0008091E90B813009F088CD89E40E948A8F20
:10E4D000182FE12C882319F00E940E8FE82E8AE471
:10E4E0000E948A8F082F882379F00E940E8FF82EC1
:10E4F000112309F490C0F5E0FE1508F089C08CE7FF
:10E5000095E00E94909E69CDF12C1111F4CF80E12D
:10E51000EFE5F2E0ACE7BCE001900D928A95E1F7FF
:10E52000112359F08E2D0E94869160937C0C70937C
:10E530007D0C80937E0C90937F0C002359F08F2DDF
:10E540000E94F0906093800C7093810C8093820CF9
:10E550009093830C60E080E50E94C88F8823C1F10E
:10E560001123D1F0E091FD17F091FE172081318148
:10E570004281538160917C0C70917D0C80917E0C66
:10E5800090917F0C0F94446760937C0C70937D0C8A
:10E5900080937E0C90937F0C0023D1F0E091FD17C7
:10E5A000F091FE1724813581468157816091800C5E
:10E5B0007091810C8091820C9091830C0F94446730
:10E5C0006093800C7093810C8093820C9093830CE9
:10E5D00040E050E0BA0186E40E94B18F6B017C01FB
:10E5E00020E030E0A9010F94A5691816CCF420E0D2
:10E5F00030E040E752E4C701B6010F943F686983F9
:10E600007A838B839C83CE0101960E94E644E5CCFD
:10E61000002309F47CCF25E02F1508F078CF6FCFC9
:10E6200060E070E0CB01EBCF8FE08093270DD5CC7D
:10E6300080918909882381F1893009F0CECC04EDDD
:10E64000A02E02E0B02E8FE5C82E82E0D82EE12C5D
:10E6500000E010E0D5018D915D010E948A8FF82EB7
:10E66000882361F0133011F4082FFE2C0E94128FC2
:10E67000F6016083718382839383EF2C1F5FF4E044
:10E68000CF0ED11C143031F7EE2009F457C00E9490
:10E6900066470E946F49A1CC14EDC12E12E0D12E25
:10E6A000F12CE12C00E010E0D6018D916D010E946B
:10E6B0008A8F382E8823D9F10E94128F4B015C017A
:10E6C000133059F0F701E550F24F2081318142813A
:10E6D00053810F9444674B015C01F701E15AFD4FF0
:10E6E0002081318142815381C501B4010F94446777
:10E6F0002B013C012DEB37E346E855EB0F94A56960
:10E7000087FD0AC02DEB37E346E855E3C301B201AC
:10E710000F94756018165CF41330C1F480926B028C
:10E7200090926C02A0926D02B0926E02032D1F5F58
:10E73000B4E0EB0EF11C143009F0B6CF002309F45D
:10E74000A8CF8BE692E00E943438A3CFF701EF5CAC
:10E75000F24F5F01A30192016081718182819381F7
:10E760000F944567D5016D937D938D939C9313977B
:10E77000812F0E94083BDBCF80918A0990918B0901
:10E780008937910511F40C946A7D08F0D0C18D345D
:10E79000910509F465C608F0EEC08A31910509F4C7
:10E7A0009AC508F091C08431910509F4E0C408F0DD
:10E7B0006EC08131910509F4A1C408F042C00297EE
:10E7C00008F0F4CB80E50E948A8FC12CD12C760111
:10E7D000882321F00E94EE8B6B017C0183E50E946F
:10E7E0008A8F882361F00E94128F20E030E04AE790
:10E7F00054E40F94DB600F94B8686B017C010E94B5
:10E80000723480918D0990918E09892B09F471C41D
:10E810000F946A3580918A0990918B096DE975E0B2
:10E82000892B11F465E975E030E020E045EA55E018
:10E8300082E00E9444A240E0C701B6010E9410D8C5
:10E84000CCCB429709F0B2CB83E50E948A8F882314
:10E8500009F4EAC70F9426386093ED167093EE160C
:10E860008093EF169093F0160E94128F20E030E014
:10E870004AE754E40F94DB600F94B8686093010298
:10E88000709302028093030290930402A6CB873117
:10E89000910509F4A1C470F48531910509F498C477
:10E8A000469709F083CB8091BA1982FD96CB0E94DE
:10E8B000D7EA93CB8831910509F4A3C4499709F0AD
:10E8C00075CB0E94FED989CB8032910509F487C5AA
:10E8D000C0F58D31910509F46BC570F48B3191054C
:10E8E00009F40CC54C9709F061CB80918D0990918A
:10E8F0008E090E94C9EF71CB8E31910509F45FC575
:10E900004F9709F053CB0E94034C6C8F7D8F8E8FF5
:10E910009F8FBE016F5F7F4FCE014C960E940631E4
:10E92000CE0101960F94551E0E94CEB8BE016F5FB6
:10E930007F4F89E196E00E940EAC8AE00E94059E1E
:10E940004CCB8934910509F477C550F48132910597
:10E9500009F46EC5C09709F029CB0E9413AF3DCBD7
:10E960008B34910509F478C58C34910509F01ECBE0
:10E970000E943E5232CB8C36910509F42ECB08F022
:10E9800071C08535910509F492C790F582359105DE
:10E9900009F43AC720F58E34910509F465C581352F
:10E9A000910509F003CB0E948AF50E94F4300E9481
:10E9B0006A9A0E946D9A1092960C1092950C109281
:10E9C000940C68EE73E080E090E00E9450990E9401
:10E9D000729A60E084EE96E00E94B455FECA8335D8
:10E9E000910509F419C78435910509F42DCFDECAC4
:10E9F0008936910509F415C600F58C35910509F4A1
:10EA00007BC78836910509F0D1CA80916B1183FDCF
:10EA1000E4CA0E94166C87FDE0CA83E50E948A8FD3
:10EA2000882341F00E940E8F0E94423461E080E012
:10EA30000F9471540F94D053D0CA8A36910509F4BB
:10EA40001BC68B36910509F0B1CA60E080E50E94D3
:10EA5000A58F823008F0C1CAE82FF0E0E05DF14FE9
:10EA60001082BBCA8237910509F4E7C7A0F58F363B
:10EA7000910509F42AC6C8F48D36910509F486C5B6
:10EA80008E36910509F092CA8EE40E948A8F8823FF
:10EA900009F4A3CA0E94DA8E60939D1270939E12AD
:10EAA00080939F129093A01298CA8037910509F421
:10EAB00094CA8137910509F079CA83E50E948A8F4B
:10EAC000882309F449C60E94EA8E8D3308F03FC6B8
:10EAD0008093000282CA8637910509F4BEC7B8F454
:10EAE0008337910509F4B1C78537910509F05ECAEE
:10EAF00080918D0990918E09009709F4AAC7DC01D5
:10EB00002C91222309F4A5C70F94551E66CA873796
:10EB1000910509F4DBC78837910509F047CA81E000
:10EB20008093A40B8093A30B0E94D74A56CA8239C4
:10EB3000E1E09E0711F40C94E08008F073C1833D7E
:10EB4000910511F40C946D7E08F0C2C0883C9105CB
:10EB500009F4C8C7D0F58C38910509F40DC628F41E
:10EB60008D37910509F4ADCE21CA8B39910509F491
:10EB700024C68E3B910509F019CA80916B1183FD63
:10EB80002CCA83E50E948A8F182F882309F40BC6AC
:10EB90000E940E8F0E947F8D60E081E00F9471547F
:10EBA0002091F9163091FA168091F7169091F81687
:10EBB000821793070CF4FEC586EC96E060E00E9495
:10EBC000B455812F0E942EF208CA8C3C910511F495
:10EBD0000C94F07D40F5893C910509F4D7C78B3C36
:10EBE000910509F0E3C90E94166C87FDF6C964ED32
:10EBF000E62E62E0F62E10E000E0D7018D917D0157
:10EC00000E943C8F882349F00E94128FF801EB5438
:10EC1000FE4E64A375A386A397A30C5F1F4F00311C
:10EC2000110559F7DAC98D3C910511F40C94697EF0
:10EC30005DE3E52E5DE0F52E10E08E3C910509F0D8
:10EC4000B5C988E5810F0E943C8F882351F00E944E
:10EC5000128FF7016083718382839383812F0E94D7
:10EC6000083B1F5FF4E0EF0EF11C133051F7809169
:10EC70003C0987FD0ECD80913D09837009F009CDD7
:10EC800040913D0D50913E0D60913F0D7091400DB2
:10EC90008CE097E00E9482A44091410D5091420D7A
:10ECA0006091430D7091440D82EF96E50E9482A41D
:10ECB0004091450D5091460D6091470D7091480D62
:10ECC0008FEE96E50E9482A48AE00E94059E85C987
:10ECD0008D3221E0920711F40C946E7F08F06CC025
:10ECE0008831A1E09A0711F40C94CE7E08F045C05B
:10ECF0008C3D910511F40C94717E8D3D910509F0C8
:10ED000055C90E94166C082F87FD67C983E50E94CC
:10ED10008A8F002E000C110B7801EE0CFF1C88234B
:10ED200011F40C94B47E0E940E8FF701ED58FD4F44
:10ED300091838083000F111F000F111F980121592B
:10ED40003D4F7901BC01990F880B990B0F947C60A2
:10ED50002AE037ED43E25CE30F94DB600F541E4E74
:10ED6000D8012D913D914D915C910F94DB60F7019D
:10ED7000608371838283938330C98232E1E09E078E
:10ED800011F40C946A7F8C32914009F00FC964E051
:10ED900071E083E50E94978F8C0168EE73E080E557
:10EDA0000E94978F893823E1920710F088E893E159
:10EDB000B8010E94055311C9803321E0920711F474
:10EDC0000C94F07F00F58E32A1E09A0711F40C94B8
:10EDD00064808F32914009F0E9C870E060E085E41A
:10EDE0000E94DD8FF82E3FEF831711F40C94D98029
:10EDF000882311F40C94AA8086EA97E00E94909EE2
:10EE00000F941B1DEAC88039E1E09E0711F40C94B1
:10EE1000DC808139914009F0C9C80E94F58F0E94B9
:10EE20006F49DBC88C3022E0920711F40C94DC812E
:10EE300008F07AC08C3AA1E09A0711F40C941C8176
:10EE400008F043C08D39E1E09E0711F40C94418332
:10EE500078F58A3921E0920709F4BFC88C399140CE
:10EE600009F0A4C880913A09887811F00C94E880E0
:10EE700080913C09867011F00C94E8800E94CEB815
:10EE80008AEE97E00E94909E809120020E946CA4DE
:10EE900040911C0250911D0260911E0270911F0250
:10EEA0008AEC97E00E9482A48AE00E94059E95C8A1
:10EEB000843AA1E09A0711F40C941881853A9140A4
:10EEC00009F074C80E941CAC88C8863FE1E09E0728
:10EED00011F40C94CE8168F4843F21E0920711F480
:10EEE0000C94CA81853F914009F060C80F94C01806
:10EEF00074C8873FA1E09A0711F40C94D281883F2F
:10EF0000914009F053C881E08093E10A0E949A334E
:10EF10001092E10A882309F460C80E94CEB887E302
:10EF200098E00E94909E59C88C36E3E09E0709F451
:10EF300054C808F08EC08D3B22E0920711F40C9467
:10EF4000078208F077C08835A2E09A0711F40C9484
:10EF5000ED818B35924009F029C80E94166C082F6C
:10EF600087FD3BC885E50E943C8F882369F10E949C
:10EF7000128F4B015C01E02E002E000CFF0820E0F8
:10EF800030E0A9010F94A56987FF04C0B7FAB094D7
:10EF9000B7F8B09420E030E84BE354E4C501B40185
:10EFA0000F94A569970153E0220F331F5A95E1F79B
:10EFB0002D52354F181614F40C94F181D9018D920D
:10EFC0009D92AD92BC9213978CE40E943C8F882353
:10EFD00011F40C94ED6F0E94128F6B017C01002ED6
:10EFE000000C110B20E030E0A9010F94A56987FF08
:10EFF00004C0F7FAF094F7F8F09420E030E84BE31F
:10F0000054E4C701B6010F94A569980143E0220FAB
:10F01000331F4A95E1F72D52354F181614F40C940E
:10F02000FC81D9011496CD92DD92ED92FC92179756
:10F030000C94ED6F8E3BE2E09E0711F40C940B8272
:10F040008335934011F00C94D66F0E943B6C0C9466
:10F05000ED6F873E23E0920711F40C943183C8F4DE
:10F060008438A3E09A0711F40C94C682803A934046
:10F0700011F00C94D66F20918D0930918E099091EA
:10F08000BA1992609093BA19C9010E94C9EF0C9401
:10F09000ED6F883EE3E09E0711F40C945A83893E9D
:10F0A000934011F00C94D66F8091B01981110C949B
:10F0B0005E830E948A8D0E94BEEF0E94034C6D33D6
:10F0C00071058105910520F08DE998E00E94B283D9
:10F0D00089E998E00E94B28384EE8093970985E8DD
:10F0E00098E00E94909E81E898E00E94B2830C9480
:10F0F000ED6F8EEA95E00E94E04F8CCB80913A094B
:10F1000084FD17C080913C0987FD13C080913D09A3
:10F11000837079F460E081EC95E00E94B4555F98CB
:10F120008A988091080181708093060112980C944E
:10F13000ED6F88E50E943C8F81115F9889E50E9400
:10F140003C8F81118A988AE50E943C8F882329F0A0
:10F150008091080181708093060185E40E943C8FB4
:10F16000882311F40C94ED6F12980C94ED6F80913C
:10F17000BA1983FF25C089ED95E00E94909E809189
:10F18000BA1983FF17C08AED99E10E944EEB8BE11B
:10F19000EAEDF9E1DE01119601900D928A95E1F711
:10F1A00070E060E0CE0101960F94D119CE01019676
:10F1B0000E94B28D8AEC95E00E94909E0C94ED6FB7
:10F1C0000E94CEB88AEE95E00E94909E0C94ED6F5E
:10F1D0000E94E8EA0C94ED6F80918D0990918E0960
:10F1E000FC012191222331F02032D9F7DF01119760
:10F1F0001C92F7CF60E00E9412F0109297090C94D5
:10F20000ED6F83E50E948A8F882321F00E94DA8EB9
:10F210000E94D76984E50E948A8F8823A9F00E9402
:10F22000DA8E6B017C010E94354CC092BA09D092F3
:10F23000BB09E092BC09F092BD09CD28CE28CF28A9
:10F2400019F081E080939B1680919A168823F9F03B
:10F2500080E090E0A0EAB1E489839A83AB83BC8329
:10F260001C8E1D8E1E8E1F8E18A219A21AA21BA202
:10F2700010E000E020E0AE014F5F5F4FBE01645E32
:10F280007F4FCE0180960E94EBCA0C94ED6F0E94D6
:10F290005C9A882381F00E94D1E20E94915187E814
:10F2A0009DE00E9476EA10920413109205131092CA
:10F2B00006131092071361E08EEF9CE00E94EBA111
:10F2C0004BEE5CE064EF75E085E00F94121D0F9447
:10F2D0008D1E0C94ED6F8091BA1983FD02C00C94C1
:10F2E000ED6F83E50E948A8F882311F40C94ED6FF3
:10F2F0000E94DA8E0E94D7690C94ED6F83E40E941D
:10F300003C8F882361F18AE096E00E94909E809174
:10F31000211B8823F9F0BE016F5F7F4F8EE19BE1D7
:10F320000E9409EACE0101960E94BD4ECE010196CF
:10F330000E9494EB80911617882339F080E20E9496
:10F34000059E86E197E10E94BD4E8AE00E94059EDF
:10F350000C94ED6F80E096E00E94909EF6CF83E5DE
:10F360000E948A8F882301F10E94EA8E182F8C3325
:10F3700008F08CE3809314090F9426386B017C010C
:10F38000212F30E0A8EEB3E00F940D67C60ED71E14
:10F39000E81EF91EC0921009D0921109E0921209DC
:10F3A000F09213090C94ED6F0E948FE20C94ED6FB4
:10F3B0008091BA198E7F8093BA190C94ED6F809169
:10F3C000BA1983FD02C00C94ED6F0F944235809101
:10F3D0008D0990918E090E9456EF0C94ED6F8091EB
:10F3E000BA1982FD0E9472348091BA1983FD02C05D
:10F3F0000C94ED6F60E080E50E94C88F182F682F95
:10F4000080918D0990918E090E9412F083E50E94EF
:10F410008A8F882321F00E94DA8E0E94D7690E9489
:10F42000D1E211110C94ED6F0E9491510C94ED6F8B
:10F430000E94C94E0C94ED6F80E50E943C8F88239A
:10F4400011F40C94ED6F0E94EA8E853608F084E684
:10F45000809397090C94ED6F0E9491510C94ED6F7D
:10F460000E946A9A0C94ED6F70E060E083E50E9460
:10F47000DD8F8E34910531F40E94DE330F948D1EA2
:10F480000C94ED6F84E896E00E94909E6091930B3F
:10F490007091940B8BE796E00E9478A46091950B95
:10F4A0007091960B8EE696E00E9478A46091930B83
:10F4B0007091940B8091950B9091960B681B790B32
:10F4C00080919B16815021E030E0823010F030E0D6
:10F4D00020E0621B730B83E696E00E9478A48AE02A
:10F4E0000E94059E8BE596E00E94909E8091970B6E
:10F4F0009091980BA091990BB0919A0B8C8F9D8F46
:10F50000AE8FBF8FBE016F5F7F4FCE014C960E94C2
:10F510000631BE016F5F7F4F8EE496E00E940EAC15
:10F5200080919B0B90919C0BA0919D0BB0919E0B99
:10F530008C8F9D8FAE8FBF8FBE016F5F7F4FCE01CF
:10F540004C960E940631BE016F5F7F4F8EE396E0BE
:10F550000E940EAC20E030E04AE754E460919F0B3B
:10F560007091A00B8091A10B9091A20B0F943F681A
:10F57000AB01BC0186E296E00E9482A48DE60E9467
:10F58000059E8AE00E94059E0C94ED6F80916B11A0
:10F5900083FF02C00C94ED6F0E94166C082F87FF4A
:10F5A00002C00C94ED6F83E50E948A8F182F882388
:10F5B00059F10E940E8F0E94423461E081E00F9465
:10F5C0007154209164173091651780916217909162
:10F5D000631782179307F4F487E996E09F938F935C
:10F5E00082EA96E09F938F931F920E9497550F9403
:10F5F000D0530F900F900F900F900F90612F802F8E
:10F600000E94A5F30C94ED6F82E50E948A8F811110
:10F61000D0CF10CA8CE896E0112301F30F94D05399
:10F62000EDCF0E94166C182F87FD0AC087EA96E07E
:10F630000E94909E812F0E94BBF18AE00E94059E4D
:10F640002CA920931F09E5960FB6F894DEBF0FBED4
:10F65000CDBFDF91CF911F910F91FF90EF90DF9081
:10F66000CF90BF90AF909F908F907F906F905F9062
:10F670004F903F902F90089560E080E50E94A58F05
:10F68000F82E31E0381710F40C94ED6F81E40E94ED
:10F690003C8F6091300E062F811102C00FEF10E0F9
:10F6A00083E50E948A8F882349F00E94DA8E8B01BD
:10F6B0006F3F710519F010F00FEF10E0EF2DF0E043
:10F6C000E05DF14F00830C94ED6F83E50E943C8F69
:10F6D000882331F060E083E50E94A58F80936B1151
:10F6E0000E94CEB888EB96E00E94909E80916B11AC
:10F6F000882351F110E000E020E080916B1190E050
:10F70000B0E0A0E0002E04C0B695A7959795879528
:10F710000A94D2F780FF12C0FF24F394F20E222342
:10F7200019F08CE20E94059EF801EE0FFF1FE255D2
:10F73000F94F859194910E94909E2F2D0F5F1F4F3E
:10F7400005301105D1F601CE8AEA96E005CE8CE3AC
:10F75000809300020C94ED6F0E94CEB810910002CD
:10F760008FEB96E00E94909E812F0F944B1B8AE0B6
:10F770000E94059E0C94ED6F80916B1183FF02C077
:10F780000C94ED6F83E50E948A8F882311F40C940A
:10F79000ED6F0E940E8F0E947F8D61E080E00F94DC
:10F7A00071540C94ED6F82E50E948A8F8111F0C92B
:10F7B0000C94ED6F85ED96E001CA83E50E948A8F77
:10F7C000882311F40C94ED6F0E94EA8E182F8C336D
:10F7D00008F08CE3809319090F9426386B017C01A3
:10F7E000212F30E0A8EEB3E00F940D67C60ED71EB0
:10F7F000E81EF91EC0921509D0921609E092170969
:10F80000F09218090C94ED6F8091270D8F7D806127
:10F810008093270D0C94ED6F8091270D8F7E806271
:10F820008093270D0C94ED6F80913A0984FD0CC0F4
:10F8300080913C0987FD08C080913D09837021F4C7
:10F840000E94F4300C94ED6F0E94723488E50E949F
:10F850003C8F882331F05F9A8091AF118E7F809327
:10F86000AF1189E50E943C8F882331F08A9A8091FC
:10F87000AF118D7F8093AF118AE50E943C8F882362
:10F8800059F08091080180958170809306018091E4
:10F89000AF118B7F8093AF1185E40E943C8F88234A
:10F8A00011F40C94ED6F0E94419A0C94ED6F83E576
:10F8B0000E943C8F882311F40C94ED6F0F9426382E
:10F8C0006093ED167093EE168093EF169093F016FA
:10F8D0000E94128F20E030E04AE754E40F94DB608E
:10F8E0000F94B86860931A0970931B0980931C09E0
:10F8F00090931D090C94ED6F0E94166C87FF02C057
:10F900000C94ED6F80913A0984FD09C080913C0907
:10F9100087FD05C080913D09837009F489C0F4ED2D
:10F92000CF2EF2E0DF2EA5EBEA2EA1E1FA2E10E0B9
:10F93000D6018D916D010E948A8F882309F465C0DC
:10F94000133009F06DC00E94128F4B015C0120E062
:10F9500030E040EA51E40F94756087FF4EC0A50186
:10F9600094016091D5117091D6118091D711909129
:10F97000D8110F943F682B013C01AC019B016091B1
:10F98000280E7091290E80912A0E90912B0E0F94C3
:10F99000DB606093280E7093290E80932A0E90935B
:10F9A0002B0EA30192016091E5117091E6118091F7
:10F9B000E7119091E8110F94DB606093E51170936B
:10F9C000E6118093E7119093E8116091140E709105
:10F9D000150E8091160E9091170E0F947A60A30168
:10F9E00092010F94DB600F94B8686093140E7093CB
:10F9F000150E8093160E9093170E8092D51190924B
:10FA0000D611A092D711B092D8111F5FF4E0EF0E7B
:10FA1000F11C143009F08CCF0E944E340C94ED6F21
:10FA20000E94128FF701648B758B868B978BEDCFBD
:10FA300081E00F94E9340C94ED6F0F94F83284E177
:10FA400098E10E9417FD0C94ED6F0E9421300C94F8
:10FA5000ED6F0F948D1E0C94ED6F00918D09109138
:10FA60008E0994E0F12C40E09150F9F0F80180818A
:10FA7000282F2B7F213499F421812133B1F4813453
:10FA800011F1853409F441E098012E5F3F4F89015F
:10FA90002F5F3F4FF80180818032C9F3E5CF803579
:10FAA00021F4818180538A3078F341110E94CEB8CD
:10FAB000FF2021F086EF96E00E94909EC8010E94F0
:10FAC000B16B0C94ED6FFF24F394DECF0E94E5310F
:10FAD0000C94ED6F1092A40B1092A30B0E94D74AC6
:10FAE0000C94ED6F0E94166C182F87FF02C00C94C7
:10FAF000ED6F0091300D84E40E948A8FB82E882328
:10FB0000C9F10E94128F6B017C0120E030E0A90155
:10FB10000F9475608823C1F124E01202F0011124D2
:10FB2000E45DF24FC082D182E282F38220E030E0D5
:10FB3000A901C701B6010F94A5691816D4F420E0F5
:10FB400030E040E05FE3C701B6010F94DB609B014A
:10FB5000AC010F94DB602BED3FE049E450E40F94DF
:10FB6000DB60609305027093060280930702909316
:10FB700008020B2D602F83E50E94C88F8093300D03
:10FB80000E94BC340C94ED6F80E0F8CF0E94166C9C
:10FB900087FF02C00C94ED6F04ED12E075EBE72EC9
:10FBA00071E1F72EE8EDCE2EE2E0DE2ED8018D9148
:10FBB0008D010E943C8F882359F00E94128F0F9470
:10FBC000B868F70160837183828393830E94882FD2
:10FBD000F4E0EF0EF11CC016D10641F70C94ED6F66
:10FBE00080913B0987FD2DC080913C098E7049F5BD
:10FBF0004091E9115091EA116091EB117091EC1173
:10FC00008CEF96E00E9482A44091ED115091EE118C
:10FC10006091EF117091F01189EF96E00E9482A43B
:10FC20004091F1115091F2116091F3117091F41122
:10FC300087E496E40E9482A48AE00E94059E0C94C8
:10FC4000ED6F83E50E948A8F882391F00E94128FC6
:10FC50006093E9117093EA118093EB119093EC118A
:10FC60006093F1117093F2118093F3119093F4115A
:10FC700080E50E948A8F882351F00E94128F609342
:10FC8000E9117093EA118093EB119093EC1182E5E6
:10FC90000E948A8F882351F00E94128F6093ED1189
:10FCA0007093EE118093EF119093F01184E50E9410
:10FCB0008A8F882311F40C94ED6F0E94128F609349
:10FCC000F1117093F2118093F3119093F4110C944D
:10FCD000ED6F0E94EAA00C94ED6F0E94D2B80C94D4
:10FCE000ED6F82E40E943C8F882341F08091750281
:10FCF0009091760290930A028093090282E50E9415
:10FD00003C8F882341F08091090290910A029093E0
:10FD100076028093750283E50E948A8F882331F0F2
:10FD20000E940E8F909376028093750280913A091B
:10FD300090913B09A0913C09B0913D09892B8A2BF8
:10FD40008B2B11F00C94ED6F60917502709176021F
:10FD500083E197E00E94A3A485E20E94059E8AE0C9
:10FD60000E94059E0C94ED6F0E94CEB885E40E941F
:10FD7000059E80E3800F0E94059EF701ED58FD4F20
:10FD80006081718187E197E00E94A3A485E20E94CF
:10FD9000059E8AE00E94059E0C94ED6F80E50E940E
:10FDA0003C8F882311F40C94ED6F0E940E8F8C0110
:10FDB000892B09F082C083E50E943C8F882391F053
:10FDC0000E940E8F8F3F980731F48EEE97E10E94CC
:10FDD000779A0C94ED6FBC018EEE97E10E94E59A44
:10FDE0000C94ED6F0E94CEB870E060E082E297E084
:10FDF0000E94A3A48091F01708E5C02E02E0D02E47
:10FE0000C81AD10887FDD394CC0CDD1CCC0CDD1CAA
:10FE10000D2C000CEE08FF088091EF1798E8892E52
:10FE2000912C881A910887FD9394880C991C880C52
:10FE3000991C092C000CAA08BB088091EE1790E0D1
:10FE40008F3FC9F1FC01EE0FFF1FE80FF91FEB55C3
:10FE5000F84E81819281B3E0880F991FBA95E1F73E
:10FE6000B0E0A0E014E0B595A795979587951A9511
:10FE7000D1F702969C012F5F3F4F032E000C440BDD
:10FE8000550B281939094A095B09A4EBB0E00F9416
:10FE9000FA66A7019601281939094A095B090F94E6
:10FEA000DB66B9018FE197E00E94A3A48AE00E947B
:10FEB000059E0C94ED6F80E0DDCF0E9418ACB80178
:10FEC00089E397E00E94A3A48AE297E00E94909EB3
:10FED0000C94ED6F0E947D6D0C94ED6F60E085E4F5
:10FEE0000E94A58F811174C080E50E943C8F8823F9
:10FEF00051F00E94128F6093671770936817809378
:10FF0000691790936A1789E40E943C8F882381F0D7
:10FF10000E94128F2CEA35EC47E25EE30F94DB601F
:10FF200060936B1770936C1780936D1790936E1797
:10FF300084E40E943C8F882381F00E94128F2CEA77
:10FF400035EC47E25EE30F943F6860936F17709360
:10FF5000701780937117909372170E94CEB84091DA
:10FF60006717509168176091691770916A1788E454
:10FF700097E00E9482A42CEA35EC47E25EE36091B0
:10FF80006B1770916C1780916D1790916E170F948D
:10FF90003F68AB01BC0184E497E00E9482A42CEA94
:10FFA00035EC47E25EE360916F17709170178091B6
:10FFB0007117909172170F94DB60AB01BC0180E464
:10FFC00097E00E9482A48AE00E94059E0C94ED6F47
:10FFD0000E9418AC8CE497E00E94909E0C94ED6F08
:10FFE00080E50E943C8F882351F00E94128F60931D
:10FFF000FC167093FD168093FE169093FF1689E40D
:020000021000EC
:100000000E943C8F882381F00E94128F2CEA35ECED
:1000100047E25EE30F94DB60609300177093011773
:10002000809302179093031784E40E943C8F8823E7
:1000300081F00E94128F2CEA35EC47E25EE30F94C8
:100040003F68609304177093051780930617909389
:1000500007170E94CEB84091FC165091FD16609192
:10006000FE167091FF1686E697E00E9482A42CEAA5
:1000700035EC47E25EE360910017709101178091C3
:100080000217909103170F943F68AB01BC0182E601
:1000900097E00E9482A42CEA35EC47E25EE360918F
:1000A00004177091051780910617909107170F9408
:1000B000DB60AB01BC018EE597E00E9482A48AE080
:1000C0000E94059E0C94ED6F83E50E943C8F182FD3
:1000D000882369F00E940E8F9C0190935E028093AA
:1000E0005D0291E0232B09F090E09093320E80E5C1
:1000F0000E943C8F882361F020915D0230915E0266
:10010000232B11F00E94FE8E8093320E0C94ED6F23
:1001100011110C94ED6F0E94CEB886E897E00E9412
:10012000909E8091320E882391F08EE697E00E9497
:10013000909E60915D0270915E0285E797E00E945B
:10014000A3A481E797E00E94909E0C94ED6F8AE64D
:1001500097E0EDCF04EB10E083E50E948A8F8823BF
:1001600019F00E940E8F8C0165E070E083E40E941C
:10017000DD8FE82E60E085E50E94C88FD82E60E014
:1001800089E997E00E94B455B801110F880B990BCB
:100190000F947C6069837A838B839C832D2D4E2DF5
:1001A0006F2DCE0101960F947E0C0F948D1E0C9432
:1001B000ED6F06E410E0D0CF0E9472340C94ED6F26
:1001C0000E94EC8F0E94FE8F0E946F490C94ED6F8D
:1001D00088E40E943C8F882321F00E94FE8E809349
:1001E0001E0982E50E943C8F082F83E50E943C8F08
:1001F000182F011102C0882341F00E94109A112388
:1002000021F00E94FE8E8093200284E40E943C8FA5
:10021000882311F40C94ED6F0E94128F60931C02DE
:1002200070931D0280931E0290931F020C94ED6F39
:100230000E945FCE0C94ED6F87E00E94C26B81112B
:100240000C94ED6F77EFC72E7DE0D72E8FE592E00F
:1002500099A788A7DE0111961D017D0110E000E03D
:10026000C6010E94FE8BE8A5F9A581909190A1900E
:10027000B190F9A7E8A7A50194010F9444672B0159
:100280003C01D7014D925D926D927C92139720E0D4
:1002900030E040EA51EC0F94A56987FD0AC020E0E8
:1002A00030E040EA51E4C301B2010F9475601816C2
:1002B0007CF4F801E55EF14FE4911E164CF4B7FAB8
:1002C000B094B7F8B094F70180829182A282B38291
:1002D000D7018D909D90AD90BD907D0120E030E0E4
:1002E00040EA51ECC501B4010F94A56987FD3FC0F8
:1002F00020E030E040EA51E4C501B4010F9475609C
:100300001816ACF10F5F1F4FB4E0CB0ED11C0330B9
:10031000110509F0A5CF6DE3E62E6DE0F62E10E095
:10032000F10181919191A191B1911F01F701819307
:100330009193A193B1937F01812F0E94083B1F5F8E
:10034000133071F70E946F4960E08BEF97E00E94D5
:10035000B45563E972E084E690E00E9405536AEBCD
:1003600072E084E690E00E9405530C94ED6F0E94C9
:1003700018AC89E198E00E94909E61E08BE098E0E3
:100380000E94B45568E270E088EC90E00E9405534A
:100390000C94ED6F0E94FE550C94ED6F0F94530A70
:1003A0000C94ED6F61E083E50E94C88F91E089278E
:1003B0000F9492110C94ED6F8091BA1982FF05C0D1
:1003C00080648093BA190C94ED6F83FD02C00C9485
:1003D000ED6F0F9442350C94ED6F0E94F3D80C949E
:1003E000ED6F80E090E8ABE3B4E4F90180839183A2
:1003F000A283B3830C94E47780E090E8ABE3B4E4A9
:10040000F90184839583A683B7830C94ED6F0E94D2
:1004100007CA0C94ED6F0E94166C182F87FF02C05C
:100420000C94ED6F8AE50E948A8F812C912C90E2CA
:10043000A92E91E4B92E882379F040E050E0BA016A
:100440008AE50E94B18F4B015C0120E030E0A901F8
:100450000F94A56918167CF580E090E0A0EAB0E45E
:1004600089839A83AB83BC832091670230916802B1
:100470004091690250916A02C501B4010F94456729
:100480006B017C0120E030E048EC53E40F94756090
:1004900087FD06C0C12CD12C88ECE82E83E4F82E11
:1004A000CC8EDD8EEE8EFF8EBE016F5F7F4FCE0154
:1004B0004C960E94374685E50E943C8F882309F4BC
:1004C0005AC00E94128F6B017C0120E030E0A9012C
:1004D000C701B6010F94A56987FF04C0F7FAF0942D
:1004E000F7F8F094F7FAF094F7F8F094C982DA820A
:1004F000EB82FC8280E00E9438C3882321F0CE0189
:1005000001960E94749920E030E0A901C501B40170
:100510000F94A569181614F00C94ED6F80E090E02C
:10052000A0EAB0E489839A83AB83BC83A5019401DC
:1005300060916702709168028091690290916A02ED
:100540000F9444676B017C0120E030E0A9010F9417
:10055000A56918161CF0C12CD12C7601CC8EDD8E2D
:10056000EE8EFF8EBE016F5F7F4FCE014C960E94D4
:1005700037460C94ED6F28E01202F0011124ED5281
:10058000F54FC080D180E280F3809FCFA0902C0EE9
:10059000B0902D0EC0902E0ED0902F0E8BE40E94A6
:1005A0008A8F882339F10E94128F7B018C0120E011
:1005B00030E0A9010F94A56987FD0AC020E030E072
:1005C00040E251E4B701C8010F9475601816A4F415
:1005D0008FE30E94059E8BE40E94059E8DE498E0C7
:1005E0000E94909E85E498E00E94909E82E498E0AC
:1005F0000E94909E750186019701A801B501C60170
:100600000F947560882361F00E947234C701D8018D
:1006100080932C0E90932D0EA0932E0EB0932F0E40
:1006200080913A0990913B09A0913C09B0913D0914
:10063000892B8A2B8B2B11F00C94ED6F0E94CEB876
:1006400040912C0E50912D0E60912E0E70912F0E18
:1006500081E698E00E9482A48AE00E94059E0C94A4
:10066000ED6F81E08093E90B1092DC1660E083E58A
:100670000E94C88F81110C94ED6F0F946D210C9422
:10068000ED6F83E50E943C8F882341F00E94FE8E2F
:100690008093DB0A0E94928D0C94ED6F0E94CEB87D
:1006A0008CE698E00E94909E8091DB0A0E946CA4E8
:1006B0000C94ED6F0E949E9E0C94ED6F0E94BFEE15
:1006C00081110C94ED6F0C94597810918A090F9454
:1006D00026386093ED167093EE168093EF16909384
:1006E000F016112311F40C94ED6F812F0E9405F187
:1006F0000C94ED6F11110C948E7011E00C948970B4
:100700008823D9F30C949170DF92EF92FF920F93AC
:100710001F93CF93DF93EC01E0908D0CF0908E0C43
:100720008AE0D82E6AE070E0CE010F94E66B8C016F
:10073000009711F0FC011082CE010E94396A81E01D
:100740000E94186E0115110519F0E801D992EACF3F
:10075000C701DF91CF911F910F91FF90EF90DF9034
:100760000C94396A4F925F926F927F928F929F9210
:10077000AF92BF92CF92DF92EF92FF920F931F93AF
:10078000CF93DF93CDB7DEB77C014DB65EB66090F8
:100790008D0C70908E0C8DB69EB66AE070E0C7012D
:1007A0000F94B05F6C018C010E191F09892B21F485
:1007B000C7010F94C25F8C01C80101962DB73EB7E7
:1007C000281B390B0FB6F8943EBF0FBE2DBF8DB757
:1007D0009EB701965C01A801B7010F94E35FF50194
:1007E000E00FF11F1082C5010E94396A81E00E946A
:1007F000186EC114D10451F076019FEFE91AF90A7D
:100800000FB6F8949EBE0FBE8DBEC5CF0FB6F8943E
:100810009EBE0FBE8DBEC3010E94396A0FB6F8940A
:100820005EBE0FBE4DBEDF91CF911F910F91FF9025
:10083000EF90DF90CF90BF90AF909F908F907F9080
:100840006F905F904F900895CF93DF93C0910913FD
:10085000C093070E81E6C89FE0011124C55FDC4EFE
:1008600080916B1180FF05C00E94CEB8CE010E941E
:10087000B16BCE010E94396A80E0DF91CF910C9478
:10088000186E08950F931F93E62FF0E0EB53F54F8A
:10089000008110E030E020E0082E04C03695279556
:1008A000179507950A94D2F700FD07C0FA018083D7
:1008B000618381E01F910F91089580E0FBCFFC01DF
:1008C0002081022E000C330B621773070CF4608337
:1008D00008958F929F92AF92BF92CF92DF92EF9244
:1008E000FF920F931F93CF93DF93EC017B018A015B
:1008F0006901FB01208131814281538168817981C5
:100900008A819B810F944567688379838A839B835F
:10091000F80120813181428153816C817D818E81FA
:100920009F810F9445676C837D838E839F83F6013F
:100930002081318142815381688579858A859B85B3
:100940000F944567688779878A879B87F70160815D
:100950007181828193819B01AC010F94DB609B01CB
:10096000AC016C857D858E859F850F9445676C876E
:100970007D878E879F87F801608171818281938155
:100980009B01AC010F94DB609B01AC016889798904
:100990008A899B890F944567688B798B8A8B9B8B9F
:1009A000F8012081318142815381F7016081718199
:1009B000828193810F94DB609B01AC016C897D89FE
:1009C0008E899F890F9445676C8B7D8B8E8B9F8B57
:1009D000F6012081318142815381F701608171816B
:1009E000828193810F94DB609B01AC01688D798DCE
:1009F0008A8D9B8D0F944567688F798F8A8F9B8F27
:100A0000F6012081318142815381F8016081718139
:100A1000828193810F94DB609B01AC016C8D7D8D95
:100A20008E8D9F8D0F9445676C8F7D8F8E8F9F8FDE
:100A300088A099A0AAA0BBA0F701C080D180E280C5
:100A4000F38020E030E0A901C701B6010F94A56949
:100A500087FF04C0F7FAF094F7F8F094A701960125
:100A6000B401C5010F94756087FD02C06401750172
:100A7000C8A2D9A2EAA2FBA28CA09DA0AEA0BFA052
:100A8000F801C080D180E280F38020E030E0A9014D
:100A9000C701B6010F94A56987FF04C0F7FAF09467
:100AA000F7F8F094A7019601B401C5010F947560A1
:100AB00087FD02C064017501CCA2DDA2EEA2FFA2F7
:100AC00020E030E040E85FE36CA97DA98EA99FA9F2
:100AD0000F9445676CAB7DAB8EAB9FABDF91CF9135
:100AE0001F910F91FF90EF90DF90CF90BF90AF904C
:100AF0009F908F900895CF92DF92EF92FF92E091B6
:100B0000FD17F091FE1720E030E0A90164817581A6
:100B1000868197810F9445676B017C0120E030E06E
:100B200040EE51E40F94756087FF06C0C12CD12CB4
:100B300080EEE82E81E4F82EC701B601FF90EF9019
:100B4000DF90CF900895CF92DF92EF92FF92E091E5
:100B5000FD17F091FE1720E030E044EB53E4608194
:100B60007181828193810F9445676B017C0120E044
:100B700030E842EB53E40F94A56918163CF4C12CFD
:100B800080E8D82E82EBE82E83E4F82EC701B60168
:100B9000FF90EF90DF90CF900895CF92DF92EF9289
:100BA000FF92E091FD17F091FE1720E030E0A901DF
:100BB00060817181828193810F9445676B017C0113
:100BC00020E030E040E450E40F94756087FF05C0FA
:100BD000C12CD12C80E4E82EFE2CC701B601FF9079
:100BE000EF90DF90CF9008952FEFFC0120832183B9
:100BF0000895861797070CF4CB010895EBE1F2E115
:100C0000808181830895681779070CF4CB010895DA
:100C100090918C0A80938C0A892F08950F931F93CB
:100C2000CF938C0120E030E040E85FE3FC0160817D
:100C30007181828193810F94446723E333E34FE012
:100C400052E40F9445672BEA33ED44E65CE30F94DE
:100C5000DB600F94B168C62F663008F0CFEF20E05C
:100C600030E040E85FE3F801648175818681978117
:100C70000F94446723E333E34FE052E40F94456756
:100C80002BEA33ED44E65CE30F94DB600F94B1682C
:100C9000962F663008F09FEF8C2FCF911F910F9108
:100CA00008958091890B882321F08091C00086FFF0
:100CB000FCCF0895FA019081981305C09181961395
:100CC00002C091E092839281992331F0458156814F
:100CD0000380F481E02D199480E00895811104C00F
:100CE00083E897E30C94B28389E897E3FBCF0F93F3
:100CF0001F93CF93DF9300D01F92CDB7DEB79C0137
:100D00000CE71CE090E1EFE5F2E0D80101900D92D4
:100D10009A95E1F7F9012081318142815381F801EF
:100D200060857185828593850F944567F80160879A
:100D300071878287938780E090E0A0EAB0E489839E
:100D40009A83AB83BC83CE0101960E94E6440F9048
:100D50000F900F900F90DF91CF911F910F910895F9
:100D60002F923F924F925F926F927F928F929F92BB
:100D7000AF92BF92CF92DF92EF92FF921F93CF93E9
:100D8000DF93CDB7DEB72C970FB6F894DEBF0FBE5A
:100D9000CDBF7A011901DC012D913D914D915C91FE
:100DA0002D833E834F835887FB01408051806280B2
:100DB000738080905F0290906002A0906102B0907A
:100DC0006202A50194016D817E818F8198850F94C7
:100DD000756081110EC011E0A30192016091630260
:100DE0007091640280916502909166020F94756023
:100DF000811110E0D1012D913D914D915C91298798
:100E00003A874B875C87F701C080D180E280F3800E
:100E1000209118023091190240911A0250911B0240
:100E2000C701B6010F947560882309F44EC0C092C3
:100E30001802D0921902E0921A02F0921B028091DD
:100E40006B0290916C02A0916D02B0916E02409184
:100E50006302509164026091650270916602809213
:100E60007C0C90927D0CA0927E0CB0927F0C4093F3
:100E7000800C5093810C6093820C7093830CC09211
:100E8000840CD092850CE092860CF092870C8093B3
:100E9000880C9093890CA0938A0CB0938B0C20E063
:100EA00030E040E05FE36091E1117091E2118091E8
:100EB000E3119091E4110F94DB6069837A838B8353
:100EC0009C83CE0101960E94E6442D813E814F8194
:100ED000588520937C0C30937D0C40937E0C50936E
:100EE0007F0C4092800C5092810C6092820C709228
:100EF000830CD1012D913D914D915C916091880CB5
:100F00007091890C80918A0C90918B0C0F9445679D
:100F10006093880C7093890C80938A0C90938B0C4F
:100F200011112FC020E030E0A90169857A858B85F9
:100F30009C850F947560811133C060E070E088EC8F
:100F400092E469837A838B839C83CE0101960E940D
:100F5000E6442C960FB6F894DEBF0FBECDBFDF91EE
:100F6000CF911F91FF90EF90DF90CF90BF90AF9007
:100F70009F908F907F906F905F904F903F902F90B9
:100F800008952AEF3EE74AE25FE36091E511709130
:100F9000E6118091E7119091E8110F94DB60D1CFB9
:100FA00060E070E080EA91E4CCCF082E000C990B51
:100FB0000D94521B2F923F924F925F926F927F92AD
:100FC0008F929F92AF92BF92CF92DF92EF92FF9259
:100FD0000F931F93CF93DF93782E662E342E422EDD
:100FE000E62EF12C36E0532EC82ED12CF701589E58
:100FF000E00DF11D1124EE0FFF1FEE0FFF1FE9564C
:10100000F34F60817181828193819B01AC010F94C8
:10101000926A882309F482C0032D070D002E000C6C
:10102000110BC42DC60D0C2E000CDD0B509EF001D3
:10103000519EF00D1124EC0FFD1FEE0FFF1FEE0F60
:10104000FF1FE956F34F80809180A280B380A501F5
:101050009401C501B4010F94926A81115FC0030D20
:10106000111D37FC1A95509EC001519E900D112400
:10107000C40DD11D47FCDA95C80FD91FCC0FDD1F59
:10108000CC0FDD1FC956D34F288039804A805B8042
:10109000A2019101C201B1010F94926A81113EC077
:1010A000A2019101C501B4010F94756087FD0CC0C8
:1010B000A5019401C501B4010F944567A2019101F6
:1010C0000F9444674B015C0186E08C9DF0018D9D7F
:1010D000F00D1124EE0DFF1DEE0FFF1FEE0FFF1F91
:1010E000E956F34F80829182A282B382662D872DCA
:1010F0000F94173481E0DF91CF911F910F91FF90F2
:10110000EF90DF90CF90BF90AF909F908F907F90A7
:101110006F905F904F903F902F90089580E0EBCFBD
:101120008F929F92AF92BF92CF92DF92EF92FF92F7
:101130000F931F93CF93DF9386EFE82E8AE3F82E69
:101140009EEFC92E9AE3D92EF70185919491FC0167
:10115000A4903296B4903197C4913296049104963B
:10116000FC0184918823F9F088248A94AC1614F445
:1011700088248394002E000C110B0C2E000CDD0B28
:10118000B016110679F19A2C9C161D0651F020E03C
:10119000482D6B2D892D0E94DA87811102C0980C91
:1011A000F3CFB394EDCF88248A94B01614F4882436
:1011B00083940C2E000CDD0B002E000C110BAC16D2
:1011C0001D0681F09B2C9016110651F0282D40E051
:1011D000692D8A2D0E94DA87811102C0980CF3CF05
:1011E000A394EDCFF2E0EF0EF11CCE14DF0409F072
:1011F000ABCFDF91CF911F910F91FF90EF90DF90D8
:10120000CF90BF90AF909F908F9008958F929F92B4
:10121000AF92BF92CF92DF92EF92FF920F931F9304
:10122000CF93DF9307E91CE0C0E07801D0E0F7013D
:1012300081909190A190B1907F01A5019401C50189
:10124000B4010F94926A811119C06701F4E0CF1ABA
:10125000D108A50194016091980A7091990A809132
:101260009A0A90919B0A0F944567F60160837183F7
:10127000828393836D2F8C2F0F941734DF5FD630CA
:10128000B1F6CF5F085E1F4FC63079F6DF91CF9180
:101290001F910F91FF90EF90DF90CF90BF90AF9094
:1012A0009F908F900895FC01618180810D94173487
:1012B000CF92DF92EF92FF920F931F93CF93DF9322
:1012C0006C0107E91CE0C0E07801D0E0F601808104
:1012D0009181A281B381F70181939193A193B193FD
:1012E0007F016D2F8C2F0F941734DF5FD63071F78D
:1012F000CF5F085E1F4FC63039F7DF91CF911F9146
:101300000F91FF90EF90DF90CF9008950F931F9370
:10131000CF93DF9300D000D01F921F92CDB7DEB7DE
:101320008B01FC0123A5211102C00F9471361D828F
:101330001E821F82188620E030E040E05FE360916B
:101340006702709168028091690290916A020F941D
:10135000456769837A838B839C839E012B5F3F4F14
:10136000AE014F5F5F4F63E672E08FE592E00E944F
:10137000B0861D821E821F82188620E030E040E089
:101380005FE3F80160857185828593850F944567D9
:1013900069837A838B839C83B8016C5F7F4F9E0146
:1013A0002B5F3F4FAE014F5F5F4FC8010E94B08679
:1013B00028960FB6F894DEBF0FBECDBFDF91CF9158
:1013C0001F910F910895CF92DF92EF92FF921F939A
:1013D000CF93DF93182F662351F01092B30A109227
:1013E000AF0A1092B00A1092B10A1092B20A0F948A
:1013F00026386B017C018091AF0A9091B00AA091D0
:10140000B10AB091B20AA7019601281B390B4A0B09
:101410005B0BDA01C901B7FD3DC02091B30A17FD8E
:1014200013C0412F012E000C550B4C5F5F4F822FD4
:10143000022E000C990B4817590764F184EF91E0D4
:10144000A0E0B0E0211724F488EE93E0A0E0B0E043
:101450008C0D9D1DAE1DBF1D8093AF0A9093B00AE9
:10146000A093B10AB093B20A2170C22F30E0D32FFB
:1014700084E28C9FB0018D9F700D7C1B11246059FC
:101480007C4F82E390E00E9405538091B30A8F5F06
:101490008093B30ADF91CF911F91FF90EF90DF907F
:1014A000CF90089520E030E040E85FE30F94446778
:1014B0002BEA33ED44E65CE30F94DB600F94E768BE
:1014C0000F94B168862F653014F084E0089567FDAD
:1014D00080E008957F928F929F92AF92BF92CF92B9
:1014E000DF92EF92FF920F931F93CF93DF9300D081
:1014F00000D01F92CDB7DEB74C015B018A0120E01E
:1015000030E040E85FE3FC0160817181828193817A
:101510000F94446723E333E34FE852E40F943F68AA
:101520006B017C0120E030E0A9010F94756087FD1C
:101530003AC020E030E040EA50E4C701B6010F9421
:10154000A5691816A4F1C701B6010F94B269762EE9
:1015500020E030E040E85FE3F4016481758186813A
:1015600097810F94446723E333E34FE852E40F94E9
:101570003F686B017C0120E030E0A9010F947560A9
:1015800087FD1CC020E030E040EA50E4C701B6010E
:101590000F94A5691816ACF4C12CD12C20EAE22EC8
:1015A00020E4F22E0EC0C12CD12C7601CCCFC12C60
:1015B000D12C30EAE32E30E4F32EC5CFC12CD12C50
:1015C0007601C701B6010F94B26979826A831B82E2
:1015D000BD82AC821F830E83CE0101965C0183E045
:1015E000C82E90E1E92E00E020E040E160E080E0DC
:1015F0000F949935811105C020E040E160E00F941F
:10160000993527960FB6F894DEBF0FBECDBFDF9198
:10161000CF911F910F91FF90EF90DF90CF90BF90EF
:10162000AF909F908F907F9008950C9417F142E0B7
:101630000C9417F1CF92DF92EF92FF920F931F93CA
:10164000CF93DF936B017A01EC01C459D54F288108
:101650003CE0389F8001399F100D112427FF24C0E2
:10166000FB011182108288818F5F888388819801B5
:10167000280F311D87FD3A95C9012091ED17F6011C
:101680002817190629F024F088818C300CF43CC00E
:1016900080819181049680349C4908F475C0F601DC
:1016A00080819181049672C088819801280F311D34
:1016B00087FD3A95C9012091ED172817190699F26F
:1016C00094F28881A801480F511D87FD5A95FA01AF
:1016D000EE0FFF1FE40FF51FEB55F84E808187FFDB
:1016E000C2CF8881F801E80FF11D87FDFA95CF017F
:1016F000EE0FFF1FE80FF91FEB55F84E808160E0F9
:101700008F770F949136AFCF808191812881A80186
:10171000420F511D27FD5A959A01FA01EE0FFF1F46
:10172000E20FF31FEB55F84E21813281820F931F98
:10173000F7019183808388819801280F311D87FDEF
:101740003A95F901EE0FFF1FE20FF31FEB55F84E2C
:10175000808187FF20C08881080F111D87FD1A95A1
:10176000F801EE0FFF1FE00FF11FEB55F84E8081DF
:1017700061E08F77DF91CF911F910F91FF90EF90F4
:10178000DF90CF900D94913680E49CE9F70191832E
:1017900080838FEF8883DF91CF911F910F91FF900E
:1017A000EF90DF90CF900895282F9091270D8330F0
:1017B00021F495FD0FC094FD0FC0892F90E0B0E09B
:1017C000A0E004C0B695A795979587952A95D2F77E
:1017D0008170089581E0089580E008958091CF0A96
:1017E0009091D00A009731F04AE050E070E060E05C
:1017F0000D94905E60E070E0CB010895FC0165916E
:1018000075918591949108959B01AC01485F5F4F5C
:10181000BC016C5F7F4F0C94B0862F923F924F9229
:101820005F926F927F928F929F92AF92BF92CF9270
:10183000DF92EF92FF920F931F93CF93DF93CDB779
:10184000DEB7A6970FB6F894DEBF0FBECDBF8C01F2
:101850001B015A87498740905F0250906002609058
:101860006102709062028090630290906402A09086
:101870006502B0906602DB018D919D910D90BC9147
:10188000A02D8B8B9C8BAD8BBE8B9C01AD01C301BE
:10189000B2010F9444676B017C01D10114968D91C4
:1018A0009D910D90BC91A02D8F8B988FA98FBA8F91
:1018B0009C01AD01C501B4010F9444676B8F7C8F0F
:1018C0008D8F9E8FA985BA858D919D910D90BC912C
:1018D000A02D8B879C87AD87BE879C01AD01C3017E
:1018E000B2010F9444676F8F78A389A39AA3A98547
:1018F000BA8514968D919D910D90BC91A02D8F87E6
:10190000988BA98BBA8B9C01AD01C501B4010F94D2
:1019100044676BA37CA38DA39EA3A7019601C70177
:10192000B6010F94DB606B017C012B8D3C8D4D8DDE
:101930005E8DCA01B9010F94DB609B01AC01C70148
:10194000B6010F9445674B015C012B893C894D8999
:101950005E896B857C858D859E850F9444672B0100
:101960003C012F89388D498D5A8D6F8578898989F9
:101970009A890F9444676B017C01A3019201C30112
:10198000B2010F94DB602B013C01A7019601C70156
:10199000B6010F94DB609B01AC01C301B2010F944F
:1019A00045670F94436A6B017C012F8D38A149A1D3
:1019B0005AA1CA01B9010F94DB602B013C012BA194
:1019C0003CA14DA15EA1CA01B9010F94DB609B014E
:1019D000AC01C301B2010F9445679B01AC01C50185
:1019E000B4010F94A5691816B4F520E030E0A90100
:1019F000C701B6010F94A56987FF2AC0C701B601C8
:101A0000905820E030E040EA50E40F94A5691816A1
:101A100014F5A10169857A85C8010E940D8CA696EE
:101A20000FB6F894DEBF0FBECDBFDF91CF911F91EF
:101A30000F91FF90EF90DF90CF90BF90AF909F906D
:101A40008F907F906F905F904F903F902F90089570
:101A5000C701B601D6CF20E030E040E050E4C50138
:101A6000B4010F94A569181624F4B101C8010E94AD
:101A7000868919821A821B821C82BE016F5F7F4F8A
:101A8000C1010E94048C2DEC3CEC4CEC5CE3C701E2
:101A9000B6010F94DB609B01AC01F801608171819C
:101AA000828193810F94DB606D837E838F8398871F
:101AB000D8019B968C919B978823C9F02AE939E934
:101AC00049E95FE314966D917D918D919C911797F3
:101AD0000F94DB6069837A838B839C83BE016F5F85
:101AE0007F4F8CE79CE00E94048CF80113A6BE0196
:101AF0006B5F7F4F89859A850E94048C90CF8C38CC
:101B0000910514F08CE890E09093FA168093F91602
:101B10000C945DF5E9E4FDE082EBDF011D928A950E
:101B2000E9F708958091DB0A811104C00E948A8D33
:101B30000C94BEEF8091BA1982FD0D945D33089527
:101B40008091490D882361F09091FA0D891308C0A6
:101B50008091BA1983FF04C087E89DE00C9488EE59
:101B600080E00895FC01238121110C94BDEA0895C1
:101B700020E030E040E85FE30F9444672BEA33ED68
:101B800044E65CE30F94DB600F94E7680F94B16860
:101B900081E0653008F080E008958F929F92AF92C7
:101BA000BF92CF92DF92EF92FF92CF93DF93EC013F
:101BB0008090280D9090290DA0902A0DB0902B0DAB
:101BC00020E030E0A901C501B4010F9475608823BD
:101BD00009F454C0C880D980EA80FB80A70196012F
:101BE000C501B4010F94756018160CF04CC020911B
:101BF000AB0A3091AC0A4091AD0A5091AE0AC701D0
:101C0000B6010F947560882331F1C092AB0AD0926F
